:100000000C94AC080C94DD080C94DD080C94DD080D
:100010000C94DD080C94DD080C94DD080C94DD08CC
:100020000C94DD080C94DD080C94DD080C94DD08BC
:100030000C94DD080C94DD080C94DD080C94224B24
:100040000C94DD080C94DD080C94DD080C94DD089C
:100050000C94DD080C94DD080C94DD080C943063DE
:100060000C94DD080C94E15C0C94B75C0C94DD08F6
:100070000C94DD080C94DD080C94DD080C94DD086C
:100080000C94DD080C94DD080C94DD080C94DD085C
:100090000C94A75D0C94175D0C945E5D0C943A4C27
:1000A0000C94DD080C94DD080C94DD080C94DD083C
:1000B0000C94DD080C94DD080C94DD080C94DD082C
:1000C0000C94DD080C94DD080C94DD080C94815C24
:1000D0000C94575C0C94DD080C94DD080C94DD083E
:1000E0000C94DD085C0A150A220A5C0A5C0A6A0A9A
:1000F000770A560A5C0A5C0A850D8A0D8F0D990DE8
:10010000A30D1C0EAD0DB50DBD0DC70DD10DDB0D35
:10011000EA0DF40D1C0EFE0D080E120E171009103C
:100120000910171017101B1029102910171017107D
:100130002315FE143E153E153E153E153E153E1583
:100140003E153E153E158C115B147C147514661417
:100150003E153E153E153E153E153E153E15121533
:10016000231B171B171B231B231BFE1A0B1B0B1B0D
:10017000231B231BAA2997299729AA29AA29AA2937
:10018000B529B529AA29AA2993349634AE34C534A1
:100190000E3521354135CC3ACC3ACC3ACC3AC93A35
:1001A000C93AD03AD03AD03AD03AD03AD03AD03A06
:1001B000D03AC93AC93AD03AD03AD03AD03AD03AFD
:1001C000CE3ACC3A10620C620C621062106210627D
:1001D0001962DA6110621062736276626562696246
:1001E0006F62AD627A627E62846288628C629262C1
:1001F00096629A62AD62A062A462A8620763423608
:10020000B79BD8A71A39685618AEBAAB558C1D3CA7
:10021000B7CC5763BD6DEDFD753EF6177231BF006B
:100220000000803F08000000BE922449123EABAAA5
:10023000AA2ABECDCCCC4C3E00000080BEABAAAA00
:10024000AA3E00000000BF000000803F0000000048
:1002500000084178D3BB4387D1133D190E3CC3BD81
:100260004282AD2B3E68EC8276BED98FE1A93E4C2E
:1002700080EFFFBE01C4FF7F3F00000000000C9430
:1002800093340C949A620C94B8430C94080E0C941A
:100290001B320C9496340C9480470C94065F0C949B
:1002A000BF460C94A8430C947E620C9474450C9445
:1002B000A8620C9407470C948A430C94AD620C948A
:1002C000525A0C9419620C945E4A0C9480480C9417
:1002D000CE3A0C94A4620C948A0D0C9468320C945F
:1002E00075140C940C620C94AE340C9496620C94BD
:1002F00065620C94704E0C947A620C94105A0C94B3
:1003000052330C9480330C94015F0C94AA290C9402
:10031000A0620C9499360C9476620C946F620C94E3
:1003200027460C94DE460C9421350C94770A0C94E5
:10033000D03A0C9466140C9488620C94055F0C946B
:10034000F85A0C94C62E0C94B24F0C9411480C948D
:10035000B50D0C94014F0C9402320C94FE0D0C94CC
:10036000AD0D0C94E7480C9497490C94C7480C9435
:10037000DF080C94C26B0C94D4320C94171B0C94B1
:10038000D5430C9490440C94150A0C94B1490C94E8
:10039000B5590C94CC3A0C94990D0C94F65A0C94D3
:1003A000025A0C94D10D0C94164F0C947C140C949E
:1003B000850D0C944D490C945C500C94231B0C94AB
:1003C00029100C941B100C94E9480C94FE140C9406
:1003D00082450C940E350C9473620C943D5B0C9426
:1003E0005F490C9493490C945A320C94C9530C9461
:1003F000602B0C9447490C94F04F0C944A490C9490
:100400001C0E0C9441350C94BD0D0C94A0430C941F
:10041000120E0C94D4430C94DB4E0C9410620C948A
:10042000E44E0C940C320C94B5290C94FE1A0C94E6
:1004300063330C94A4430C9438320C94A5320C947E
:10044000CD320C94A30D0C945B140C94DA610C94D3
:100450008C620C940B1B0C94C93A0C94095F0C949D
:10046000DB0D0C94DD480C94A01F0C94220A0C9414
:1004700097290C945C2B0C9454490C9470490C945F
:1004800084620C9489430C945C0A0C949F5A0C94DB
:10049000642B0C94560A0C9493320C9490330C9465
:1004A000AD470C946E500C946A0A0C94C5340C94AD
:1004B00012150C94D3490C948F0D0C9469620C9412
:1004C0008C110C94EE590C941B5B0C9417100C942B
:1004D000F40D0C94DD330C9423150C94C70D0C947F
:1004E000CC430C943E150C9409100C94EA0D0C941A
:1004F000DF590C941B440C94C1430C94D11B0C94F5
:1005000092626364696E6F70737578585B003D002A
:100510005643230020636D643D003D0056435F68F1
:1005200065617423003D0050696E3A003D005069DA
:100530006E3A002048616C7465640A003D005265A3
:1005400073746F7265643A20003A204E6F207374A2
:100550006F7265642076616C756573202D2064650B
:100560006661756C740A00466F726365205768692E
:1005700074650A00416C7265616479204163746935
:1005800076650A005475726E696E6720584F4E0A80
:1005900000584F464620736B69707065642E20507A
:1005A00072657620636D643A005475726E656420DE
:1005B0006F66662066726F6D3A00526573746F7273
:1005C00065642066726F6D3A003E20003C0020504A
:1005D00061723D200020436D643D00205375623DF3
:1005E00000204974656D3D0052414D3D00476F74D8
:1005F00020495020616464726573733A0027697002
:10060000205B69705B2C646E735B2C67775B2C736B
:1006100075626E65745D5D5D5D27202D2073657468
:10062000207374617469632049500A004661696CE3
:10063000656420746F20636F6E66696775726520EC
:1006400045746865726E6574207573696E672044C1
:100650004843502E20596F752063616E2073657476
:10066000206970206D616E75616C6C792100537426
:10067000617274696E67206C616E00246E6F6465D0
:10068000730024666F726D61740024646174617418
:1006900079706500302D31303000696E74656765A2
:1006A000720068737600636F6C6F72004F4E2C4F50
:1006B00046462C48414C542C524553542C584F4ECE
:1006C0002C584F46462C544F47474C4500656E7595
:1006D0006D00666C6F617400322E312E300024681C
:1006E0006F6D696500757074696D652C66726565FE
:1006F0006865617000323066613432375F323031A4
:10070000392D30362D3131004C6967687448756277
:100710002000246E616D650072656164790020744B
:10072000727920616761696E20696E20352073657A
:10073000636F6E6473006661696C65642C2072631C
:100740003D004177616974696E6720666F7220723F
:10075000657461696E656420746F706963730063AA
:100760006F6E6E65637465642061732000202E2EA9
:100770002E0020757365723A003A000A4174746560
:100780006D7074696E67204D51545420636F6E6EA6
:10079000656374696F6E20746F20002473746174D4
:1007A0006500646973636F6E6E656374656400559C
:1007B00073696E67204D5154542070617373776F65
:1007C00072642066726F6D20636F6E6669670044A5
:1007D0006576696365204E616D653A0052656269B0
:1007E0006E6420737563636573732E2049502061B6
:1007F0006464726573733A004572726F723A207264
:100800006562696E64206661696C0052656E657729
:10081000656420737563636573732E20495020618E
:100820006464726573733A004572726F723A207233
:10083000656E65776564206661696C004E6F206C3B
:10084000696E6B00416363657074696E6720636FE6
:100850006D6D616E64732E2E2E0A003E3E3E004E7C
:100860006F204D414320636F6E66696775726564E2
:100870003A20736574206669726D776172652773BB
:10088000204D41430A004D6F6462757320706F6C98
:100890006C696E67206572726F723D002D0020508A
:1008A000492056616C203A004D6F64627573207068
:1008B0006F6C6C696E67206572726F723D002D00FF
:1008C00020464D2056616C203A004D6F646275736E
:1008D00020706F6C6C696E67206572726F723D007C
:1008E0002056616C3A20004D423A20004E6F742031
:1008F000737570706F7274656420726567207479A7
:1009000070650A00496C6C6567616C20617267757F
:100910006D656E74730A00757074696D650066723A
:1009200065656865617000247374617473002000EC
:1009300020000A52414D3D00202D7461726765749C
:10094000207A6F6E652D00204F464600204F4E00E6
:10095000204F46460020636D643A00204375723A8A
:1009600000205365743A0020457870697265640A06
:10097000002F00496E3A20003D00494E3A0068655C
:10098000617400766F6C00706F77657200736574C8
:10099000706F696E74006D6F64650074656D7000D2
:1009A00073657400536574436D643A002056616C3E
:1009B0003D002053746F7265200072676200687397
:1009C0007600444543524541534500494E43524504
:1009D0004153450066616C7365007472756500581B
:1009E0004F464600584F4E0048414C5400544F4724
:1009F000474C450052455354004F4646004F4E0069
:100A000054787432436D643A005265747279696E39
:100A10006720434D440A004E6F7420737570706FE9
:100A2000727465642072656720747970650A0029A4
:100A30003A0028543A003D3E004D6F6462757320C1
:100A40006F70206661696C65640A00636F756C6421
:100A5000206E6F742070617273653A200055706467
:100A6000617465640A002B002D00485454502F31E6
:100A70002E312025690020485454502F312E310D3D
:100A80000A486F73743A2025730D0A4163636570D9
:100A9000743A202A2F2A0D0A436F6E6E65637469BB
:100AA0006F6E3A20636C6F73650D0A00257300202A
:100AB000000D0A00474554006661696C6564207446
:100AC0006F20636F6E6E6563740A004552524F5219
:100AD0003A205365727665722072657475726E6520
:100AE000642000446F6E652E0A004170706C796955
:100AF0006E672E0A00436F6E6669672070617273BD
:100B0000696E67206661696C65640A00676F7420AE
:100B1000436F6E6669670A00436F6E6669672055AA
:100B200052493A20687474703A2F2F006C617A79B8
:100B3000686F6D652E7275000A282D295245535431
:100B40004152545F4C414E5F4F4E5F4D5154545F84
:100B50004552524F5253000A282D294841524452BF
:100B6000455345542C207573696E6720736F667406
:100B7000000A282D29434F554E544552000A282D6E
:100B800029444854000A282D294F57495245000A44
:100B9000282B294D4F44425553000A282B29444DF8
:100BA00058000A282B294453323438322D31303042
:100BB000000A282B294672656552616D20707269A2
:100BC0006E74696E670064653A61643A62653A659D
:100BD000663A66653A6564000A4669726D776172C5
:100BE00065204D4143204164647265737320006C3D
:100BF000617A79686F6D652E7275000A436F6E6653
:100C00006967207365727665723A000A282B295746
:100C100041544348444F47003230313130334C0067
:100C200020432B2B2076657273696F6E3A00323049
:100C300066613432375F323031392D30362D313103
:100C4000000A4C617A79686F6D652E7275204C6967
:100C500067687448756220636F6E74726F6C6C6540
:100C6000722000000020002300260029002C002F05
:100C7000003200000100000301060109013D0049A6
:100C80004E3A0000002200250028002B002E0031E3
:100C900000340002010000050108010B0100000AF8
:100CA0000B02090C0D0E08070304010000000000F0
:100CB0000000000000000000000000000000000034
:100CC00000000000000000000012111000000000F1
:100CD0000000000000000000000000000000000014
:100CE00000000000002100240027002A002D003011
:100CF00000330001010000040107010A0101021094
:100D00002020080810204010204080020102010825
:100D100004020101020408102040808040201008D5
:100D2000040201800402018040201008040201082E
:100D3000040201010204081020408001020408108E
:100D4000204080050505050705080808080202027D
:100D5000020A0A0808040404040101010101010156
:100D6000010303030303030303040707070C0C0C2D
:100D70000C0C0C0C0C020202020606060606060605
:100D8000060B0B0B0B0B0B0B0B696E00735F6F7578
:100D900074006D79686F6D6500436F6E6E65637486
:100DA00065642E00436F6E6E2E2061626F727465F3
:100DB000640043757272656E74204C414E20636FFF
:100DC0006E6669672869702C646E732C67772C7364
:100DD00075626E6574293A000A55736520746865FA
:100DE000736520636F6D6D616E64733A202768656B
:100DF0006C7027202D207468697320746578740ADC
:100E0000276D61632064653A61643A62653A65669C
:100E10003A66653A3030272073657420616E64202D
:100E200073746F7265204D41432D61646472657304
:100E30007320696E20454550524F4D0A2769702036
:100E40005B69705B2C646E735B2C67775B2C7375CE
:100E5000626E65745D5D5D5D27202D207365742075
:100E60007374617469632049500A2773617665273A
:100E7000202D207361766520636F6E666967206937
:100E80006E204E5652414D0A2767657427205B63DA
:100E90006F6E66696720616464725D27202D20672C
:100EA000657420636F6E6669672066726F6D20706F
:100EB00072652D636F6E6669677572656420555241
:100EC0004C20616E642073746F726520616464727B
:100ED0000A276C6F616427202D206C6F616420638A
:100EE0006F6E6669672066726F6D204E5652414D77
:100EF0000A2770776427202D20646566696E652057
:100F00004D5154542070617373776F72640A276B6C
:100F1000696C6C27202D207465737420776174636D
:100F200068646F670A27636C65617227202D2063F0
:100F30006C65617220454550524F4D0A27726562BB
:100F40006F6F7427202D207265626F6F7420636F3E
:100F50006E74726F6C6C657200536F66742072658C
:100F6000626F6F74696E672E2E2E00444D58696E45
:100F70002042756666657220616C6C6F63206572D5
:100F80007200496E697420696E2063683A005241AC
:100F90004D3D000A6D71747420000A6D6F646275B6
:100FA0007320000A696E7075747320000A69746595
:100FB0006D7320000A436F6E666967757265643AE7
:100FC000002C003D0050696E3A002C003D4C4F57FC
:100FD00000546865726D6F3A00444D58206F757407
:100FE00020737461727465642E204368616E6E654F
:100FF0006C733A2000444D5820696E2073746172FE
:101000007465642E204368616E6E656C733A004CA3
:101010006F61646564006C6F6164206661696C6512
:1010200064004E6F2073746F72656420636F6E6628
:101030006967004C6F6164696E6720436F6E666913
:10104000672066726F6D20454550524F4D000A7201
:10105000657175657374204D51545420436F6E66ED
:10106000696700536176656420746F20454550526E
:101070004F4D00536176696E6720636F6E666967D6
:1010800020746F20454550524F4D2E2E00536176EF
:1010900065640A005365742064796E616D6963202C
:1010A00049500A00454550524F4D20636C656172AE
:1010B00065640A0050617373776F726420757064A1
:1010C000617465640A002C20002E003E3E20004919
:1010D0006E76616C696420636F6D6D616E64004152
:1010E00063746976650A0047727020636865636B94
:1010F0003A0A002D3E005075623A2000556E6B6E24
:101100006F776E20636D64200A0053746174757389
:101110002064656666657265640A00206973200054
:1011200044656C6574696E6720636F6E662E20522D
:10113000414D207761733A00536B697070696E6737
:101140002E2E004F4F4D21005D20000A5B003A001B
:101150004D41433A0000C26B11241FBECFEFD1E2D4
:10116000DEBFCDBF00E00CBF15E0A0E0B2E0E8EECE
:10117000F9EF00E00BBF02C007900D92AE33B1074C
:10118000D9F72BE0AEE3B5E001C01D92AB35B20755
:10119000E1F718E0CCEAD8E000E006C021970109A9
:1011A000802FFE010E94D177CB3AD10780E008075B
:1011B000A9F70E947A630C94F27C0C9400002F92A1
:1011C0003F924F925F926F927F928F929F92AF92D7
:1011D000BF92CF92DF92EF92FF920F931F93CF9324
:1011E000DF93CDB7DEB769970FB6F894DEBF0FBEB9
:1011F000CDBF6C012B011A015901088BFD8AEC8AC5
:10120000DC011296ED91FC911397008111810E94EF
:10121000544E3B014C0168EE75E08DEB97E00E9467
:101220007B5B2AE0B401A3018DEB97E00E94B45BE5
:1012300061EE75E08DEB97E00E947B5BB8018DEB72
:1012400097E00E94495C6BED75E08DEB97E00E94A2
:101250007B5B6C897D898DEB97E00E94003865EDA2
:1012600075E08DEB97E00E947B5BB2018DEB97E020
:101270000E9400386EEC75E08DEB97E00E947B5B7E
:10128000F60182819381892B09F450C61B861A8648
:101290001D861C861F861E86A114B10459F1850186
:1012A0004E01FAE08F0E911CE12CF12CE214F304B4
:1012B0000CF523E0E216F104E9F0D801AD90BD9001
:1012C0008D01F401A192B1924F016CEC75E08DEBB0
:1012D00097E00E947B5BB5018DEB97E00E940038A0
:1012E00069EC75E08DEB97E00E947B5BFFEFEF1AF6
:1012F000FF0ADCCF8DEB97E00E94455C60E070E078
:10130000C6010E9497203C0124E04216510451F08E
:1013100037E04316510459F183E04816510409F0AF
:1013200053C007C0C6010E949D61892B09F025C1E9
:1013300002C6D60118968C91873009F41AC360E072
:10134000C6010E94EA20853009F0F2C56AEB75E01B
:101350008DEB97E00E947B5B65E070E08DEB97E0A2
:101360000E9400388DEB97E00E94455CE4C5F601D1
:101370008085873009F4FDC260E0C6010E94EA2042
:10138000082F10E0863081F469EA75E08DEB97E074
:101390000E947B5BB8018DEB97E00E9400388DEBDB
:1013A00097E00E94455CE9C061E975E08DEB97E04C
:1013B0000E947B5BB8018DEB97E00E9400388DEBBB
:1013C00097E00E94455CB4C5F2E04F16510409F461
:1013D000D4C04CF44114510489F031E04316510457
:1013E00009F014C1A7C085E04816510409F4E6C00D
:1013F00096E04916510409F485C008C1D601189633
:101400008C91853021F06EE0C6010E94C520F60166
:10141000808590E08A30910508F069C0FC0188273A
:10142000EE58FF4F8F4F0C94D1778C859D85892B7B
:1014300049F4F3E02F16310491F48FE7D6011896A2
:101440008C9304C0B3E02B16310449F44A855B85C4
:101450000C851E85B801C6010E943B2018C0C6013C
:101460000E9473207B01182F0A85AB01682F702F13
:10147000C6010E943B20EA86FB86812F110F990B43
:101480009D878C87802F000F990B9F878E87E88917
:10149000EE2351F101E09E01265F3F4F43E050E013
:1014A00060E070E0C6010E9499601EC04A855B85BD
:1014B0000C851E85B80114C0F889FF2359F001E09E
:1014C0009E01265F3F4F41E050E060E070E0C601C2
:1014D0000E9499604A855B85052E000C660B770B90
:1014E000C6010E943B2003C013E0212E312C0E9434
:1014F000246360933E0570933F058093400590936D
:10150000410584C0C6010E949D61892B39F464E8BD
:1015100075E08DEB97E00E947B5B0CC064E775E0A3
:101520008DEB97E00E947B5BD60118968C918730FB
:1015300009F0FEC4F6018085813009F026C560E01F
:10154000C6010E94EA20813009F01FC50E94246371
:1015500000913E0510913F052091400530914105D5
:10156000DC01CB01801B910BA20BB30B853F91409B
:10157000A105B10508F0E3C408C560E0C6010E94FA
:10158000EA208530B9F01B861A861D861C861F86C8
:101590001E8662E0C6010E94C520F889FF2351F033
:1015A00000E020E030E040E050E062E070E0C601A2
:1015B0000E949960A2E04A2E512C28C0C6010E94C8
:1015C0009D611816190614F51B861A861D861C8641
:1015D0001F861E8660E0C6010E94EA20863011F454
:1015E00062E001C065E0C6010E94C52000E020E085
:1015F00030E040E050E062E070E0C6010E94996097
:1016000063E375E08DEB97E00E947B5BEC84FD84E7
:10161000C7010F2C000CAA0BBB0B8E8B9F8BA88FC6
:10162000B98FAE85BF85BB8BAA8B2FEF30E00E94B0
:10163000E877F4E68F2E912CA12CB12CA501940112
:101640000E9490778901F6018085843009F47FC17A
:1016500050F4813009F44CC0F0F1823089F18330CC
:1016600009F4EFC162C4883009F497C338F48630B6
:1016700009F4A7C1873009F058C47BC1893009F447
:10168000FFC28F3709F051C460E0C3010E940E4CC5
:1016900060E0C30101960E940E4C60E0C301029617
:1016A0000E940E4CAE85BF852FEF30E00E94E87798
:1016B000A50194010E949077622FC301039644C153
:1016C0002FEF30E0D7010E94E877A50194010E9436
:1016D0009077D22E78C0AA85BB852FEF30E00E948C
:1016E000E877A50194010E949077622FC3012CC175
:1016F00093012D5F3F4F290132E3E316F1040CF013
:1017000049C082E390E08E199F09EA89FB898E9F88
:10171000D0018F9FB00D9E9FB00D11242FEF30E0B0
:101720000E94E87728E833E140E050E00E9490779B
:10173000622FC2010E940E4CEC84FD842EEF31E03A
:10174000D7010E94E877E2E32E2E312C412C512C58
:10175000A20191010E949077AE85BF850E94E0773B
:10176000A50194010E94907749015A019701A5E6CD
:10177000BFEF0E94E077A20191010E949077DD24E3
:10178000DA94D20E84010F3F1105E9F0E4F00FEF77
:1017900010E019C02E893F89488D598D2253310997
:1017A00041095109ABE9B0E00E94AF7722E330E094
:1017B00040E050E00E94907764E6D62ED20E60E0C2
:1017C000C2010E940E4CAA85BB852FEF30E00E941B
:1017D000E8772DE631E040E050E00E949077322F2C
:1017E000122F1F71110F110F812F880F15E5682F10
:1017F000619F060E60E0611D1124922F907420728B
:1018000037FD24C091110CC0211104C0862F809592
:10181000F62E14C055E5F52EF60E10E06BEA36C034
:1018200021110FC0182F3AEA139F010E10E0111D6D
:1018300011248BEA811B4AEAF42EF60E682F10E081
:1018400025C080E0F62EF094162F0FC0911112C023
:1018500021110DC0182F2AEA129F010E10E0111D50
:1018600011243BEAF32EF11A1B5A60E00FC0162F29
:1018700010950BC0211104C085E5860F1BEA03C03B
:101880008AEA860F90E0161B682FF12CFFEFDF1617
:1018900009F42AC0DD2009F423C0662329F02D2D88
:1018A000629F060E60E0611DFF2039F03F2D2D2D57
:1018B000329F030E30E0311DF32E112329F03D2D10
:1018C000139F010E10E0111D11242D2D2095229F34
:1018D000020E20E0211D1124620FF20E120F04C02F
:1018E0001FEFFF24FA946FEF0F3F09F422C020E0AE
:1018F000002321F0009F212D09F02F5F2223B1F05A
:10190000662321F0629F060E60E0611DFF2031F02A
:101910003F2D329F030E30E0311DF32E112321F0B5
:10192000129F010E10E0111D112403C010E0F12CD4
:1019300060E0C3010E940E4C6F2DC30101960E940E
:101940000E4C612FC30102960E940E4CEEC2E48041
:10195000F580F7018085853009F0E7C2C7010E9454
:10196000BC3BA82EB12CF2E0AF16B1040CF02BC496
:10197000DCC2D6011496ED91FC91159780858530D7
:1019800009F0D3C2C680D780C114D10409F4CDC2F6
:10199000F60161857285CE0101960E945626EC887B
:1019A000FD8808899E01265F3F4FA101B201CE014B
:1019B00001960E94DF08D6011296CD90DC90139715
:1019C000E3CF77FE06C071946194710801E010E0E6
:1019D00002C000E010E0F62C61E0862D0E94AE62AD
:1019E000012B69F0B1E04B16510429F061E0E6E00B
:1019F0004E16510409F460E0062F10E011C0F1E02A
:101A00004F16510451F091E080E026E04216510457
:101A100009F090E0092F182F02C001E010E0602FBC
:101A20008F2D0E94AA416EE275E08DEB97E00E9437
:101A30007B5BB3018DEB97E00E9400386CE275E0B0
:101A400011C177FE06C071946194710801E010E045
:101A500002C000E010E0F62C61E0862D0E94AE622C
:101A60008091A100887F8093A10080919100887F60
:101A7000809391008091A10082608093A100809169
:101A80009100826080939100AA85BB85012B99F01B
:101A9000CD01BB0FAA0BBB0B9C01AD012456310934
:101AA00041095109AFEFB0E00E94AF772CE93FEF59
:101AB0004FEF5FEF08C02FEF30E00E94E87724E699
:101AC00030E040E050E00E949077890161E08F2D86
:101AD0000E94AE620115110509F4B1C00F3F110556
:101AE00009F4AFC0F301FF27E356F34FE4918E2FC3
:101AF00090E0FC013197E231F10508F09DC08827A4
:101B0000E458FF4F8F4F0C94D17784B5806884BD23
:101B100007BD9BC084B5806284BD08BD96C080911E
:101B20008000806880938000109389000093880073
:101B30008CC08091800080628093800010938B0025
:101B400000938A0082C0809180008860809380002A
:101B500010938D0000938C0078C08091B000806855
:101B60008093B0000093B30070C08091B000806299
:101B70008093B0000093B40068C0809190008068AA
:101B80008093900010939900009398005EC080911C
:101B9000900080628093900010939B0000939A00C5
:101BA00054C08091900088608093900010939D00B5
:101BB00000939C004AC08091A00080688093A000A0
:101BC0008091A0008F7B8093A0001093A9000093C8
:101BD000A8003BC08091A00080628093A000109379
:101BE000AB000093AA0031C08091A0008860809370
:101BF000A0001093AD000093AC0027C0809120019D
:101C000080688093200110932901009328011DC052
:101C10008091200180628093200110932B0100931A
:101C20002A0113C0809120018860809320011093C5
:101C30002D0100932C0109C00038110514F460E057
:101C400001C061E08F2D0E94AA4167E275E08DEB33
:101C500097E00E947B5BB3018DEB97E00E94003818
:101C600065E275E08DEB97E00E947B5BB8018DEB40
:101C700097E00E9400388DEB97E00E94455C55C1CB
:101C80001A8560E070E0C6010E949720082FF92EA7
:101C900060E175E08DEB97E00E947B5B602F7F2D0C
:101CA0008DEB97E00E9400386EE075E08DEB97E0D9
:101CB0000E947B5B612F012E000C770B8DEB97E070
:101CC0000E9400388DEB97E00E94455C80910B06E6
:101CD00090910C06892B89F069E37AE08DEB97E00F
:101CE0000E947B5B642D6064C6010E94C520412F69
:101CF000110F550B660B770BB0C081E090E090930D
:101D00000C0680930B0626E040E855E260E070E0A8
:101D100080E297E00E94A03800930B0980E297E0F0
:101D200090930A09809309091092160A1092180AD2
:101D30001092170A80ED97E0909391098093900993
:101D40001092930910929209112339F085E090E0E6
:101D5000909395098093940904C01092950910926C
:101D6000940986E00E94053962E370E080E090E02B
:101D70000E94EA6282ED97E0909391098093900926
:101D8000109293091092920934E61302A0011124D3
:101D90005093950940939409C1C00480F581E02DCA
:101DA00061857285CE0101960E945626CE0101966C
:101DB0000E942E20882309F4B8C08985893009F053
:101DC000B4C0142DEA8460E070E0CE0101960E9458
:101DD0009720082FF92E6CE175E08DEB97E00E94BB
:101DE0007B5B602F7F2D8DEB97E00E9400386AE1CE
:101DF00075E08DEB97E00E947B5B6E2D0E2C000C46
:101E0000770B8DEB97E00E94003864E175E08DEB75
:101E100097E00E947B5B642D042C000C770B8DEB0C
:101E200097E00E9400388DEB97E00E94455C80911E
:101E30000B0690910C06892BA1F069E37AE08DEBFB
:101E400097E00E947B5B642D6064C6010E94C52000
:101E50004E2DEE0C550B660B770BC6010E943B20F6
:101E600064C081E090E090930C0680930B0626E01E
:101E700040E855E260E070E080E297E00E94A03820
:101E800000930B0980E297E090930A098093090977
:101E90001092160A1092180A1092170A123009F4BA
:101EA000F7C1153009F4F4C16E2DEE0C770B880BD9
:101EB000990B0E940B7922E538EB42E152E40E9433
:101EC000F07720E030E040E251E40E94C0792DEE4E
:101ED0003EE94CE35EE30E9461786B017C0120E007
:101EE00030E0A9010E94BB7920E030E040E05FE3F0
:101EF00087FDC9C1C701B6010E94F0770E94D3785F
:101F000083ED97E090939109809390091092930943
:101F100010929209709395096093940986E00E944B
:101F2000053910920C0610920B06B5C18FEF01C057
:101F30008DEF9FEFB0C144244394512CFBCA67E658
:101F400075E08DEB97E00E947B5B8FE7F601808761
:101F50001D861C8684E690E09F878E874A855B8578
:101F600060E074E6C6010E943B20F889FF2309F473
:101F70004DCB00E09E01265F3F4F43E050E060E024
:101F800070E0C6010E94996041CB642DC6010E9499
:101F9000C520C6010E947320F62EE72E8C01D601C3
:101FA00018962C91233008F0FCC0213070F46A3070
:101FB0007105810591052CF4B2E3FB2EE12C00E0C4
:101FC00010E04F2D5E2D602F0AC06115710581054F
:101FD000910519F01A300CF412E3AB01682F712F40
:101FE000C6010E943B204F2D5E2DB8011416150628
:101FF00016061706E4F5D60118968C9190E08A3003
:10200000910538F5FC018827E257FF4F8F4F0C945C
:10201000D177C7019A878B87802F000F990B9D87F7
:102020008C87812F110F990B9F878E8753C05B87F9
:102030004A8701E07FC05B874A87B889BB2309F4E0
:10204000E5CA00E020E030E040E050E061E070E010
:102050000AC0E889EE2309F4A8C000E020E030E0DF
:1020600040E050E0B201C6010E9499609EC02AE0A3
:1020700030E08DEB97E00E94FD5B69E475E08DEB4D
:1020800097E00E947B5BD60118968C918530C9F051
:10209000A0F48150823008F041C084E690E09B8734
:1020A0008A871D861C869F878E8744E650E060E005
:1020B00074E6C6010E943B200DC08630C9F088300E
:1020C00069F584E190E09B878A8744E150E060E015
:1020D00070E02CC001E09E01265F3F4F43E050E0DE
:1020E00060E070E0C6010E94996003E010E02EC03D
:1020F00084E690E09B878A8744E650E060E070E0E9
:10210000C6010E943B20B889BB23F1F000E020E02B
:1021100030E040E050E061E070E013C084E690E021
:102120009B878A8744E650E060E070E0C6010E9429
:102130003B2000E09E01265F3F4F41E050E060E021
:1021400070E0C6010E94996001E010E05E01EAE0E3
:10215000AE0EB11CE12CF12CD5018D909D905D014E
:102160006EE375E08DEB97E00E947B5BB7018DEB32
:1021700097E00E9400386CE375E08DEB97E00E94D9
:102180007B5BB4018DEB97E00E9400388DEB97E00C
:102190000E94455CBFEFEB1AFB0A0E151F05E1F626
:1021A00004C0243009F403CF1ECFF60180858130AE
:1021B00009F02CCA8C859D85892B09F027CA8FE7E9
:1021C000F601808723CA60E0C7010E941A38DC014B
:1021D00019968D919C911A97998B888B61E0C70114
:1021E0000E941A38FC0141845284638474842A84D6
:1021F0003B84F2E0AF16B104E9F162E0C7010E944E
:102200001A38DC0119960D911C911A97B3E0AB16A0
:10221000B10491F163E0C7010E941A38FC01818486
:102220009284F4E0AF16B10451F064E0C7010E945B
:102230001A38DC011996AD90BC901A9703C032E0B1
:10224000A32EB12C8114910461F09401D1010E945C
:10225000E07724E630E040E050E00E94907779019A
:1022600001C071019501A20168897989C6010E94A6
:1022700072265BCE0FEF1FEF8FE3882E912C92E03A
:10228000A92EB12CE2CFC701B6010E94EF7736CE5E
:1022900060E070E035CE69960FB6F894DEBF0FBEF1
:1022A000CDBFDF91CF911F910F91FF90EF90DF9005
:1022B000CF90BF90AF909F908F907F906F905F90E6
:1022C0004F903F902F9008954F925F926F927F9220
:1022D0008F929F92AF92BF92CF92DF92EF92FF9236
:1022E0000F931F93CF93DF93CDB7DEB7C15AD14081
:1022F0000FB6F894DEBF0FBECDBFE091AE05F091F2
:10230000AF053B96E831F10508F0B8C38827E856D9
:10231000FF4F8F4F0C94D1770E94246300910F06DA
:10232000109110062091110630911206061717071A
:102330002807390708F0A2C301E213E0CF56DE4FA9
:1023400019830883C159D140CD56DE4F18821982B6
:102350001A821B82C359D140CF57DE4F198308839D
:10236000C158D140CD57DE4F188219821A821B8284
:10237000C358D140CF59DE4F19830883C156D1408D
:10238000CD59DE4F188219821A821B82C356D14062
:10239000CF5BDE4F19830883C154D140CD5BDE4F44
:1023A000188219821A821B82C354D1406EE676E0ED
:1023B0008DEB97E00E947B5BBE016F567E4F86E0FF
:1023C00090E00E949F3E892B09F467C16EE773E09D
:1023D0008DEB97E00E94495C1A830983CD56DE4F4E
:1023E00088819981AA81BB81C359D1408B839C8309
:1023F000AD83BE83CE0101960E944E56BE016F573B
:102400007E4F8AE090E00E949F3E892B09F42EC106
:1024100064E973E08DEB97E00E94495C1A830983BD
:10242000CD57DE4F88819981AA81BB81C358D140A5
:102430008B839C83AD83BE83CE0101960E944E5652
:10244000BE016F597E4F8EE090E00E949F3E892B27
:1024500009F4DFC06AE973E08DEB97E00E94495C04
:102460001A830983CD59DE4F88819981AA81BB8166
:10247000C356D1408B839C83AD83BE83CE0101962E
:102480000E944E56BE016F5B7E4F82E190E00E943B
:102490009F3E892B09F477C06FE973E08DEB97E0DD
:1024A0000E94495C1A830983CD5BDE4F8881998144
:1024B000AA81BB81C354D1408B839C83AD83BE83EF
:1024C000CE0101960E944E561A830983CD5BDE4FE2
:1024D00088819981AA81BB81C354D1408B839C831D
:1024E000AD83BE83CF57DF4F19830883C158D040D7
:1024F000CD59DE4F88819981AA81BB81C356D140D5
:10250000CD57DF4F88839983AA83BB83C358D040BC
:10251000CF53DF4F19830883C15CD040CD57DE4FC6
:1025200088819981AA81BB81C358D140CD53DF4FA7
:1025300088839983AA83BB83C35CD040CF5FDE4F7F
:1025400019830883C150D140CD56DE4F88819981CF
:10255000AA81BB81C359D140CD5FDE4F8883998367
:10256000AA83BB83C350D1409E012F5F3F4FAE0172
:102570004F575F4FBE016F537F4FCE018F5F9E4F0E
:102580000E94694285C01A830983CD59DE4F888134
:102590009981AA81BB81C356D1408B839C83AD8333
:1025A000BE83CF57DF4F19830883C158D040CD5722
:1025B000DE4F88819981AA81BB81C358D140CD5714
:1025C000DF4F88839983AA83BB83C358D040CF53FE
:1025D000DF4F19830883C15CD040CD56DE4F888120
:1025E0009981AA81BB81C359D140CD53DF4F8883E4
:1025F0009983AA83BB83C35CD040AE014F5F5F4F1A
:10260000BE016F577F4FCE018F539F4F0E94B5423F
:102610003FC01A830983CD57DE4F88819981AA81F3
:10262000BB81C358D1408B839C83AD83BE83CF577E
:10263000DF4F19830883C158D040CD56DE4F8881C3
:102640009981AA81BB81C359D140CD57DF4F88837F
:102650009983AA83BB83C358D040BE016F5F7F4F6D
:10266000CE018F579F4F0E94074312C01A830983E0
:10267000CD56DE4F88819981AA81BB81C359D14053
:102680008B839C83AD83BE83CE0101960E9452430F
:102690008DEB97E00E94455C0BC166EA73E08DEB21
:1026A00097E00E94495C0FB6F894A895809160006D
:1026B000886180936000109260000FBE8091A00539
:1026C000811107C085E895E00E94764481E08093FF
:1026D000A00582E495E090936708809366080E94C5
:1026E000D941CE0101960E94752A89819A810E9462
:1026F000D04946E050E06DE97AE089E090E00E9440
:10270000863781E293E09A8389831B821C821D8233
:102710001E82CE0103960E94BA490E94CF49809141
:10272000660890916708DC0192961D921D921D9299
:102730001C929597FC0116A217A210A611A69A96B4
:102740001D921D921D921C929D9740EE5EE260E0EC
:1027500070E046AB57AB60AF71AF40EA5FE060E05E
:1027600070E0DA964D935D936D937C93DD973E9682
:1027700024E1DF011D922A95E9F726E0EDE9FAE070
:10278000DC01189601900D922A95E1F7FC01EE5BB1
:10279000FF4F10820E94D23C8C01019709F04AC081
:1027A000CE0101960E94752A89819A810E94D049A2
:1027B0006091660870916708625F7F4FCE01019655
:1027C0000E944B5CCE0103960E94BA496091660854
:1027D000709167086A5E7F4FCE0101960E944B5C44
:1027E000CE0103960E94C8496091660870916708FF
:1027F0006E5E7F4FCE0101960E944B5CCE01039628
:102800000E94C1490E94CF49609166087091670893
:10281000625E7F4FCE0101960E944B5C8B819C8152
:10282000AD81BE818093620890936308A093640891
:10283000B093650899E288E10FB6F894A895809363
:1028400060000FBE90936000A895012B19F56CE213
:1028500076E08DEB97E00E947B5B6DEF75E08DEB92
:1028600097E00E947B5B86EF9FEF9093AF0580938C
:10287000AE050E942463DC01CB01805A9541AF4F25
:10288000BF4F80930F0690931006A0931106B0934C
:102890001206F4C06DEE75E08DEB97E00E947B5B55
:1028A000CE0101960E94A456CE0101960E944E567A
:1028B00081E090E0DFC08091A80581111AC060E03E
:1028C00070E080E090E00E94CC2FD4C00E9424638E
:1028D00000910F06109110062091110630911206FA
:1028E0000617170728073907D0F10E9457278111CB
:1028F000C5C082E090E0BEC0A895CF55DE4F1882DB
:10290000C15AD140FE01EF56FE4F119211928EE056
:10291000DF011D928A95E9F70091290B10912A0B8E
:102920000115110529F0C8010E94BC3B811138C274
:102930000E9457278111A2C00091290B10912A0BE8
:102940000115110509F49AC0C8010E94BC3BE82E8C
:10295000F12CB2E0EB16F1040CF03FC28FC020E086
:1029600030E043E050E060E48E010F5F1F4FC8018C
:102970000E94C34D6CEF74E0C8010E94087CF8010E
:1029800001900020E9F7CF01801B910B0896813858
:10299000910538F50E945727882319F18091EE0898
:1029A0009091EF08019611F481E090E09093EF0888
:1029B0008093EE088091EE089091EF089093730851
:1029C0008093740847E050E06EE678E0C8010E940A
:1029D0009027AC01455051096EE678E082EA0E94EA
:1029E000B02783E090E09093AF058093AE0564E458
:1029F00078E08DEB97E00E947B5B40C00E942463EF
:102A000000910F06109110062091110630911206C8
:102A1000061717072807390788F51092AF05109297
:102A2000AE052CC00E94246300910F061091100681
:102A3000209111063091120606171707280739074B
:102A400008F457CF1BC00E946653892B09F051CF61
:102A50000E942463DC01CB0188579C4EAF4FBF4FCF
:102A600080930F0690931006A0931106B093120660
:102A700086EF9FEF9093AF058093AE050FB6F89465
:102A8000A89580916000886180936000109260003A
:102A90000FBE8091AE059091AF05181619060CF087
:102AA00059C100916608109167080115110509F4D4
:102AB00051C10E9424634B015C017801FEE3EF0EDB
:102AC000F11CF70180819181A281B381A50194015C
:102AD000281B390B4A0B5B0BCA01B901683E33E076
:102AE00073078105910508F446C028EE33E040E005
:102AF00050E00E946E77861A970AA80AB90AD70191
:102B00008D929D92AD92BC921397F80186A597A5E0
:102B1000A0A9B1A969017A01CC0CDD1CEE1CFF1C37
:102B20008C159D05AE05BF0528F416A617A610AA9C
:102B300011AA09C0821B930BA40BB50BF80186A741
:102B400097A7A0ABB1ABF80182A993A9A4A9B5A995
:102B50008C159D05AE05BF0528F412AA13AA14AA68
:102B600015AA09C0821B930BA40BB50BF80182AB0D
:102B700093ABA4ABB5ABF80186A597A5A0A9B1A965
:102B8000892B8A2B8B2B69F4EE5BFF4F808183307E
:102B900041F484E08083C8010E94D23C01967C010C
:102BA00002C0E12CF12CF80182A993A9A4A9B5A92E
:102BB000892B8A2B8B2BA1F4EE5BFF4F8081833016
:102BC00011F081110DC01082F8013E9684E1DF0101
:102BD0001D928A95E9F7C8010E94D23C03967C01B8
:102BE000B2E0EB16F10429F0E4E0EE16F10409F08E
:102BF0004AC0CE0101960E94752A89819A810E945D
:102C0000D0496091660870916708625F7F4FCE017E
:102C100001960E944B5CCE0103960E94BA496091D6
:102C20006608709167086A5E7F4FCE0101960E9428
:102C30004B5CCE0103960E94C84960916608709172
:102C400067086E5E7F4FCE0101960E944B5CCE01FD
:102C500003960E94C1490E94CF4960916608709115
:102C60006708625E7F4FCE0101960E944B5C8B81AC
:102C70009C81AD81BE818093620890936308A0938C
:102C80006408B0936508F3E0EF16F10409F451C04D
:102C900064F431E0E316F10451F142E0E416F1048A
:102CA00009F058C06BE078E049C054E0E516F10443
:102CB00009F442C085E0E816F10409F04BC06CE36A
:102CC00078E08DEB97E00E947B5B8DEB97E00E94B4
:102CD000455C0E94572781110E94D1560E942463AF
:102CE000DC01CB01805D9A48AF4FBF4F13C068E253
:102CF00078E08DEB97E00E947B5B0E945727811163
:102D00000E94D1560E942463DC01CB0188519C4F64
:102D1000AF4FBF4F80930F0690931006A0931106FC
:102D2000B093120686EF9FEF9093AF058093AE05A8
:102D300011C068EF77E0DDCF6CED77E08DEB97E0C9
:102D40000E947B5BCE0101960E94A456CE010196A3
:102D50000E944E5699E288E10FB6F894A8958093A8
:102D600060000FBE909360008091AE059091AF051A
:102D7000CF55DE4F0FB6F894DEBF0FBECDBFDF914B
:102D8000CF911F910F91FF90EF90DF90CF90BF9068
:102D9000AF909F908F907F906F905F904F9008952D
:102DA00060E0C8010E941A38DC0119960D911C914F
:102DB0001A971093AF0A0093AE0A6FEC77E08DEB91
:102DC00097E00E947B5BB8018DEB97E00E94495C25
:102DD0008DEB97E00E94455CABCD61E0C8010E949D
:102DE0001A38FC0161847284F2E0EF16F104A9F054
:102DF00062E0C8010E941A38FC0181849284F3E0E9
:102E0000EF16F10471F063E0C8010E941A38DC018A
:102E100019960D911C911A9707C08BE5882E87E0B3
:102E2000982E8E010F551E4F40E150E0BE016F56A7
:102E30007E4F86E390E00E94532F892B51F4B5E03A
:102E4000EB16F1040CF022C3FE01EF56FE4F7F019A
:102E500004C09E012F563E4F790170920209609284
:102E60000109909204098092030989E09FE59093FB
:102E7000FA088093F9085E013FE7A31A3EEFB30A10
:102E800040E150E062EA77E0C5010E940F706E01F8
:102E90004FE9C41A4EEFD40A20E030E041E050E0A0
:102EA00060E2C6010E94C34D40E250E06BE977E06A
:102EB000C6010E94F16F6BE777E08DEB97E00E940F
:102EC0007B5BB3018DEB97E00E94495C69E777E09B
:102ED0008DEB97E00E947B5BB4018DEB97E00E9445
:102EE000003862E777E08DEB97E00E947B5BB801EA
:102EF0008DEB97E00E94495C6DE677E08DEB97E003
:102F00000E947B5BD8018C91811104C0E12CF12CD3
:102F100000E010E08090AE0A9090AF0A0E94572720
:102F200081113BC1609101097091020980916C0887
:102F300090916D084091030950910409DC01ED91D5
:102F4000FC916115710521F00088F189E02D16C012
:102F50000684F785E02D21E233E03A83298340900F
:102F6000FD085090FE086090FF08709000094B82A9
:102F70005C826D827E82BE016F5F7F4F19958130CA
:102F8000910509F003C19093EF088093EE0887E064
:102F9000E2E1F2E0DE01119601900D928A95E1F7EF
:102FA000FE013196A3E7B8E0CE01089621912D935A
:102FB000E817F907D9F70115110529F0E114F10413
:102FC00021F086EF03C086E301C086EB80937A0888
:102FD00010927B088FE080937C08F4010190002020
:102FE000E9F7CF018819990940968138910508F0D1
:102FF000C1C04FE050E06EE678E0C4010E94902727
:10300000F60101900020E9F73197EC19FD09E80F6E
:10301000F91F3296E138F10508F0ACC0AC016EE65C
:1030200078E0C6010E949027F50101900020E9F7A1
:103030003197EA19FB09E80FF91F3296E138F105DB
:1030400008F098C0AC016EE678E0C5010E949027B8
:103050000115110579F1F80101900020E9F7319788
:10306000E01BF10B9C012E5F3F4FE20FF31FE13895
:10307000F10508F07FC0AC016EE678E0C8010E945F
:103080009027E114F104B1F0F70101900020E9F775
:103090003197EE19FF099C012E5F3F4FE20FF31F9E
:1030A000E138F10508F066C0AC016EE678E0C701D2
:1030B0000E949027AC01455051096EE678E080E10E
:1030C0000E94B0270E9424636093F0087093F10877
:1030D0008093F2089093F3086093F4087093F508D6
:1030E0008093F6089093F70880916C0890916D0892
:1030F000DC01ED91FC910084F185E02D1995892B7F
:10310000C1F40E9424630091F4081091F508209105
:10311000F6083091F708DC01CB01801B910BA20B64
:10312000B30B88399A43A105B105F0F28CEF9FEFFC
:103130001DC0CE018F579F4F0E9406540497D1F4B3
:1031400080917108811111C00E9424636093F4087A
:103150007093F5088093F6089093F7081092F8089A
:10316000109208091092070918C090E0909308097E
:103170008093070980916C0890916D08DC01ED91B6
:10318000FC910488F589E02D199593C18EEF9FEF8E
:1031900090930809809307098CC10091AE0A1091A1
:1031A000AF0A6FE577E08DEB97E00E947B5BB8019B
:1031B0008DEB97E00E94495C8DEB97E00E94455CA7
:1031C00081E08093A80520E030E043E050E060E437
:1031D000CE018F5F9E4F0E94C34D6CEF74E0CE0115
:1031E0008F5F9E4F0E94087CCE018F5F9E4F0E9492
:1031F0005F3E20E030E042E050E060E4CE018F5FCF
:103200009E4F0E94C34D6CEF74E0CE018F5F9E4FC6
:103210000E94087CBE016F5F7E4F8DEB97E00E949D
:103220009F5B8DEB97E00E94455CCE018F5F9E4FC8
:103230000E945F3E20E030E041E050E060E4CE01DB
:103240008F5F9E4F0E94C34D6CEF74E0CE018F5F85
:103250009E4F0E94087CBE016F5F7E4F8DEB97E012
:103260000E949F5B8DEB97E00E94455CCE018F5FD3
:103270009E4F0E945F3EFE01EF53FF4F119211924D
:103280001EE3DF01212F1D922A95E9F71A82198288
:10329000FE0133968EE7DF011D928A95E9F720E063
:1032A00030E041E050E060E4CE018F539F4F0E9438
:1032B000C34D40E450E06BE977E0CE018F539F4F60
:1032C0000E94F16F40E850E068E177E0CE0101969E
:1032D0000E940F70BE016F5F7F4FCE018F539F4FD3
:1032E0000E94692820E030E041E050E060E4CE0137
:1032F0008F539F4F0E94C34D40E450E062E177E05E
:10330000CE018F539F4F0E94F16F40E850E068E07C
:1033100077E0CE0101960E940F7040E850E065EF23
:1033200076E0CE0101960E94F16FBE016F5F7F4F84
:10333000CE018F539F4F0E94692820E030E041E08A
:1033400050E060E4CE018F539F4F0E94C34D40E494
:1033500050E067E279E0CE018F539F4F0E94F16FFA
:1033600040E850E065EE76E0CE0101960E940F70D5
:10337000BE016F5F7F4FCE018F539F4F0E94692820
:1033800020E030E041E050E060E4CE018F539F4FF9
:103390000E94C34D40E450E06EED76E0CE018F53C5
:1033A0009F4F0E94F16F40E850E068ED76E0CE015B
:1033B00001960E940F70BE016F5F7F4FCE018F5349
:1033C0009F4F0E946928A0910D06B0910E0610979C
:1033D00009F443C08091190290911A02AE014F5B2B
:1033E0005E4FFA01819391932EE111922A95E9F7AC
:1033F0009E012F573F4FF9018193919311921A9596
:10340000E9F716960D911C911797E0900D06F09034
:103410000E06E114F10471F00115110559F0D801FF
:1034200018968C918530A9F7C8010E94BC3B88236F
:1034300081F36BC020E030E041E050E060E4CE0179
:103440008F539F4F0E94C34D40E450E06BE776E0FE
:10345000CE018F539F4F0E94F16F84E090E09093D4
:10346000AF058093AE050E942463DC01CB01885731
:103470009C4EAF4FBF4F80930F0690931006A093C2
:103480001106B093120662E477E0B3CA64E080915B
:10349000290B90912A0B0E941A38DC011996ED90A5
:1034A000FC901A976FEA77E08DEB97E00E947B5BC8
:1034B000D4CC009107091091080966E377E08DEB01
:1034C00097E00E947B5BB8018DEB97E00E9400388B
:1034D0006EE177E08DEB97E00E947B5B8DEB97E0F0
:1034E0000E94455C0E942463DC01CB0188579C4EFE
:1034F000AF4FBF4F80930F0690931006A093110615
:10350000B09312068CE090E0B5CA60E0C8010E945A
:103510001A38FC0181859285A385B4858A3091058E
:1035200008F463C020E030E041E050E060E4CE0108
:103530008F539F4F0E94C34DF8016081718140E419
:1035400050E0CE018F539F4F0E942E7C62EC73E0BF
:10355000CE018F539F4F0E94087C40E450E06AE800
:1035600076E0CE018F539F4F0E94F16FBE016F5BDB
:103570007E4FCE018F539F4F0E946928CF57DF4F58
:103580008881C158D040882361F120E030E041E0DB
:1035900050E060E4CE018F539F4F0E94C34DD8018D
:1035A0006D917C9140E450E0CE018F539F4F0E947B
:1035B0002E7C62EC73E0CE018F539F4F0E94087CFB
:1035C00040E450E062E876E0CE018F539F4F0E94C6
:1035D000F16FBE016F577F4FCE018F539F4F0E94F7
:1035E0006928F8010281138110CFFC0140E250E00C
:1035F0008827E055FF4F8F4F0C94D17762ED76E02E
:10360000CE018F5B9E4F0E940F70CF57DF4F188205
:10361000C158D04087CF6DEC76E0CE018F5B9E4FD6
:103620000E940F7040E450E06CEA76E017C066EA52
:1036300076E0CE018F5B9E4F0E940F7040E450E019
:1036400062EA76E00BC06AE976E0CE018F5B9E4FBE
:103650000E940F7040E450E064E976E0CE018F579D
:103660009F4F0E940F705ECFBC018230910508F41D
:103670000895613E8EE1780748F49B0195E0369508
:1036800027959A95E1F748E0420F01C04FEF91E08E
:10369000242F30E0290F311D35952795229FF00109
:1036A000239FF00DF00D11246E177F0718F44FEFD4
:1036B000420F04C02F3F39F091E0920F491740F7B5
:1036C0008FEF890F08958FEF0895CF93DF930097C1
:1036D00009F447C0FC012081222309F442C0EC0117
:1036E00060EA79E00E94E86F892BF1F16BE979E0FB
:1036F000CE010E94E86F892BD1F166E979E0CE0115
:103700000E94E86F892BB1F16DE879E0CE010E944B
:10371000E86F892B91F167E879E0CE010E94E86FAC
:10372000892B71F163E879E0CE010E94E86F892B63
:1037300051F16EE779E0CE010E94E86F892B31F1FB
:103740006EEB79E0CE010E94E86F892B11F16AEBF4
:1037500079E0CE010E94E86F892BF1F489E090E0D6
:103760001DC080E090E01AC081E090E017C082E0C8
:1037700090E014C083E090E011C084E090E00EC0BF
:1037800085E090E00BC086E090E008C087E090E024
:1037900005C088E090E002C08FEF9FEFDF91CF91EE
:1037A00008952F923F924F925F926F927F928F92E5
:1037B0009F92AF92BF92CF92DF92EF92FF920F93C0
:1037C0001F93CF93DF93CDB7DEB72A970FB6F89448
:1037D000DEBF0FBECDBF5C016B01042F7901672BEB
:1037E00009F459C021153105F1F0D9018C918823D4
:1037F000D1F06FE270E0C9010E94137C009739F0AC
:10380000FC011192CF010E94651B4C0102C0812C6A
:10381000912CC7010E94651B7C01019731F08A94AD
:103820008928C1F502C0E12CF12C6DEF79E0C601C9
:103830000E94E86F892B09F4BFC069EF79E0C601E7
:103840000E94E86F892B09F495C064EF79E0C60106
:103850000E94E86F892B11F543E0842E912C60E0E3
:103860007AE08DEB97E00E947B5BB4018DEB97E0F3
:103870000E9400388DEB97E00E94455CBFEF8B16ED
:103880009B0611F00CF0A8C0EEEF8E16EFEF9E062F
:103890000CF496C084C280E090E081C26DEE79E0C5
:1038A000C6010E94E86F892B09F454C068EE79E0E4
:1038B000C6010E94E86F892B09F450C064EE79E0DC
:1038C000C6010E94E86F892B09F44CC06FED79E0C6
:1038D000C6010E94E86F892B09F448C06AED79E0BF
:1038E000C6010E94E86F892B09F466C064ED79E097
:1038F000C6010E94E86F892BE9F16BEC79E0C60103
:103900000E94E86F892BD1F162EC79E0C6010E9438
:10391000E86F892BB9F1D6018C918D32B9F190ED18
:10392000980F9A3098F18B37A1F18332B9F143E0C7
:1039300050E06EEB79E0C6010E940170892B99F18D
:1039400043E050E06AEB79E0C6010E940170892BE8
:1039500079F524C034E0832E912C81CF25E0822E8E
:10396000912C7DCF96E0892E912C79CF87E0882EFF
:10397000912C75CF12E0812E912C71CFB8E08B2E57
:10398000912C6DCFA9E08A2E912C69CF812C912C9E
:1039900066CFFEEF8F2E99249A9461CFEDEF8E2E95
:1039A00099249A945CCF7CEF872E99249A9457CFD0
:1039B00088248A94982C53CF88248394912C4FCFB9
:1039C000FCEF8F16FFEF9F06E1F02DEF82162FEF31
:1039D000920609F45BC0D7C18114910491F031E0E3
:1039E0008316910409F0CFC1D501ED91FC910190AE
:1039F000F081E02D20E030E040E050E061E070E058
:103A0000BFC1CE0101962C01812C912C182F5A8612
:103A10003401AFEF6A1A7A0A4301F60180818823E4
:103A2000C9F06F018191882329F08D3219F08053FC
:103A30008A30B8F7C6010E94C16F1C016CE270E0C9
:103A4000C6010E94137C6C01892B39F0FFEFCF1A5D
:103A5000DF0A03C080E090E001C0C101D2018D9374
:103A60009D932D01C114D10439F093E069167104BE
:103A700079F643E0842E912CD501ED91FC910190D3
:103A8000F081E02D212F3A85A40178C1CE0107965F
:103A90009E01275F3F4F3F932F93215031093F9362
:103AA0002F939F938F9385E494E09F938F93DF925E
:103AB000CF920E94C77C0FB6F894DEBF0FBECDBF79
:103AC000039709F0E7CE1F8188858984912F81179C
:103AD00008F4982FC82C981508F4C92E1C19982E94
:103AE0009C188C189C2D90959F3F39F080E0909504
:103AF0000E94341BD82ED09402C0DD24DA94892D84
:103B000090E0810F911D880D911D892B29F4CD2CFA
:103B1000C094D12C10E0FFC0FFEFDF16F9F0D110F8
:103B200002C0DD24D3944D2C512C612C712C6FEFED
:103B30007FEF80E090E0A30192010E949077A12F97
:103B4000B0E00E94AF77172FA92DB0E00E94AF77A9
:103B5000972EA82DB0E00E94AF77872E692C712C8C
:103B6000610E711C680C711C2FEF62167104FCF45D
:103B70006114710419F466246394712C930140E07C
:103B800050E06FEF7FEF80E090E00E949077A12FF0
:103B9000B0E00E94AF77172FA92DB0E00E94AF7759
:103BA000972EA82DB0E00E94AF77872E05C03FEF7B
:103BB0006316710409F06CF42C2D362D230F08F4D4
:103BC0002FEF922F2F3F29F080E00E94341BC82E48
:103BD00002C0CC24CA94292D981408F4282D21174A
:103BE00008F4212F21132FC091100DC0122F20E8AF
:103BF000121B08F410E020E6129F010E10E0111DC8
:103C00001124105387C0892D90E0422F50E0481BAB
:103C1000590B8417950744F4192D20E6129F010EC5
:103C200010E0111D112476C016E5190D121B24E0B9
:103C3000121B08F410E020E6129F010E10E0111D87
:103C40001124105E67C092123AC081101AC02BEA8C
:103C5000722F711B08F470E0172F3FE2139F010EC3
:103C600010E0111D1124792D721B08F470E020E67C
:103C7000729F070E70E0711D1124170F1695105CCE
:103C800049C0282D30E0892D90E0821B930B182D20
:103C90002817390744F420E6129F010E10E0111D89
:103CA0001124105A37C025E5121B08F410E020E358
:103CB000129F010E10E0111D112410582BC011117C
:103CC0000DC0182D20E8121B08F410E020E3129F0D
:103CD000010E10E0111D112418571CC0212F30E0D7
:103CE000882D90E0821B930B2817390744F420E6B7
:103CF000129F010E10E0111D112410560BC025E576
:103D0000121B08F410E020E6129F010E10E0111DB6
:103D1000112410541F5F212F30E0ADE6B1E00E9466
:103D2000C277412C512C32014A94A30192010E9486
:103D300090773A8329832D2D30E0A4E6B0E00E94ED
:103D4000C277A30192010E9490773C832B832C2D94
:103D500030E0A4E6B0E00E94C277A30192010E9485
:103D600090773E832D83D501ED91FC910190F081F8
:103D7000E02D9E012F5F3F4F43E050E060E070E098
:103D8000C50119950CC0D501ED91FC910190F08110
:103D9000E02D20E030E040E050E0B401F1CF2A9681
:103DA0000FB6F894DEBF0FBECDBFDF91CF911F914C
:103DB0000F91FF90EF90DF90CF90BF90AF909F90CA
:103DC0008F907F906F905F904F903F902F900895CD
:103DD0008F929F92AF92BF92CF92DF92EF92FF921B
:103DE0000F931F93CF93DF93E0910D06F0910E0692
:103DF000309709F468C0812EC02F932EC22EA52EB5
:103E0000D42EB72ED62FBC01CF010E9427388C01AB
:103E1000009709F45BC0DC0118968C91853009F09D
:103E200055C060E0C8010E941A387C0161E0C801F9
:103E30000E941A38FC0101851285D70119962D912F
:103E40003C911A972130310569F02CF4232BF1F5C0
:103E50006C2FC80118C02230310549F027303105D8
:103E6000A9F034C06C2FC80103960E940E4C6D2F30
:103E7000C8010E940E4C6D2DC80101960E940E4C87
:103E80006C2DC80102960E940E4C20C0892BF1F0C7
:103E900080858530D9F4E680F780E114F104B1F033
:103EA0000C2F182D2C2D392D4D2D5A2D6D2F7B2D8E
:103EB000F701818592850E94E81ED7011296ED9048
:103EC000FC901397EACF80E090E002C081E090E0A0
:103ED000DF91CF911F910F91FF90EF90DF90CF90E6
:103EE000BF90AF909F908F900895CF92DF92EF9206
:103EF000FF920F931F93CF93DF93E0912D0BF091DF
:103F00002E0B3097A1F09085953089F469017A01E4
:103F1000EB01682FCF010E941A38FC018185928540
:103F2000009729F09601A701BE010E94E81EDF91CB
:103F3000CF911F910F91FF90EF90DF90CF90089558
:103F4000AF92BF92CF92DF92EF92FF920F931F93A7
:103F5000CF93DF938091260B9091270B892B09F447
:103F600072C0E1E0F0E0C0E0D0E0CC24C394D12CFA
:103F7000B6010C2E02C0660F771F0A94E2F740913B
:103F8000F9055091FA057F0184E0E80EF11CCF019C
:103F9000B12C9C01A0910602B0910702A817B907A5
:103FA00020F42091060230910702A091400BB091BD
:103FB000410BA20FB31FAC90A091260BB091270B21
:103FC0009C0121503109A20FB31F0A2D10E02C9142
:103FD00030E00217130729F0462B572BAC92BB2475
:103FE000B3940196E816F906A1F65093FA054093AA
:103FF000F905BB2011F18091260B9091270BE80F5A
:10400000F91F028110E0218130E0408150E03197BA
:10401000608170E0CE010E94751F0E942463DC0164
:10402000CB01845D9E4FAF4FBF4F8093F5059093BA
:10403000F605A093F705B093F8052196F701C43073
:10404000D10509F095CFDF91CF911F910F91FF908E
:10405000EF90DF90CF90BF90AF900895DC01129663
:10406000ED91FC911397309721F081E09085953088
:1040700009F080E00895CF92DF92EF92FF92CF9304
:10408000DF93DC011696ED91FC911797309721F1A3
:104090002085223009F56A017B01EC0162EB79E0B1
:1040A0008DEB97E00E947B5B6CEA79E08DEB97E00B
:1040B0000E947B5B2AE030E0B701A6018DEB97E020
:1040C0000E94FD5B8DEB97E00E94455CEE81FF81D5
:1040D000C186D286E386F486DF91CF91FF90EF9080
:1040E000DF90CF900895FC0186819781009789F039
:1040F000FC012085223041F0253079F460E00E94F7
:104100001A38009779F0FC01618572858385948562
:1041100008956FEF7FEFCB0108956EEF7FEF8FEF84
:104120009FEF08956DEF7FEF8FEF9FEF08950F934F
:104130001F93CF93DF93FC01C481D581209799F021
:104140008885823029F4672B71F489859A8518C097
:10415000853061F48B01CE010E94BC3B90E00817D2
:1041600019073CF003C08FEF9FEF0AC08EEF9FEF5F
:1041700007C0602FCE010E941A38FC01818592850C
:10418000DF91CF911F910F910895CF93C62F63E0D8
:10419000FC01828193810E941A380097C9F04C2F4C
:1041A00050E060E070E0FC014187528763877487CC
:1041B00064EA79E08DEB97E00E947B5B6C2F8DEBDE
:1041C00097E00E9442388DEB97E0CF910C94455CCC
:1041D000CF910895CF93C62F63E0FC018281938134
:1041E0000E941A38009731F0FC018185C11103C08B
:1041F0008F7001C08FEFCF910895BF92CF92DF9261
:10420000EF92FF920F931F93CF93DF93EC010E94E5
:104210002E20882309F441C08A819B810E94BC3BE7
:10422000082F10E0C801880F991F9C012B593D4FA2
:10423000790132E0B32E04301105D4F4F701C190B6
:10424000D1907F010E946636009751F0FC01B08644
:10425000A601DD0C660B770B418752876387748755
:10426000BC018A819B810E9449380F5F1F4FE3CFB9
:104270000A811B8160E0C8010E941A38FC01818517
:10428000888761E0C8010E941A389D838C8362E0B0
:10429000C8010E941A389F838E83DF91CF911F91AE
:1042A0000F91FF90EF90DF90CF90BF900895CF9344
:1042B000DF93EC01FB0124813581408151816281D2
:1042C00073810E94FD5BCE01DF91CF9108958F92A3
:1042D0009F92AF92BF92CF92DF92EF92FF920F9395
:1042E0001F93CF93DF93CDB7DEB7C054D1090FB67C
:1042F000F894DEBF0FBECDBF8C015B01FC01F380E3
:104300006AE779E08DEB97E00E947B5B6F2D8DEB88
:1043100097E00E94423868E779E08DEB97E00E94D1
:104320007B5BB5018DEB97E00E9400388DEB97E049
:104330000E94455CF801C080D18060E574E0C60150
:104340000E9427384C0165E574E0C6010E942738B9
:104350008C016AE574E0C6010E9427387C016FE594
:1043600074E0C6010E9427386C010097D1F0FC016F
:104370006185728540E450E0CE0101960E944C7C3C
:104380000E945727882369F08091AB05882309F4A0
:104390004BC007C0F80161857285FB0180818111E6
:1043A00067C08114910409F468C0F40161857285C5
:1043B000CE0101960E945626CE0101960E942E2023
:1043C000882309F45AC0AB2879F00115110551F47E
:1043D000E12CF12C01E020E030E040E050E061E031
:1043E00070E00EC0F80112C0E114F10471F4E12C88
:1043F000F12C01E020E030E040E050E062E070E0CD
:10440000CE0101960E94DF0838C0F70161857285F0
:10441000FB018081882389F120E030E041E0CE017A
:1044200001960E94D11B29C06FE270E0CE01019677
:104430000E94137C892B51F4F6012185328543E0DB
:1044400050E060E4CE0101960E94C34DA114B10476
:1044500039F00115110509F09DCF64E674E008C03C
:10446000E114F10419F467E674E002C0F70193CF98
:10447000CE0101960E94692894CFC05CDF4F0FB631
:10448000F894DEBF0FBECDBFDF91CF911F910F918A
:10449000FF90EF90DF90CF90BF90AF909F908F9064
:1044A0000895FF920F931F93CF93DF93EC011D822A
:1044B0001C821A821B82088119810115110509F4D9
:1044C00052C0F8018085863009F04DC080911306F6
:1044D00090911406892B09F446C06BE674E0C8017C
:1044E0000E942738009719F0FC0181858A83F80122
:1044F000808191810E94C16FF82E8B836DE674E0FC
:10450000C8010E942738009759F51A8163E779E0BE
:104510008DEB97E00E947B5B6F2D8DEB97E00E9407
:10452000423861E779E08DEB97E00E947B5B612F79
:104530008DEB97E00E9442388DEB97E00E94455C3E
:1045400040E050E06DE674E0888199810E94663811
:104550006DE674E0888199810E942738009719F0F0
:1045600009969D838C83DF91CF911F910F91FF90CE
:104570000895EF92FF920F931F93CF93DF93809153
:10458000F9059091FA05C4E0D0E021E030E0AC01FB
:1045900042235323452B29F0A901409550958423AC
:1045A0009523220F331F219791F79093FA0580935B
:1045B000F9050E9424630091F5051091F6052091FC
:1045C000F7053091F805601771078207930708F423
:1045D00057C0012B022B032B09F452C01092F50592
:1045E0001092F6051092F7051092F805E12CF12CC7
:1045F000E091260BF091270BEC0FFD1F038110E0DB
:10460000228130E0418150E0608170E0C7010E946A
:10461000751F8FEFE81AF80A249684E0E816F10473
:1046200039F7C1E0D0E080910602909107028C1723
:104630009D0728F4809106029091070201C0CE01E7
:104640002091400B3091410BF901E80FF91F608177
:104650008DEB97E00E9442386FE674E08DEB97E0B7
:104660000E94495C2196C131D105E9F68DEB97E0B6
:10467000DF91CF911F910F91FF90EF900C94455CCB
:10468000DF91CF911F910F91FF90EF9008952F929E
:104690003F924F925F926F927F928F929F92AF92D2
:1046A000BF92CF92DF92EF92FF920F931F93CF931F
:1046B000DF93CDB7DEB728970FB6F894DEBF0FBEF5
:1046C000CDBF8C016B010E948D35019609F4D3C2D8
:1046D000D801ED91FC910284F385E02DC801199574
:1046E0007C018F3FBFEF9B0709F4C5C2D801ED9154
:1046F000FC910684F785E02D682FC8011995B2E278
:10470000EB16F10429F4B601C8010E94AE35B5C21A
:10471000EDE2EE16F10429F0C701C0970A9708F000
:1047200044C1D801ED91FC910284F385E02DC801CC
:1047300019957C018F3FBFEF9B0709F49CC28D97B1
:1047400089F4D801ED91FC910284F385E02DC80134
:1047500019957C01019609F48EC2EFEFFFEFF887FF
:10476000EF8304C021E030E038872F83C701C09772
:10477000A12CB12C0A97C8F49AE0992E9A9CC001FA
:104780009B9C900D1124B701605371095B01A80E29
:10479000B91ED801ED91FC910284F385E02DC8018A
:1047A00019957C01C0970A9748F3BEE2EB16F10415
:1047B000D1F0C7018F7D85349105A9F0EF81F8858F
:1047C000AE9EC001AF9E900DBE9E900D1124092E8D
:1047D000000CAA0BBB0BF60181879287A387B487D5
:1047E00082E08087D8C0B501BB0C880B990B0E9472
:1047F0000B792B013C01FEE2EF16F104A1F5D80183
:10480000ED91FC910284F385E02DC80119957C019E
:10481000212C312C20E030E040E251E4C301B20110
:104820000E94C0794B015C01B70160537109072EEA
:10483000000C880B990B0E940B79A50194010E9432
:10484000F0772B013C01B1E02B1A3108D801ED9132
:10485000FC910284F385E02DC80119957C01C09775
:104860000A97C0F202C0212C312CC7018F7D8534FC
:10487000910509F042C0D801ED91FC910284F385C5
:10488000E02DC80119957C018B32910559F4D801AE
:10489000ED91FC910284F385E02DC80119957C010E
:1048A000B1E00CC08D9761F4D801ED91FC910284C8
:1048B000F385E02DC80119957C01BFEFBE8302C0CE
:1048C000E1E0EE83A12CB12C8AE0982EC701C097BD
:1048D0008A309105B0F49A9C90019B9C300D112474
:1048E0005C01A20EB31ED801ED91FC910284F38508
:1048F000E02DC80119957C01E9CFB1E0BE83A12C60
:10490000B12CEF81F885BF01FF0F880B990B0E9436
:104910000B79A30192010E94C0792B013C01B501E2
:10492000BB0C880B990B0E940B794B015C01FE813B
:104930006F2FFF0F770B880B990B0E940B799B0150
:10494000AC01C501B4010E94C0794B015C01B10109
:10495000330C880B990B0E940B799B01AC01C501AC
:10496000B4010E94F0779B01AC0160E070E080E24E
:1049700091E40E942D7A9B01AC01C301B2010E9417
:10498000C079D60119966D937D938D939C931C9756
:1049900083E018968C93D801ED91FC910684F785FD
:1049A000E02D6E2DC801199522C0BBE5EB16F10470
:1049B00009F060C0D801ED91FC910284F385E02DEF
:1049C000C80119958B35910509F055C185E0F601AF
:1049D0008087C8010E948D35D801ED91FC91028439
:1049E000F385E02DC80119958D35910519F480E006
:1049F00090E043C1D801ED91FC910684F785E02D4C
:104A0000682FC8011995BB24BA940E9466367C01B0
:104A1000009709F430C1BB2021F0F601978386830B
:104A200008C0D40113969C938E931297FC01958233
:104A30008482C8010E948D35B701C8010E944723B6
:104A4000892B09F018C1C8010E948D35D801ED915C
:104A5000FC910284F385E02DC8011995B12C470122
:104A60008C32910591F221E030E08D35910509F00D
:104A700089C086C0BBE7EB16F10409F088C0D801F5
:104A8000ED91FC910284F385E02DC80119958B37D7
:104A9000910509F0F0C086E0F6018087C8010E9408
:104AA0008D35D801ED91FC910284F385E02DC8018C
:104AB00019958D37910509F49ACFD801ED91FC91A4
:104AC0000684F785E02D682FC801199599249A94DA
:104AD0000E9466367C01009709F4CDC0992021F030
:104AE000F6019783868308C0D50113969C938E9315
:104AF0001297FC01B582A482C8010E948D35B701CE
:104B0000C8010E94AE35019609F4B5C0C8010E94E3
:104B10008D35D70119968D919C911A9711969C937A
:104B20008E931A961C921E921997D801ED91FC91C2
:104B30000284F385E02DC8011995CA9709F09BC03E
:104B4000C8010E948D35B701C8010E944723019614
:104B500009F491C0C8010E948D35D801ED91FC91F6
:104B60000284F385E02DC8011995912C57018C32F0
:104B7000910509F4ADCF21E030E08D37910511F4B6
:104B800020E030E088279927821B930B76C0BEE691
:104B9000EB16F10411F519821A821B821C82D801CE
:104BA000ED91FC910484F585E02D44E050E0BE01D8
:104BB0006F5F7F4FC8011995049709F05CC044E00E
:104BC00050E061E774E0CE0101960E943E7C0097C0
:104BD00009F051C0F601108650C0F6E6EF16F10458
:104BE00021F59E012F5F3F4F790185E0D9011D928C
:104BF0008A95E9F7D801ED91FC910484F585E02DC3
:104C000045E050E0B901C80119950597A1F545E0C7
:104C100050E066E774E0C7010E943E7C009759F5BA
:104C200021E0F6012087118628C0F4E7EF16F10491
:104C300011F519821A821B821C82D801ED91FC9118
:104C40000484F585E02D44E050E0BE016F5F7F4FA6
:104C5000C8011995049779F444E050E06CE774E0DA
:104C6000CE0101960E943E7C009729F421E0F601D6
:104C70002087218702C08FEF9FEF28960FB6F89408
:104C8000DEBF0FBECDBFDF91CF911F910F91FF907F
:104C9000EF90DF90CF90BF90AF909F908F907F90DC
:104CA0006F905F904F903F902F900895CF93DF9338
:104CB000EC0181E792E0998388836115710559F0D1
:104CC00080910D0690910E06009729F00E942738DA
:104CD0009B838A8302C01B821A82CE01DF91CF910F
:104CE0000C94FD206F927F928F929F92AF92BF9211
:104CF000CF92DF92EF92FF920F931F93CF93DF93A8
:104D0000CDB7DEB72C970FB6F894DEBF0FBECDBF80
:104D10004C01762E672E6A01590180910B06909105
:104D20000C06892BA1F069E37AE08DEB97E00E94F5
:104D30007B5B60E4C4010E94C520A701FF0C660BE9
:104D4000770BC4010E943B208FEF9FEF9BC081E057
:104D500090E090930C0680930B0626E240E855E223
:104D600060E070E080E297E00E94A03870920B094A
:104D700080E297E090930A09809309091092160A3D
:104D80001092180A1092170A0115110541F001300E
:104D9000110539F4FE2CEE24EE24EA9402C0FF241F
:104DA000FA94C701A0E0B0E08F839887A987BA87FB
:104DB00080E190E09C878B87A60160E070E04983EA
:104DC0005A836B837C839E838D83672D762D8DEB39
:104DD00097E00E94003866E37AE08DEB97E00E944E
:104DE0007B5BBE016F5F7F4F8DEB97E00E94572189
:104DF0008C0162E37AE00E947B5BB501C8010E94EE
:104E000000386FE27AE0C8010E947B5BBE01695FF7
:104E10007F4FC8010E9457210E94455CA114B10434
:104E200091F082E0A816B10409F5D0929109C092E0
:104E300090091092930910929209F0929509E092CC
:104E4000940986E010C0D0929109C0929009E110B7
:104E500003C080E090E002C080E09FEF9093930950
:104E60008093920985E00E94053906C067E17AE0E7
:104E70008DEB97E00E947B5B10920C0610920B0664
:104E800080E090E02C960FB6F894DEBF0FBECDBF49
:104E9000DF91CF911F910F91FF90EF90DF90CF9016
:104EA000BF90AF909F908F907F906F900895CF9319
:104EB00080916C0890916D08009771F1DC01ED9183
:104EC000FC910688F789E02D1995C1E0811125C074
:104ED000C0E08091070990910809892BF1F48DEFCA
:104EE0009FEF909308098093070980916C08909137
:104EF0006D08DC01ED91FC910680F781E02D19959C
:104F000080916C0890916D08DC01ED91FC91048812
:104F1000F589E02D199501C0C0E08C2FCF9108953F
:104F2000CF93DF93EC01FA013296E60FF71FDC0115
:104F3000AD014C1B5D0BCF01861B970B2D912223DE
:104F400011F02193F5CF9C01241B350B620F731FC9
:104F5000FB013297508331964083DF91CF910895C2
:104F6000EF92FF920F931F93CF93DF9300D01F9286
:104F7000CDB7DEB77B01BA0130E0962F9F77660F81
:104F8000672F661F770B71956115710509F09068A1
:104F900021E0230FE1E0F0E0EC0FFD1FE30FF11D36
:104FA00090836115710511F0322FE7CF30E0B70122
:104FB000621B730B6C5F7F4FDB018C93DE011196DC
:104FC000F701E21BF30B359685E0E80EF11CEE16B7
:104FD000FF0619F08D918193FACF80916C08909122
:104FE0006D082F5F3F4F8901040F151FDC01ED9104
:104FF000FC910280F381E02DA80119957C010E94AB
:1050000024636093F0087093F1088093F208909302
:10501000F30881E00E151F0509F080E00F900F9056
:105020000F900F90DF91CF911F910F91FF90EF9014
:105030000895DF92EF92FF920F931F93CF93DF9328
:105040008C01D62EE72EEA01F22E0E9457278823E4
:10505000B9F1F80101900020E9F73197E01BF10B5D
:10506000CE010796E80FF91FE138F10548F545E054
:1050700050E06EE678E0C8010E949027AC01ED2D6B
:10508000FE2DDC01A259B74F9F012C0F3D1FE217E7
:10509000F30719F081918D93FACF2597FF2011F036
:1050A00081E301C080E34C0F5D1F6EE678E0DF9185
:1050B000CF911F910F91FF90EF90DF900C94B0274C
:1050C00080E0DF91CF911F910F91FF90EF90DF90E3
:1050D0000895FB0101900020E9F73197AF01461BCD
:1050E000570B21E00C941928CF92DF92EF92FF9298
:1050F0000F931F93CF93DF931F921F92CDB7DEB70D
:105100006C0161E00E94EA20182F86FF1BC0C601D7
:105110000E9473207A83698369E07AE08DEB97E0DF
:105120000E947B5B612F70E06F7BE12CF12C01E032
:105130009E012F5F3F4F41E050E0C6010E94DF0813
:1051400081E001C080E00F900F90DF91CF911F911F
:105150000F91FF90EF90DF90CF9008958F929F92E4
:10516000AF92BF92CF92DF92EF92FF920F931F9375
:10517000CF93DF931F921F92CDB7DEB76C017B01F7
:1051800062E070E00E9497208C0197FF03C080E0EE
:1051900090E099C063E070E0C6010E949720AC01E6
:1051A0001816190614F04FE350E0E982FA82013034
:1051B000110531F48F2D880F880BF9828A8303C083
:1051C000023011052CF489819A8199279A83898369
:1051D000A981BA8124E630E00E94E8779A01550F50
:1051E000440B550B0E94907749015A0189013A837B
:1051F000298360E0C6010E94EA20E82EF12CC60156
:105200000E947320092C000CAA08BB0868157905B8
:105210008A059B0559F4012BE9F182E0E816F104B7
:1052200059F085E0E816F104A9F506C0012B71F1EB
:1052300082E0E816F10479F500E020E030E040E09B
:1052400050E061E070E0C6010E94996000E09E01BC
:105250002F5F3F4F41E050E060E070E0C6010E94E8
:10526000996086E0E816F10439F0EA94EF2821F01D
:1052700061E0C6010E94C52049815A81052E000CBB
:10528000660B770BC6010E943B2004C085E0E81640
:10529000F10431F418C085E0E816F104B9F6CCCF7A
:1052A00082E0E816F104B1F362E0C6010E94C52075
:1052B00000E020E030E040E050E062E070E0C60155
:1052C0000E949960E7CF0F900F90DF91CF911F91CF
:1052D0000F91FF90EF90DF90CF90BF90AF909F9095
:1052E0008F900895CF92DF92EF92FF920F93CF931A
:1052F000DF9300D000D0CDB7DEB77C0161E00E9423
:10530000EA2085FF40C0C82ED12CC7010E9473201F
:10531000382F292FF701808590E08A30910528F5F4
:10532000FC018827E654FF4F8F4F0C94D177698397
:105330007A83832F330F990B9C838B83822F220FC9
:10534000990B9E838D8300E09E012F5F3F4F43E0CA
:1053500050E008C07A83698300E09E012F5F3F4FD1
:1053600041E050E060E070E006C000E020E030E0A6
:1053700040E050E0B601C7010E949960B6016F7D20
:10538000C7010E94C52026960FB6F894DEBF0FBE57
:10539000CDBFDF91CF910F91FF90EF90DF90CF9035
:1053A00008958F929F92AF92BF92EF92FF920F93C8
:1053B0001F93CF93DF938C017B0149015A010E9417
:1053C0006636EC01892BF9F083E0888789869A8616
:1053D000AB86BC8688819981009711F00E94896D07
:1053E000C7010E94BC7B99838883BE01C801DF91FD
:1053F000CF911F910F91FF90EF90BF90AF909F9032
:105400008F900C944938DF91CF911F910F91FF90AD
:10541000EF90BF90AF909F908F900895FB01019007
:105420000020E9F73197AF01461B570B20E00C94A1
:1054300019280F931F93CF93DF93EC012097F9F076
:105440000A811B81888587FD06C08E819F81009718
:1054500011F00E94192A8885843031F489859A8553
:10546000009711F00E94896D88819981009711F051
:105470000E94896DCE010E94896DE801DFCFDF9126
:10548000CF911F910F9108950F931F93CF93DF93A7
:10549000009791F08C010E946636EC01892B61F037
:1054A000C8010E948D35BE01C8010E9447230196A4
:1054B00031F4CE010E94192A80E090E001C0CE01B3
:1054C000DF91CF911F910F910895CF93C82F462F51
:1054D00061E070E00E94FB4461E070E08C2F0E946C
:1054E000D1458111F9CFCF91089520E5FC012083AA
:1054F00011820895FC018485843011F00C94614779
:1055000080E008958F929F92AF92BF92CF92DF92E8
:10551000EF92FF920F931F93CF93DF936B017C0168
:10552000142F9B01AC010E947D7A882319F061E859
:1055300074E027C046015701E894B7F82FEF3FEF1A
:105540004FE75FE7C501B4010E947D7A81110DC06C
:105550002FEF3FEF4FE75FE7C501B4010E945C7892
:1055600018161CF465E874E00CC02FEF3FEF4FE70E
:105570005FE4C701B6010E94BB79181694F469E88C
:1055800074E08DEB97E0DF91CF911F910F91FF9029
:10559000EF90DF90CF90BF90AF909F908F900C9442
:1055A0009F5B2FEF3FEF4FE75FECC701B6010E9413
:1055B0005C7887FDE4CF20E030E0A901C701B601A7
:1055C0000E945C7887FF0BC06DE28DEB97E00E9434
:1055D000365BEC01F7FAF094F7F8F09402C0C0E003
:1055E000D0E000E060E070E080E09FE3101741F061
:1055F00020E030E040E251E40E9461780F5FF6CF96
:10560000A70196010E94F0776B017C010E94DA7875
:105610004B015C012AE0AB01BC018DEB97E00E94DD
:10562000B45BC80FD91F1123C9F1C501B4010E9491
:1056300009799B01AC01C701B6010E94EF776B01AC
:105640007C016EE28DEB97E00E94365BC80FD91F9C
:1056500020E030E040E251E4C701B6010E94C07989
:105660004B015C010E94DA786B01E12CF12C2AE0FD
:10567000B701A6018DEB97E00E94B45BC80FD91F5C
:10568000C701B6010E9409799B01AC01C501B401B3
:105690000E94EF776B017C011150D1F6CE01DF91B2
:1056A000CF911F910F91FF90EF90DF90CF90BF901F
:1056B000AF909F908F90089560E08DE00C94AA4188
:1056C00061E08DE00C94AA410F931F93CF93DF9379
:1056D000EB0182EA9AE09F938F9381EA9AE09F938D
:1056E0008F9380EA9AE09F938F938FE99AE09F933C
:1056F0008F938EE99AE09F938F938DE99AE09F9321
:105700008F938DE894E09F938F938B818F938A8101
:105710008F930E94C77C2DB73EB7205F3F4F0FB6D7
:10572000F8943EBF0FBE2DBF069794F40A80DB812C
:10573000C02D6BE47AE08DEB97E00E947B5BBE01AD
:105740008DEB97E0DF91CF911F910F910C94495C05
:105750000E94EA5F0DE91AE0C0E0D0E0F801619133
:105760008F01CE010E9450772196C630D105B1F746
:105770006DE57AE08DEB97E0DF91CF911F910F916E
:105780000C947B5B2F923F924F925F926F927F922D
:105790008F929F92AF92BF92CF92DF92EF92FF9241
:1057A0000F931F93CF93DF93CDB7DEB7C256D109C6
:1057B0000FB6F894DEBF0FBECDBF00911506109155
:1057C00016060115110509F4C7C20E942463C09092
:1057D0001B06D0901C06E0901D06F0901E06C61613
:1057E000D706E806F90608F08EC0D8011696AD90E7
:1057F000BC90179763E0862EA114B10409F474C01D
:10580000F5018085863009F06BC06396BFAEAEAE01
:105810006397CE018F5A9F4F0E9451226596EFAC3D
:105820006597EE2009F45CC067968EAD9FAD6797D3
:10583000892B09F455C06496FFAC6497F0E4FF1619
:1058400009F49EC0FF1508F497C023E0C22ECF14C0
:1058500008F446C0F1FC87C110E062E08E2D0E9482
:10586000AE6265962FAD659730E0F901E356F34FD0
:105870008491F901E350F34F0491F901ED5BF24F8C
:10588000F490FF2009F472C181110E945862EF2D3B
:10589000F0E0EE0FFF1FED59F34FA591B491EC919D
:1058A0000E2331E020E009F430E0832F922F212FE6
:1058B00030E051E02817390709F050E0052F10E0DB
:1058C0006796EEADFFAD6797628173810617170784
:1058D00009F46CC14181442309F44BC14150418317
:1058E000F501A280B38088CF0E942463DC01CB0144
:1058F000C296A11DB11D80931B0690931C06A09318
:105900001D06B0931E060E94246300911706109195
:1059100018062091190630911A060617170728074E
:10592000390708F019C2E0911506F09116060681B4
:1059300017810115110579F0D80118968C918630E0
:1059400031F41A830983CE0101960E945122F80195
:1059500002811381EECF0E942463DC01CB018857C2
:105960009C4EAF4FBF4F8093170690931806A0939D
:105970001906B0931A06F0C192E4D92EFD10B0CFEB
:1059800062EA74E063968EAD9FAD63970E942738FC
:105990008C01F1FC02C062E001C060E08E2D0E942B
:1059A000AE6265968FAD6597863308F08653909109
:1059B0007B00282F2870977F922B90937B00877015
:1059C000806480937C0080917A00806480937A0068
:1059D00080917A0086FDFCCFC0907800809179009C
:1059E000D12CD82A0115110509F4FAC0D80118964E
:1059F0008C91853009F0F4C0C8010E94BC3B982E00
:105A0000B3E0B81708F076C063E0C8010E941A3806
:105A1000FC0181859285A3969FAF8EAFA39762E02C
:105A2000C8010E941A38DC0119964D905D906D9066
:105A30007C901C9761E0C8010E941A381C0160E04C
:105A4000C8010E941A38DC0119962D913D914D91A3
:105A50005C911C976D962CAF3DAF4EAF5FAF6D97CD
:105A60009601DD0C440B550B6D96CCACDDACEEAC69
:105A7000FFAC6D972C193D094E095F09A396EEAC5A
:105A8000FFACA397C701FF0CAA0BBB0BBC01CD0158
:105A900064197509860997090E945E77D1011996E4
:105AA0002D913D914D915C911C976D96CCACDDACE8
:105AB000EEACFFAC6D972C193D094E095F096D9650
:105AC0002CAF3DAF4EAF5FAF6D970E949077420E07
:105AD000531E641E751E620145E0E42E9E1010C028
:105AE00064E0C8010E941A38DC0119968D919C91DE
:105AF0001A9708C0E0E0F4E0A396FFAFEEAFA397DB
:105B000081E090E0A396EEACFFACA397EC14FD040B
:105B10000CF4670132E0F32E9F1064C00D2C000CD2
:105B2000EE08FF0860E0C8010E941A38FC01818578
:105B30009285A385B485C816D906EA06FB06C4F18A
:105B400061E0C8010E941A38FC0181859285A38515
:105B5000B4858C159D05AE05BF050CF0C1CECC24D7
:105B6000C394D12C27C011E060E078CE80E090E0B3
:105B70009ECE64964FAD649740FF0AC02817390740
:105B800071F461E08081811160E0608370E002C0A7
:105B90005083B801CE018F5A9F4F0E9467216796AC
:105BA000EEADFFAD6797138302839ACE818298CEC4
:105BB000C12CD12C6796EEADFFAD679782819381A2
:105BC0008C159D0519F1B601CE018F5A9F4F0E9489
:105BD00067216796EEADFFAD6797D382C28216C08C
:105BE00081E090E06796EEADFFAD6797228133814B
:105BF0007601E21AF30A9701F7FE03C03195219569
:105C00003109821793070CF098C011826796EEADA8
:105C1000FFAD6797818185300CF062CE82819381E0
:105C20008C159D0509F45CCE6996DFAECEAE699702
:105C300065961FAD65976FE77CE08DEB97E00E945E
:105C40007B5B612F8DEB97E00E9442386DE77CE033
:105C50008DEB97E00E947B5BB6018DEB97E00E9495
:105C600000388DEB97E00E94455C63960EAD1FAD4A
:105C7000639760E574E0C8010E9427387C016FE5F6
:105C800074E0C8010E9427388C01009779F1DC018B
:105C900019966D917C911A9740E450E0CE010196DF
:105CA0000E944C7C6FE270E0CE0101960E94137C52
:105CB000892B51F4F8012185328543E050E060E4FE
:105CC000CE0101960E94C34D4AE0BE016F5B7F4F3B
:105CD00069968EAD9FAD69970E9449700E945727C3
:105CE000882321F08091AB05882371F1E114F10440
:105CF000E9F0D70119966D917C911A97CE01019622
:105D00000E945626CE0101960E942E20882371F013
:105D1000E12CF12C01E09E01295A3F4F41E050E077
:105D200060E070E0CE0101960E94DF086796EEAD5C
:105D3000FFAD6797D382C282D3CD818186300CF0CC
:105D400065CF8F5F818362CFBE016F5B7F4FCE01D6
:105D500001960E946928CACFCE59DF4F0FB6F8943A
:105D6000DEBF0FBECDBFDF91CF911F910F91FF908E
:105D7000EF90DF90CF90BF90AF909F908F907F90EB
:105D80006F905F904F903F902F900895A8950E943C
:105D90006411029724F00E94FC540E94C22B0C94C0
:105DA000B9228091AB058F5F8093AB05A8950E94C7
:105DB000C22B8091AB0581508093AB05089561E4BF
:105DC0007CE08DEB97E00E947B5B6EE27CE08DEBEC
:105DD00097E00E947B5B60E27CE08DEB97E00E94A5
:105DE0007B5B68E17CE08DEB97E00E947B5B8DEB59
:105DF00097E00E94455C6BE07CE08DEB97E00E94B1
:105E00007B5B6BEF7BE08DEB97E00E947B5B6FEE43
:105E10007BE08DEB97E00E947B5B68ED7BE08DEB98
:105E200097E00E947B5B66EC7BE08DEB97E00E9445
:105E30007B5B61EB7BE08DEB97E00E947B5B62EA32
:105E40007BE08DEB97E00E947B5B6AE97BE08DEB6A
:105E500097E00E947B5B6FE87BE08DEB97E00E9410
:105E60007B5B65E87BE08DEB97E00E947B5B6DE7F9
:105E70007BE08DEB97E00E947B5B61E77BE08DEB45
:105E800097E00E947B5B67E57BE08DEB97E00E94EB
:105E90007B5B68E37BE08DEB97E00E947B5B8DEBA7
:105EA00097E00C94455CAF92BF92CF92DF92EF9255
:105EB000FF920F931F93CF93DF936C017B018A01B5
:105EC0000E94487781508E3FA0F45701C0E0D0E097
:105ED00001501109C017D1077CF4C6018C0F9D1F1A
:105EE0000E944877F50181935F01882329F021966C
:105EF000F1CF80E090E005C0CE0DDF1D188281E07B
:105F000090E0DF91CF911F910F91FF90EF90DF9084
:105F1000CF90BF90AF900895CF92DF92EF92FF9213
:105F20000F931F93CF93DF936C01EB010990002037
:105F3000E9F72197C61BD70BC032D10514F0CFE18A
:105F4000D0E08B01E12CF12CEC16FD0664F4F80195
:105F500061918F01C7018C0D9D1D0E945077FFEF4D
:105F6000EF1AFF0AF1CF60E0C6018C0F9D1FDF9191
:105F7000CF911F910F91FF90EF90DF90CF900C94F5
:105F80005077882319F066E67AE002C068E67AE086
:105F90008DEB97E00C947B5BAF92BF92CF92DF9238
:105FA000EF92FF920F931F93CF93DF93CDB7DEB79E
:105FB000C058D1090FB6F894DEBF0FBECDBF8E0119
:105FC0000F5B1F4FD8011D921C92FE01ED5BFF4F2E
:105FD0002EE1DF011D922A95E9F7029774F0FB018B
:105FE000628173814FE150E0C8010E944C7CB8018E
:105FF00086E190E00E948C2F10C040E250E0B80192
:1060000086E190E00E94532F892B39F440E250E062
:106010006CE27BE0C8010E940F708091A20A1F927F
:106020008F938091A10A1F928F938091A00A1F9253
:106030008F9380919F0A1F928F9380919E0A1F9247
:106040008F9380919D0A1F928F9386EA94E09F938D
:106050008F931F9280E48F93CE0101966C019F93E2
:106060008F930E945B7C68E17BE08DEB97E00E9460
:106070007B5BB8018DEB97E00E94495CB6018DEB2C
:1060800097E00E94495C8DEB97E00E94455C0FB65B
:10609000F894A895809160008861809360001092C8
:1060A00060000FBE7E0191E6E90EF11CD701139648
:1060B0001C921E92129788EE93E0A0E0B0E0F701E8
:1060C00084839583A683B78384E084878BEF92E0F3
:1060D0009183808316870587108A178680E590E074
:1060E000928B818B158A6DED73E389E996E30E94AB
:1060F0008D708C010FB6F894DEBF0FBECDBF892B1B
:10610000E1F183E090E00E94F16CD8011D969C9330
:106110008E931C97FC01F182E0821282C7010E94DB
:106120001B44882319F0C7010E948245D7011F969E
:106130006D917C9150975196AD90BC90529761159E
:10614000710569F0CE0189589F4F0E944B5CA501F3
:10615000BE0169587F4FC7010E945E4A07C0F70120
:1061600065857685A501C7010E94704E181619062F
:106170000CF496C0C8010E94723600E010E0F701EE
:10618000E388F48899E288E10FB6F894A8958093A3
:1061900060000FBE909360000115110509F467C0FF
:1061A000F8ECEF16F10409F056C06CE07BE08DEBE3
:1061B00097E00E947B5BEB961FAE1EAEEB97ED96D1
:1061C0001FAE1EAEED978FEF9FEFEF969FAF8EAF96
:1061D000EF9789E792E0E9969FAF8EAFE997C158B4
:1061E000DF4F19830883CF57D040F8940E943D6059
:1061F000CE0189589F4F0E94442A909314068093A1
:1062000013067894C8010E9472368091130690910B
:106210001406892B79F465EF7AE08DEB97E00E9404
:106220007B5B0E942463DC01CB018856954CAF4F09
:10623000BF4F2BC06AEE7AE08DEB97E00E947B5B4C
:106240000E94D75063EE7AE08DEB97E00E947B5B73
:1062500082E090E0C5C06BEC7AE08DEB97E00E94A5
:106260007B5BB7018DEB97E00E94003806C068EBBE
:106270007AE08DEB97E00E947B5B0E942463DC0157
:10628000CB0188579C4EAF4FBF4F80930F06909322
:106290001006A0931106B093120685EF9FEFA0C0E1
:1062A000D7011D96BC901D971E96AC90DF92CF92A1
:1062B00084EB9AE09F938F931F930F930E94167124
:1062C000DF92CF928FEA9AE09F938F931F930F9361
:1062D0000E941671D8011C96ED91FC911D9781E0EA
:1062E0008283DF92CF928CEA9AE09F938F931F93E1
:1062F0000F930E941671D8011C96ED91FC911D9789
:106300001282AF92BF9286E79AE09F938F931F937A
:106310000F930E94167181EB9AE09F938F931F93C6
:106320000F930E941671F701148A138AD8011C96E4
:10633000ED91FC911D97A080B1800FB6F894DEBF5F
:106340000FBECDBF83E3C82ED12CD501ED91FC91BA
:106350000084F185E02DC501199541975CF4B1E009
:10636000CB1AD10839F064E170E080E090E00E943F
:10637000EA62EBCF6E01F7E7CF0ED11CDF92CF922E
:106380008AE69AE09F938F931F930F930E94337135
:106390000F900F900F900F900F900F90019709F0B2
:1063A000EECEF60180819181D70154969C938E9315
:1063B0005397D12C80E08A3039F4BAE0DB1609F427
:1063C000DECE9AE0D92E03C08D3009F0D82EC80158
:1063D0000E94D8708F3F79F7C8010E947236CFCEE5
:1063E000C058DF4F0FB6F894DEBF0FBECDBFDF91B0
:1063F000CF911F910F91FF90EF90DF90CF90BF90C2
:10640000AF9008950E94CC2F9093AF058093AE0576
:1064100083E29AE00C948245CF93DF93EC01E8810C
:10642000F9810284F385E02DCE0119950196B9F723
:10643000DF91CF910895FC01A285B3851097A9F053
:1064400086859785029788F0CD010196938782878C
:106450006C93868597850197978786870284F38555
:10646000E02D108281E090E0089580E090E00895B2
:10647000FC01868197818F3F2FEF920729F02FEF44
:106480003FEF378326830895A085B185109789F063
:10649000248535852115310561F0CD01019691875F
:1064A00080878C912150310935872487082E000C74
:1064B000990B0895FC0186819781019639F481E05A
:1064C00024853585232B19F480E0089581E0089513
:1064D000CF92DF92EF92FF920F931F93CF93DF93B0
:1064E0007C016A018B01C0E0D0E0CC15DD0589F0AC
:1064F000D701ED91FC910284F385E02DC701199538
:106500008F3FBFEF9B0729F0F80181938F01219600
:10651000ECCFCE01DF91CF911F910F91FF90EF90C3
:10652000DF90CF900895CF93C62FDC01ED91FC91C1
:106530000088F189E02D1995DC01ED91FC91019025
:10654000F081E02D6C2FCF911994CF93DF93EC0164
:106550008E819F810196D9F4288539858A859B850E
:10656000820F931F81159041A0F4E881F981028484
:10657000F385E02DCE011995813291056CF3E88108
:10658000F9810684F785E02D682FCE01199581E009
:1065900001C080E0DF91CF910895062E000C770BAB
:1065A000FC01778366830895CF93DF93EC018E819E
:1065B0009F81019611F5E881F9810088F189E02D2C
:1065C000CE011995DC01ED91FC910084F185E02D5F
:1065D0001995892BA1F0E881F9810284F385E02DDA
:1065E000CE0119958132910534F3E881F981068451
:1065F000F785E02D682FCE01199581E001C080E07C
:10660000DF91CF9108950F931F93CF93DF93EC0108
:106610008B0165ED74E00E94495C01151105B9F12B
:10662000F80161918F01662391F1603220F06232AE
:1066300011F06C3541F56CE5CE010E94365BF80136
:10664000319780818C30D1F044F48930D9F08A3090
:10665000B9F0883029F762E616C0823259F024F486
:106660008D30F1F662E70FC08F3231F08C35C1F614
:106670006CE509C062E207C06FE205C066E603C0D0
:106680006EE601C064E7CE010E94365BC9CF62E2CC
:10669000CE010E94365B80E090E0DF91CF911F91A8
:1066A0000F910895FC012085318582859385AC0189
:1066B0004F5F5F4F53874287820F931F0E9450772F
:1066C00081E090E00895FC01868197818F3F2FEF54
:1066D000920729F02FEF3FEF378326830895208517
:1066E000318582859385AC014F5F5F4F5387428729
:1066F000820F931F0E944877082E000C990B089573
:10670000FC01868197818F3F2FEF920729F02FEFB1
:106710003FEF378326830895808591850C94D87048
:10672000CF92DF92EF92FF92CF93DF93EC018E81B5
:106730009F818F3F2FEF920759F02FEF3FEF3F835D
:106740002E83DF91CF91FF90EF90DF90CF9008954F
:106750000E9424636B017C01A4EFCA0EA1E0DA1E43
:10676000E11CF11CE881F9810088F189E02DCE015E
:106770001995DC01ED91FC910084F185E02D1995CE
:10678000892B39F40E9424636C157D058E059F05C5
:1067900048F3E881F9810088F189E02DCE0119954F
:1067A000DC01ED91FC910284F385E02DDF91CF9126
:1067B000FF90EF90DF90CF901994EF92FF920F939C
:1067C0001F93CF93DF93009719F48FEF9FEF80C053
:1067D000FC01E484F584D7010D911C91D801ED9161
:1067E000FC910688F789E02DC8011995882369F383
:1067F000D801ED91FC910084F185E02DC801199537
:10680000D801ED91FC91892B61F30284F385E02D91
:10681000C8011995EC010196C1F2F8018589882318
:1068200029F06C2F8DEB97E00E944238D701129629
:106830008C91882309F44BC0C532D10509F047C0BB
:10684000D801ED91FC910084F185E02DC8011995E6
:1068500002975CF0D801ED91FC910688F789E02D54
:10686000C80119958111ECCFB0CFD1E0C0E0D801BB
:10687000ED91FC910284F385E02DC80119958F3FBD
:10688000BFEF9B0709F4A1CF9C01215431092A31A4
:10689000310530F09C01215631092A31310538F497
:1068A0008D2F8295807F829FC00D11240AC0C097D2
:1068B0008A30910530F49D2F9295907F989FC00D5E
:1068C0001124D150A0F68C2FCC0F990B01C0CE0112
:1068D000DF91CF911F910F91FF90EF9008958F92CC
:1068E0009F92AF92BF92CF92DF92EF92FF920F935F
:1068F0001F93CF93DF936115710509F4FFC0FB016E
:106900000085002E000C110B220B330B07301105F4
:1069100008F0F4C0DB01EC01F8018827EC53FF4FCD
:106920008F4F0C94D17761E774E006C019968C9173
:10693000882389F06CE774E0CE01DF91CF911F913D
:106940000F91FF90EF90DF90CF90BF90AF909F900E
:106950008F900C949F5B66E774E0EECF19964D9193
:106960005D916D917C911C972AE030E0CE01DF9122
:10697000CF911F910F91FF90EF90DF90CF90BF903C
:10698000AF909F908F900C94FD5B1996CD90DD9009
:10699000ED90FC901C9720E030E0A901C701B60102
:1069A0000E945C7887FF09C067ED74E0CE010E9409
:1069B000495CF7FAF094F7F8F094C701B6010E9429
:1069C000DA784B015C012AE0AB01BC01CE010E94E8
:1069D000B45B69ED74E0CE010E94495CC501B4016D
:1069E0000E9409799B01AC01C701B6010E94EF77B3
:1069F0002DEC3CEC4CE45DE30E94F07720E030E0CD
:106A000040E251E40E94C0790E94DA78AB0160E074
:106A100070E02AE0CE010E94B45B70C019966D91BF
:106A20007C911A97CE01DF91CF911F910F91FF902A
:106A3000EF90DF90CF90BF90AF909F908F900C948D
:106A4000033316960D911C9117976BE5CE010E94AA
:106A5000365B019619F48FEF9FEF52C001151105B7
:106A600071F0B801CE010E946F340196A1F3F801D4
:106A7000028113810115110589F36CE2E7CF6DE501
:106A80002FC016960D911C9117976BE7CE010E94AF
:106A9000365B019601F30115110509F1F8016081DA
:106AA0007181CE010E9403330196A9F26AE3CE01FF
:106AB0000E94365B019679F2B801CE010E946F34D4
:106AC000019649F2F801028113810115110519F3AC
:106AD0006CE2CE010E94365B0196E9F6BCCF6DE711
:106AE000CE010E94365B21E030E0019611F020E0FB
:106AF00030E088279927821B930B02C080E090E04A
:106B0000DF91CF911F910F91FF90EF90DF90CF9089
:106B1000BF90AF909F908F900895CF93DF93EC013B
:106B2000E881F9810284F385E02DCE0119958F3F2C
:106B30002FEF920771F0E881F9818132910594F38A
:106B40000684F785E02D682FCE01199580E090E04E
:106B500002C08FEF9FEFDF91CF910895EF92FF92E8
:106B60000F931F93CF93DF938C017B01DC01ED9199
:106B7000FC910284F385E02D1995829709F078C085
:106B800084E0F701808786E090E00E94F16CEC01E0
:106B9000892B09F46DC0EFE1F6E0F983E88380E02A
:106BA00091E0DF019C011D9221503040E1F79B8371
:106BB0008A831D821C82D801ED91FC910284F385A9
:106BC000E02DC80119958F3FBFEF9B0709F44DC019
:106BD0008232910509F44FC0803291050CF44BC00C
:106BE0008C35910511F0BE013DC0D801ED91FC91AD
:106BF0000284F385E02DC80119958F3FBFEF9B07F5
:106C0000A1F18236910531F15CF48F329105F9F0F2
:106C10008C359105C9F0829771F6BE0182E222C0DF
:106C20008E369105D1F034F48636910521F6BE01F9
:106C30008CE018C08237910599F08437910509F0EE
:106C4000BACFBE0189E00EC0BE018CE50BC0BE010B
:106C50008FE208C0BE0188E005C0BE018AE002C024
:106C6000BE018DE00E94EC5EA6CFCE010E94896D30
:106C70008FEF9FEF24C08C819D81009749F0E881C0
:106C8000F9818E0F9F1FFC0131978081882321F0AD
:106C9000BE0180E00E94EC5E8C819D810E94F16CBF
:106CA0008C01009739F06FE176E00E94277CCE01DD
:106CB0000E94896DF7011287018780E090E0DF91E3
:106CC000CF911F910F91FF90EF9008958DE090E08C
:106CD0000E94F16C009729F02DE0FC0111922A9599
:106CE000E9F708950F931F93CF93DF930097E1F097
:106CF000EC010C851D850115110579F0D8018D91E8
:106D00009C91009739F0DC01ED91FC910488F589A4
:106D1000E02D1995C8010E94896DCE01DF91CF91B8
:106D20001F910F910C947670DF91CF911F910F916D
:106D30000895AF92BF92CF92DF92EF92FF920F939E
:106D40001F93CF93DF9300D01F92CDB7DEB76115AD
:106D5000710509F496C06B01182FDB011C96AD90EC
:106D6000BC901D97F501E080F180D701ED91FC9179
:106D70000688F789E02DC7011995811104C0C60165
:106D80000E9472367EC0F5019281911114C0D70124
:106D9000ED91FC910190F081E02D612FC7011995D3
:106DA000F7018589882309F469C0612F8DEB97E08D
:106DB0000E94365B63C0812F8F7D81548A3138F306
:106DC00080ED810F8A3018F383ED810F8230F8F265
:106DD0001F35E9F21E37D9F21132B1F086EC810F7E
:106DE000823090F08AED810F873070F01D3361F0B2
:106DF000812F8F7E8F3241F08DED810F823020F018
:106E00001B3511F01D3511F491FFC1CF19821A8283
:106E10001B821C82812F012E000C990B9F931F93C4
:106E20008BED94E09F938F938E010F5F1F4F1F9305
:106E30000F930E94987C6E01F4E0CF0ED11C0F904E
:106E40000F900F900F900F900F90D701ED91FC9144
:106E50000190F081E02DD8016C91C7011995F701DF
:106E60008589882331F0D8016C918DEB97E00E94E1
:106E7000365B0F5F1F4F0C151D0539F780E090E062
:106E800002C08FEF9FEF0F900F900F900F90DF9148
:106E9000CF911F910F91FF90EF90DF90CF90BF9017
:106EA000AF9008952C9A08952C980895CF92DF9270
:106EB000EF92FF920F931F93CF93DF93EC017A0130
:106EC0008B016C01C40ED51ECC15DD05A9F00E9406
:106ED00054378FE00E943F448D2F0E943F448C2FF7
:106EE0000E943F44219680E00E943F44F801819334
:106EF0008F010E945237E8CFC701DF91CF911F91D8
:106F00000F91FF90EF90DF90CF900895CF92DF9296
:106F1000EF92FF920F931F93CF93DF93EC017A01CF
:106F20008B016C01C40ED51ECC15DD05A1F00E94AD
:106F3000543780EF0E943F448D2F0E943F448C2F96
:106F40000E943F442196F80181918F010E943F44A5
:106F50000E945237E9CFC701DF91CF911F910F9166
:106F6000FF90EF90DF90CF9008951F93CF93DF9322
:106F7000D82F192FC62F0E94543780EF0E943F440C
:106F8000812F0E943F448D2F0E943F448C2F0E94EE
:106F90003F440E94523781E0DF91CF911F910895C5
:106FA0001F93CF93DF93182F66E270E00E94D145C4
:106FB000C82FD0E067E270E0812F0E94D145DC2F1E
:106FC000CC279E01282BC901DF91CF911F910895F5
:106FD0001F93CF93DF93182F60E270E00E94D1459A
:106FE000C82FD0E061E270E0812F0E94D145DC2FF4
:106FF000CC279E01282BC901DF91CF911F910895C5
:10700000AB01770F660B770B2AE030E00C94FD5B49
:107010000F931F93CF93DF93EC010E947B5B8C0156
:10702000CE010E94455C800F911FDF91CF911F918F
:107030000F910895FC0186819781009739F06623AE
:1070400029F06150FC0182819381F7CF08950F935D
:107050001F93CF93DF938B01FC01C681D7812097CB
:1070600059F0B801888199810E94F57B892B21F024
:107070000A80DB81C02DF3CFCE01DF91CF911F912C
:107080000F910895462F50E060E070E02AE00C94E4
:10709000B45BDC011696ED91FC91179761157105B3
:1070A000A1F0309729F417967C936E931697089564
:1070B00082819381009711F0FC01FACF7383628380
:1070C000DB011596FC93EE9314970895CF92DF920F
:1070D000EF92FF920F931F93CF93DF938C017B016D
:1070E0006A010E946636EC01892B09F182E08887EB
:1070F000A601DD0C660B770B49875A876B877C8767
:1071000088819981009711F00E94896DC7010E94C2
:10711000BC7B99838883BE01C801DF91CF911F9109
:107120000F91FF90EF90DF90CF900C944938DF9152
:10713000CF911F910F91FF90EF90DF90CF90089526
:10714000CF92DF92EF92FF921F93CF93DF93EC01E8
:107150006A017B01122FE889F98982E08083411559
:10716000514E61057105B1F060E079E08DE390E08A
:10717000A70196010E946E77DA01C9010197A10962
:10718000B109B695A795979587959C01211580E142
:107190003807A8F0E889F989108260E874E88EE180
:1071A00090E0A70196010E946E77DA01C90101976C
:1071B000A109B109B695A795979587959C01EC858E
:1071C000FD853083EE85FF852083188EEC89FD894F
:1071D0001083EA89FB89808180618083EA89FB8949
:1071E000808188608083EA89FB89808180688083D0
:1071F000EA89FB8980818F7D8083DF91CF911F9108
:10720000FF90EF90DF90CF9008958F929F92AF9272
:10721000BF92CF92DF92EF92FF920F931F93CF9383
:10722000DF93CDB7DEB7DA950FB6F894DEBF0FBEA9
:10723000CDBFC82E80910B098983CA8221E0C21676
:10724000A0F074E07C1518F487E1C8120EC080919C
:107250000C0990910D099B838C8380910E0990916C
:107260000F099D838E8386E001C082E08E010F5F4F
:107270001F4F90E19C1528F0AFE0CA1630F49BEF49
:1072800001C09AEE9C0D923078F420919009909173
:107290009109F801E80FF11D908391E0980FF80132
:1072A000E90FF11D8E5F2083BFE0CB1641F1BC15C5
:1072B00058F0E5E0CE16A1F0F6E0CF12B6C020916E
:1072C00094099091950910C026E1C21609F48EC068
:1072D00077E1C71609F459C090E1C912A6C055C09C
:1072E0002091920990919309F801E80FF11D908384
:1072F00091E0980FF801E90FF11D8E5F95C0209184
:10730000920930919309F801E80FF11D308342E0B2
:10731000480F91E0980FF801E90FF11D2083B901A2
:1073200067707727A3E036952795AA95E1F7672B35
:1073300019F091E0920F01C0922FB3E0B80FF8015D
:10734000E40FF11D90838C5F60E070E0A0E04FEFF0
:10735000480F9A1303C08B2F890F67C050E09B0121
:1073600035952795400F511F220F331FF901EC5619
:10737000F64FA0FD02C0208101C02181FA012083C7
:10738000AF5F6F5F7F4F8F5FE2CF209192093091A7
:107390009309F801E80FF11D308391E0980FF8018F
:1073A000E90FF11D208392E0980FF801E90FF11D1C
:1073B0008D5F922F990F908390E03327E92FF0E0B3
:1073C000E217F30794F5EE0FFF1FEC56F64F5081CE
:1073D0004181F801E80FF11D408341E0480FF801B9
:1073E000E40FF11D8E5F50839F5FE8CF9091940969
:1073F00020919509F801E80FF11D208321E0280F65
:10740000F801E20FF11D9083209196099091970960
:1074100032E0380FF801E30FF11D908393E0980FED
:10742000F801E90FF11D8C5F20837801F8012FEF3F
:107430003FEFD02E9E2F901B9817A0F491912927F3
:1074400048E050E0B9017695679520FF06C09B01A2
:1074500091E0292790EA392701C09B014150510949
:1074600089F7E8CFF801E80FF11D2083B2E0BB2EC9
:10747000B80E8F5FF801E80FF11D3083F801EB0DB6
:10748000F11D10828091090990910A09DC01ED91AA
:10749000FC910284F385E02D1995019699F7E0910E
:1074A0001F0AF091200A309709F019958091090977
:1074B00090910A092E2D2D192B1558F4F701619181
:1074C0007F01DC01ED91FC910190F081E02D199597
:1074D000EDCFDC01ED91FC910680F781E02D19954F
:1074E000E091210AF091220A309709F019950E9443
:1074F00024634B015C01A8E0EA2EF12CD12C809191
:10750000090990910A09DC01ED91FC910084F18553
:10751000E02D1995892BC1F08091090990910A09F4
:10752000DC01ED91FC910284F385E02D1995909199
:107530000B09891711F0FF2099F1F801EF0DF11DEA
:107540008083EA94F39407C0E0911D0AF0911E0A2B
:10755000309709F01995B5E0FB1222C0EA818E2F11
:107560008F7790E08C159D0509F0A2C0E7FF04C05D
:107570008B81882381F181C08E2F90E0FC013197AF
:10758000E731F10568F48827E553FF4F8F4F0C94DE
:10759000D177F3E0EF2E04C0EB8002C0E5E0EE2EE1
:1075A0000E942463DC01CB0188199909AA09BB094F
:1075B000813D9740A105B10538F480E0EE2031F01F
:1075C000882309F49CCF59C082EEF8CF811155C0B1
:1075D000F4E0FF15C0F58FEF9FEF60E0EF2DF0E0D6
:1075E0009F0122503109462F50E0D801421753071E
:1075F000BCF4A40FB51F4C91842748E050E0DC0197
:10760000B695A79580FF06C0CD0171E0872770EA87
:10761000972701C0CD014150510989F76F5FE3CF32
:10762000A20FB31F2C9130E0AC015527421753072E
:1076300009F040C0892F9927EC0FFD1F208130E011
:1076400082179307B9F58A818530B0F58330B0F59C
:10765000813090F05B81652F70E075956795209182
:107660001C0A40E0842F90E0861797070CF452C064
:1076700020931C0A50FD6CC080E01092160A1092F4
:10768000180A1092170A10921B0AD3950FB6F89495
:10769000DEBF0FBECDBFDF91CF911F910F91FF9045
:1076A000EF90DF90CF90BF90AF909F908F90089514
:1076B00081EEE3CF83EEE1CF8731F1F66B8170E0AD
:1076C0007595679520911C0A40E0842F90E08617FD
:1076D00097071CF020931C0ACFCF4034C0F49C01C4
:1076E0002E5F3F4F220F331F880F991FFC01E75F6A
:1076F000F64FDE01A20FB31F8C9190E0982F8827E0
:10770000D801A20FB31F2C91822B90878783242F3F
:107710004F5FDBCF4034C8F4880F991FFC01E75F4F
:10772000F64FA5E0B0E0AC0FBD1FA80FB91F2C911C
:1077300030E0322F2227A4E0B0E0AC0FBD1FA80F2D
:10774000B91F8C91282B30872783242F4F5F8ACF36
:10775000403468F4880F991FFC01E75FF64FDE01A3
:10776000A80FB91F14968C9190E09087878381E0D1
:10777000840F80931C0A80CFDC011696ED91FC915A
:10778000179780E0309729F08F5F0280F381E02D1A
:10779000F9CF08957F928F929F92AF92BF92CF922E
:1077A000DF92EF92FF920F931F93CF93DF93CDB7AA
:1077B000DEB7A6970FB6F894DEBF0FBECDBF8C0123
:1077C000762E942E852E20E2B22ECE0101967C01DB
:1077D000FC012B2D11922A95E9F781E293E09AA3FF
:1077E00089A38FEF8BA38CA38DA38EA3680183E461
:1077F000C80ED11C43E450E0BE016F5D7F4FC6014F
:107800000E948048019609F4B9C081E089838A8387
:1078100086E0A82EAB821C82F80164817581868186
:1078200097810E94D9776D837E838F83988789861D
:107830009A8680E890E09C878B874CE150E0B70106
:10784000C6010E94D543F7012B2D11922A95E9F725
:10785000480188E0880E911CF401D70101900D9237
:10786000AA94E1F740E150E0B701C6010E94D54378
:10787000F7011192BA94E9F796E0A92EB12C40E2F3
:1078800050E0B701C6010E94D543F1E0AF1AB1083C
:10789000B1F783E6898392E89A8393E59B838C838F
:1078A00085E38D8381E08E837F829DE3988797E0D7
:1078B00099878A8786E0F401DE011B9601900D927C
:1078C0008A95E1F78CE0898B8A8B61EE74E0CE01BA
:1078D00043960E94277CF8016385CE0149960E9459
:1078E000DB57F8016485CE014B960E94DB57F80107
:1078F0006585CE014D960E94DB574EE150E0B70101
:10790000C6010E94D543F3E07F121EC082E3898343
:1079100084E08A83F80196859B8397859C83908970
:107920009D8391899E8396E39F838887828D898733
:10793000838D8A87848D8B87858D8C874CE050E082
:10794000B701C6010E94D54387E3898386E08A8315
:1079500091E09B8393E09C838D838FE08E838AE309
:107960008F838BE388878FEF898749E050E0B701E9
:10797000C6010E94D543C6010E94AD47A6960FB628
:10798000F894DEBF0FBECDBFDF91CF911F910F9155
:10799000FF90EF90DF90CF90BF90AF909F908F902F
:1079A0007F9008952F923F924F925F926F927F92B5
:1079B0008F929F92AF92BF92CF92DF92EF92FF92FF
:1079C0000F931F93CF93DF9300D000D0CDB7DEB7D6
:1079D0008C010E945D6E2FEC37E040E050E00E9489
:1079E0009077DC01CB010196A11DB11DF8018483C4
:1079F0009583A683B78380839183A283B383580141
:107A0000F3E4AF0EB11CC5010E94744564E470E05C
:107A1000C5010E948047882309F436C10E9424636F
:107A20002B013C01812C912CC8018E5B9F4F9E83C2
:107A30008D8348EEC42E43E0D42EE12CF12C52E08D
:107A4000252EAD81BE818C91833009F404C1811152
:107A500020C0F80184819581A681B7810196A11D7E
:107A6000B11D84839583A683B7830E942463641920
:107A7000750986099709A70196010E946E77A901E9
:107A800061E0C8010E94CA3B81E0AD81BE818C9358
:107A9000CAC08430F9F4F80184819581A681B78148
:107AA0000196A11DB11D84839583A683B7830E948F
:107AB00024636419750986099709A70196010E9434
:107AC0006E77A90163E0C8010E94CA3BAD81BE8107
:107AD0002C92A9C0813059F5F80142AD53AD64AD87
:107AE00075AD9E012F5F3F4FC8010E94F057382EA1
:107AF000F2E08F1392C089819A81AB81BC81F80139
:107B000084839583A683B7830E94246364197509CF
:107B100086099709A70196010E946E77A90163E083
:107B2000C8010E94CA3BAD81BE813C927CC08230BC
:107B300009F079C0F80142AD53AD64AD75AD9E0159
:107B40002F5F3F4FC8010E94F057382EF5E08F138A
:107B50005DC0E3E0AD81BE81EC93F80182A193A109
:107B6000A4A1B5A1892B8A2B8B2B41F484E893E047
:107B7000A0E0B0E082A393A3A4A3B5A3F80186A1DB
:107B800097A1A0A5B1A5892B8A2B8B2B61F482A18B
:107B900093A1A4A1B5A1B695A7959795879586A31E
:107BA00097A3A0A7B1A7F80182A593A5A4A5B5A501
:107BB000892B8A2B8B2BA9F482A193A1A4A1B5A117
:107BC000AC01BD0123E076956795579547952A95B9
:107BD000D1F7841B950BA60BB70B82A793A7A4A77D
:107BE000B5A7F80186A197A1A0A5B1A586A797A7DB
:107BF000A0ABB1AB82A593A5A4A5B5A582AB93AB71
:107C0000A4ABB5AB88248394912C0DC0F6E08F1300
:107C100004C0AD81BE811C9206C0BFEF3B1203C001
:107C2000ED81FE811082F1E08F16910409F409CFF5
:107C30000E942463DC01CB0184199509A609B709C8
:107C4000F80126A937A940AD51AD281739074A07D1
:107C50005B0708F0F6CEC5010E947445F8018481E7
:107C60009581A681B7810196A11DB11D848395835D
:107C7000A683B7830E942463F801FE966083718314
:107C800082839383C40102C080E090E026960FB601
:107C9000F894DEBF0FBECDBFDF91CF911F910F9142
:107CA000FF90EF90DF90CF90BF90AF909F908F901C
:107CB0007F906F905F904F903F902F900895CF935B
:107CC000DF93FC0101900020E9F79F01281B390B8D
:107CD000285F3F4F2138310570F5EC010E9457278E
:107CE000882349F18091EE089091EF08019611F4F4
:107CF00081E090E09093EF088093EE088091EE0889
:107D00009091EF08909373088093740847E050E0D7
:107D10006EE678E0CE010E949027FC01E859F74F0B
:107D20001682AC01445051096EE678E082E8DF919A
:107D3000CF910C94B02780E0DF91CF910895CF923E
:107D4000DF92EF92FF920F931F93CF93DF936C011B
:107D50008B017B0182E0E80EF11CC0E0D0E0C6019F
:107D60008C0F9D1F0E944877F70181937F01219618
:107D7000C430D105A1F7F8019281992319F081E06F
:107D80009F3F09F480E090E0DF91CF911F910F9128
:107D9000FF90EF90DF90CF900895EF92FF920F93B6
:107DA0001F93CF93DF937C018B010E5F1F4FC0E0C9
:107DB000D0E0F80161918F01C7018C0F9D1F0E94D7
:107DC00050772196C430D105A1F7DF91CF911F9153
:107DD0000F91FF90EF900895FC01DC018D918111CE
:107DE000FDCF40E050E020E030E08AE0919199231F
:107DF00001F1243031055CF59E3271F44F3F51059D
:107E000009F02CF5DB01A20FB31F12964C932F5FE4
:107E10003F4F40E050E0EACF849FD001859FB00DF6
:107E20001124492F990F550B405351094A0F5B1FDD
:107E3000DDCF4F3F510509F054F4243031053CF4B7
:107E4000FB01E20FF31F428381E090E0089580E0A0
:107E500090E008954F925F926F927F928F929F92DF
:107E6000AF92BF92CF92DF92EF92FF920F931F9348
:107E7000CF93DF93CDB7DEB763970FB6F894DEBF2D
:107E80000FBECDBF7C015B013A01FB0120E080E029
:107E900090E06AE03191332309F140ED430F4A301D
:107EA00080F4689FA001699F500D1124CA01C097FA
:107EB000830F911D37FD9A958F3F910559F350F32C
:107EC00013C03E3289F4233079F0D301A20FB11DE3
:107ED00012968C932F5F80E090E0DCCF233021F46A
:107EE000F301858381E021C0F701428153816481E0
:107EF000758180915C0890915D08A0915E08B091B9
:107F00005F08481759076A077B0709F499C10E945F
:107F100024638701085F1F4F6F7077277C5FC8015C
:107F20000E948047813019F080E090E0FCC181E23E
:107F300093E09A838983F70182819381A481B5813B
:107F40008B839C83AD83BE8345E350E0BE016F5FAE
:107F50007F4FC8010E948048892B19F4C12CD12C75
:107F60006AC10E942463F7017783668376276727B7
:107F700076277A83698342E050E0BE016F5F7F4FCE
:107F8000C8010E94D54381E090E09E878D8742E042
:107F900050E0BE01635F7F4FC8010E94D54380E07F
:107FA00091E09E878D8742E050E0BE01635F7F4F86
:107FB000C8010E94D5431E861D8642E050E0BE01E6
:107FC000635F7F4FC8010E94D54342E050E0BE018D
:107FD000635F7F4FC8010E94D54342E050E0BE017D
:107FE000635F7F4FC8010E94D5434501F501808141
:107FF000882301F164015601F60181912F01882344
:1080000021F08E3211F06201F6CFC818D9081C1485
:108010001D0474F4CF8641E050E0BE01615F7F4FE4
:10802000C8010E94D543A601B401C8010E94D543EE
:108030004201DCCF1F8641E050E0BE01615F7F4F0F
:10804000C8010E94D543C12CDD24D394DE86CD86A1
:1080500042E050E0BE01635F7F4FC8010E94D543FC
:10806000DE86CD8642E050E0BE01635F7F4FC801EF
:108070000E94D543C8010E94AD47892B09F46ECFF9
:10808000E3E0AE2EB12C230122E0420E511C0E94EF
:1080900024633B014C01C8010E94074718161906CA
:1080A000B4F00E942463DC01CB0186199709A8096A
:1080B000B909813A9F40A105B105E0F40E94D12E93
:1080C00061E070E080E090E00E94EA62E4CFF701B6
:1080D0004281538164817581808D918DA28DB38D94
:1080E000481759076A077B0749F4848D958DC59712
:1080F00029F409C0CC24CA94DC2C92C05EEFC52EB2
:10810000DD24DA948DC0F70181A192A10C970CF4C3
:108110009FC04CE050E0BE016F5F7F4FC8010E94DE
:10812000BF468B819C819827892798279A8B898BBA
:1081300029813A81322723273227F7014681578147
:108140002417350709F07FC097FF7DC08F709270AC
:10815000892B09F0E3C06F80788476246724762425
:108160006114710409F4D5C0C12CD12C8D819E817C
:10817000982789279827C816D90608F46EC0812C3D
:10818000912C41E050E0BE016D5E7F4FC8010E941E
:10819000BF468B89982F907C09F091C0811185C0D2
:1081A00042E050E0BE01615F7F4FC8010E94BF46C0
:1081B00042E050E0BE01635F7F4FC8010E94BF46AE
:1081C000C8010E94DE46C8010E94DE46C8010E9426
:1081D000DE46C8010E94DE4642E050E0BE016F5E0E
:1081E0007F4FC8010E94BF468F85988981159140B5
:1081F00009F06DC0CD84DE84DC24CD24DC2481E054
:10820000C816D10409F063C089899A898115944000
:1082100009F07AC044E050E0B201C8010E94BF46B4
:108220000E94D12E81E0A81AB10829F0FFEFCF16E5
:10823000DF0609F42CCFC8010E947445C60173C043
:108240008EEF9FEF70C04CEFC42EDD24DA94E8CFA0
:108250009DEFC92EDD24DA94E3CF41E050E0BE016A
:10826000635F7F4FC8010E94BF468D85882351F010
:108270008D859FEF980F9D87882321F0C8010E946C
:10828000DE46F6CF8D858111E8CFC8010E94DE461B
:10829000C8010E94DE46C8010E94DE46C8010E9455
:1082A000DE46FFEFCF1ADF0A61CF8B899FEF980F71
:1082B0009B8B882341F0C8010E94DE46F6CFC8019F
:1082C0000E94DE461B8A8B8981115BCF69CFC12C4E
:1082D000D12C89899A89982789279827C816D90681
:1082E00038F4C8010E94DE46FFEFCF1ADF0AF1CF53
:1082F0002FEF821A920A6814790409F042CF26EF10
:10830000C22EDD24DA948CCF77EFC72EDD24DA94E9
:1083100087CF3AEFC32EDD24DA9482CF8BEFC82EBD
:10832000DD24DA947DCF63960FB6F894DEBF0FBEDE
:10833000CDBFDF91CF911F910F91FF90EF90DF9014
:10834000CF90BF90AF909F908F907F906F905F90F5
:108350004F9008951F93CF93DF93282F30E0F901BA
:10836000E356F34F8491F901E350F34FD491F901AF
:10837000ED5BF24FC491CC23C1F0162F81110E9406
:108380005862EC2FF0E0EE0FFF1FED57F34FA59171
:10839000B4919FB7F894111104C08C91D095D82353
:1083A00002C0EC91DE2BDC939FBFDF91CF911F9138
:1083B00008951F93CF93DF931F921F92CDB7DEB71F
:1083C0006CE271E080E090E00E94EA621FB7F894EE
:1083D0008091A30A811127C0E8E7FDE08491E2E3E0
:1083E000FDE09491E82FF0E0EE0FFF1FED51F34F09
:1083F000A591B491EC91E92321F461E085E30E9419
:10840000AA4161E085E30E94AE628CB580618CBDBB
:108410008CB580648CBD61E084E30E94AE6261E053
:1084200083E30E94AE628091A30A8F5F8093A30AC8
:108430001FBF249ACE0101960E94752A89819A81D4
:108440000E94D04967E080E090E00E94B53765E582
:108450008BE190E00E94B53765E58AE190E00E94EB
:10846000B5370E94CF4980E090E49093FC0580935B
:10847000FB0580E090E6909304068093030680E07D
:1084800098E49093FE058093FD0580E098E6909334
:1084900006068093050680E090E5909300068093A1
:1084A000FF0580E090E7909308068093070680E040
:1084B00098E5909302068093010680E098E79093F8
:1084C0000A06809309060F900F90DF91CF911F91BC
:1084D0000895AF92BF92CF92DF92EF92FF920F93E7
:1084E0001F93CF93DF931F921F92CDB7DEB75C012E
:1084F0008B016A0179010E94D941CE0101960E9447
:10850000752A89819A810E94D04946E050E06DE940
:108510007AE089E090E00E948637C50102960E94C9
:10852000BA49C60102960E94C849C70102960E9434
:10853000C1490E94CF49F80182819381A481B5810C
:108540008093620890936308A0936408B0936508D1
:108550000F900F90DF91CF911F910F91FF90EF90AF
:10856000DF90CF90BF90AF900895CF92DF92EF92BF
:10857000FF92CF93DF93CDB7DEB768970FB6F8942D
:10858000DEBF0FBECDBFFA0121E233E03A8329837B
:108590005FEF5B835C835D831E8238872F83C2809D
:1085A000D380E480F580C986DA86EB86FC863E8738
:1085B0002D87FB0142815381648175814F87588BE0
:1085C000698B7A8B3C8B2B8BFC0182819381A481FC
:1085D000B5818D8B9E8BAF8BB88F9E012F5F3F4FE8
:1085E000AE01495F5F4FBE01635F7F4FCE0143968F
:1085F0000E94694268960FB6F894DEBF0FBECDBFE9
:10860000DF91CF91FF90EF90DF90CF9008950F937F
:108610001F93CF93DF93CDB7DEB768970FB6F8946B
:10862000DEBF0FBECDBFFB01DC0112964D915D9107
:108630006D917C9115974D8B5E8B6F8B788F81E25E
:1086400093E09A83898321E0288F0D891E892F89E1
:10865000388D0B831C832D833E8398878F83028103
:1086600013812481358109871A872B873C879E8750
:108670008D874F87588B698B7A8BAE014F5F5F4F29
:10868000BE01695F7F4FCE010D960E94B54268968C
:108690000FB6F894DEBF0FBECDBFDF91CF911F9113
:1086A0000F910895CF93DF93CDB7DEB762970FB6E2
:1086B000F894DEBF0FBECDBFFC0182819381A481FF
:1086C000B5818F87988BA98BBA8B21E233E03A83EF
:1086D000298341E04A8B4F85588969897A894B8380
:1086E0005C836D837E8338872F8389879A87AB87E6
:1086F000BC87BE016F5F7F4FCE0107960E94074384
:1087000062960FB6F894DEBF0FBECDBFDF91CF915A
:1087100008950895CF93DF931F92CDB7DEB7698395
:10872000DC01ED91FC910280F381E02D41E050E00D
:10873000BE016F5F7F4F19950F90DF91CF91089524
:10874000FC01818D928D0895FC018489958908959D
:1087500021E233E0FC0131832083FB014089518910
:1087600062897389FC01428353836483758308950E
:10877000DC01ED91FC91048CF58DE02D199480E0E5
:108780000895FC019485FB018485981303C081E062
:10879000943009F480E0089521E0FC018485843060
:1087A00009F420E0822F089508958F929F92AF924E
:1087B000BF92DF92EF92FF920F931F93CF93DF93BD
:1087C0001F921F92CDB7DEB77C014B018A01FC01DD
:1087D000A688B788D08CCE0101960E94752A89811F
:1087E0009A810E94D0498D2D0E94BF578017910712
:1087F00020F48D2D0E94BF578C019801A401B50172
:108800008D2D0E945A570E94CF49F701868997897A
:10881000800F911F978B868BC8010F900F90DF916F
:10882000CF911F910F91FF90EF90DF90BF90AF908D
:108830009F908F900895CF93DF93FC01248524307F
:10884000D1F0EC010E947A2A843181F0882371F002
:10885000883161F08C3161F4E881F9810084F1851F
:10886000E02DCE01199521E0892B19F420E001C0FB
:1088700021E0822F01C080E0DF91CF9108958EBD6D
:1088800000000DB407FEFDCF8EB50895DF92EF9284
:10889000FF920F931F93CF93DF931F921F92CDB739
:1088A000DEB7D82ECE0101960E94752A89819A8161
:1088B0000E94D049E12CF12C8D2D0E94D0378C01E3
:1088C000892B21F08D2D0E94D0377C010E151F05BC
:1088D00099F70E94CF49C8010F900F90DF91CF9177
:1088E0001F910F91FF90EF90DF900895FC0113828C
:1088F000128288EE93E0A0E0B0E084839583A683A3
:10890000B78383E393E09183808381E293E0978749
:108910008687108A118A128A138A84E0808F0895CC
:10892000AF92BF92CF92DF92EF92FF920F931F937D
:10893000CF93DF93CDB7DEB7AF970FB6F894DEBF16
:108940000FBECDBF7C015B016A0101E213E01A8317
:1089500009831B821C821D821E82CE0109960E9401
:1089600076441BA70AA71CA61DA61EA61FA68091BB
:10897000620890916308A0916408B09165088EA385
:108980009FA3A8A7B9A78B839C83AD83BE831886BA
:108990001F82AE01465D5F4FB501CE0101960E9478
:1089A0002A3F81309105B1F4D701ED91FC91048803
:1089B000F589E02D1DA30CA38CA59DA5AEA5BFA593
:1089C0008EA39FA3A8A7B9A7A601BE016C5D7F4F88
:1089D000C7011995AF960FB6F894DEBF0FBECDBF95
:1089E000DF91CF911F910F91FF90EF90DF90CF908B
:1089F000BF90AF9008959B0190E00496982F882730
:108A0000642F820F931F0C94B5371F93CF93DF937E
:108A10001F921F92CDB7DEB7182FCE0101960E948C
:108A2000752A89819A810E94D04960E170E0812F86
:108A30000E94652A4FEF62E070E0812F0E94FB44A4
:108A40000E94CF490F900F90DF91CF911F91089511
:108A5000DF92EF92FF920F931F93CF93DF931F92BA
:108A60001F92CDB7DEB7182FD62E7A01022F0E94A3
:108A70000545CE0101960E94752A89819A810E943E
:108A8000D0494D2D402B60E070E0812F0E94FB44C7
:108A9000E114F10459F4E090AC0AF090AD0A8FEFC4
:108AA000E81AF80AF092AD0AE092AC0A4F2D64E0A1
:108AB00070E0812F0E94FB444E2D65E070E0812F15
:108AC0000E94FB4461E070E0812F0E94652A0E94B1
:108AD000CF4981E00F900F90DF91CF911F910F91BF
:108AE000FF90EF90DF900895CF93DF93FC01808D8E
:108AF000843029F0EF010E94054584E0888FDF91E2
:108B0000CF910895CF92DF92EF92FF920F931F9330
:108B1000CF93DF931F921F92CDB7DEB7FC01F48491
:108B2000F4E0FF1699F18C01CE0101960E94752A9E
:108B300089819A810E94D04968E070E08F2D0E945F
:108B4000652A0E94CF490E9424636B017C01C80101
:108B50000E947A2A8823B9F062E370E080E090E016
:108B60000E94EA620E942463DC01CB018C199D09FA
:108B7000AE09BF09883E9340A105B10540F3F80155
:108B800084850E94054584E0F80184870F900F904A
:108B9000DF91CF911F910F91FF90EF90DF90CF90D9
:108BA0000895CF93DF9390E00496982F8827EC01E7
:108BB000C60FD71F0E9454378FE00E943F448D2F6D
:108BC0000E943F448C2F0E943F4480E00E943F441B
:108BD000C82F0E9452378C2FDF91CF910895CF92EA
:108BE000DF92FF920F931F93CF93DF931F921F92F9
:108BF000CDB7DEB7F82E6B01CE0101960E94752A23
:108C000089819A810E94D04968E270E08F2D0E948C
:108C1000D145082F10E069E270E08F2D0E94D14508
:108C2000702F6627682B21E030E0A6018F2D0E946F
:108C300012570E94CF4981E090E00F900F90DF9192
:108C4000CF911F910F91FF90DF90CF900895CF9318
:108C5000DF931F92CDB7DEB7FC01218D328D232B20
:108C600049F0BE016F5F7F4F808D0E94EF45898183
:108C700090E002C08FEF9FEF0F90DF91CF910895AA
:108C80008F929F92BF92CF92DF92EF92FF920F93BB
:108C90001F93CF93DF931F921F92CDB7DEB7B82EED
:108CA0006B017A01CE0101960E94752A89819A8111
:108CB0000E94D049812C912C8B2D0E94D0378C01A1
:108CC000892B21F08B2D0E94D0374C0108151905F6
:108CD00099F70115110599F463E070E08B2D0E945E
:108CE000D1458431D9F18823C9F101E010E08C31FC
:108CF00011F400E010E01195019511092FC0E01664
:108D0000F1060CF487011016110644F568E270E0D4
:108D10008B2D0E94D145E82EF12C69E270E08B2D5D
:108D20000E94D145FE2CEE24E82A9801A601B70145
:108D30008B2D0E941257E00EF11E4F2D68E270E05D
:108D40008B2D0E94FB444E2D69E270E08B2D0E941A
:108D5000FB4460E470E08B2D0E94652A0E94CF499D
:108D6000C8010F900F90DF91CF911F910F91FF904D
:108D7000EF90DF90CF90BF909F908F900895CF930A
:108D8000DF93FC01218D328D2115310519F48FEF10
:108D90009FEF11C0EC014217530708F0A901888D1D
:108DA0000E9440461816190694F7298D3A8D281B03
:108DB000390B3A8F298FDF91CF9108950F931F932D
:108DC000CF93DF931F92CDB7DEB7FC01218D328D9B
:108DD000232B61F08C0141E050E0BE016F5F7F4FBB
:108DE000808D0E944046181619061CF08FEF9FEFE9
:108DF00008C0F801818D928D0197928F818F8981B2
:108E000090E00F90DF91CF911F910F9108950F93F4
:108E10001F93CF93DF93CDB7DEB728970FB6F894A3
:108E2000DEBF0FBECDBF8C01D80159968D919C91AC
:108E30005A97892B41F0ED91FC910284F385E02D46
:108E4000C8011995F1CFF801808D0E94464418168B
:108E5000190654F548E050E0BE016F5F7F4FD8011E
:108E600058968C910E94404618161906FCF4D801B9
:108E7000509684E0FE01319601900D928A95E1F7BB
:108E80008D8190E0982F88272E81820F911DF80107
:108E9000958B848B8F8190E0982F88272885820F6F
:108EA000911D928F818F02C080E090E028960FB6CE
:108EB000F894DEBF0FBECDBFDF91CF911F910F9110
:108EC00008951F93CF93DF931F921F92CDB7DEB704
:108ED000182FCE0101960E94752A89819A810E94DD
:108EE000D04963E070E0812F0E94D145182F0E9485
:108EF000CF49812F0F900F90DF91CF911F9108954F
:108F0000EF92FF921F93CF93DF93FC01208D2430CB
:108F100011F080E01CC07B01EC0110E0812F0E9469
:108F20006147811102C0188F05C08831E1F31F5FCE
:108F30001430A1F7888D843061F3FD86EC861A8E9B
:108F4000198E20E0A70162E00E94284581E0DF91B0
:108F5000CF911F91FF90EF9008951F93CF93DF93D0
:108F60001F921F92CDB7DEB7FC01108DCE01019686
:108F70000E94752A89819A810E94D04960E270E03E
:108F8000812F0E94652A62E070E0812F0E94D14506
:108F900084FD1DC062E070E0812F0E94D14583FFF7
:108FA0000BC048E162E070E0812F0E94FB440E9408
:108FB000CF4980E090E015C00E94CF49CE010196D4
:108FC0000E94752A89819A810E94D049DCCF40E1B4
:108FD00062E070E0812F0E94FB440E94CF4981E053
:108FE00090E00F900F90DF91CF911F910895CF9354
:108FF000DF93C82FD62F472F60E170E00E94FB441B
:109000004D2F61E170E08C2FDF91CF910C94FB44E8
:1090100090E0982F882744E050E0845F9B4F0C94A9
:109020008637BF92CF92DF92EF92FF920F931F93FA
:10903000CF93DF9300D000D0CDB7DEB7FC01208DF9
:10904000243009F04CC06A017B018C01B12C63E033
:1090500070E08B2D0E94D145811103C0F801B08EC4
:1090600006C08831D9F3B394F4E0BF12F0CFF80111
:10907000808D8430A1F196E0E9E2F3E0DE01119603
:1090800001900D929A95E1F7F70193819F779C8368
:1090900094819D8395819E83B7016E5F7F4F0E946F
:1090A0000848B601F801808D0E94F747F801808DCD
:1090B00090E0982F882746E050E0BE016F5F7F4F19
:1090C0008A5F9B4F0E948637F801128E118E20E82E
:1090D000A60162E0808D0E94284581E001C080E009
:1090E00026960FB6F894DEBF0FBECDBFDF91CF91AD
:1090F0001F910F91FF90EF90DF90CF90BF90089558
:10910000DF92EF92FF920F931F93CF93DF931F9203
:109110001F92CDB7DEB7FB01DC0157961C921E9261
:1091200056972281211109C02381211106C0248173
:10913000211103C025812223F1F041155105D9F0F9
:109140007A018F01FC01D08CCE0101960E94752A14
:1091500089819A810E94D049B8016E5F7F4F8D2D21
:109160000E940848B7018D2D0E94F7470E94CF4901
:1091700081E090E002C080E090E00F900F90DF91DE
:10918000CF911F910F91FF90EF90DF900895CF93B3
:10919000DF931F92CDB7DEB76983DC01ED91FC91BF
:1091A0000280F381E02D41E050E0BE016F5F7F4F10
:1091B00019950F90DF91CF910895DC01ED91FC910D
:1091C000068CF78DE02D199591E089270895862F5B
:1091D000089581E086270895CF93DF931F92CDB73E
:1091E000DEB7898320911E0B3981E0911F0BF0912E
:1091F000200B822F90E080959095F89400800822B3
:1092000000824BE000C05DE000005A95E9F7008065
:1092100008220894379508F4022A00824A9599F7A3
:1092200078940F90DF91CF91089585ED8093BC00E5
:109230008091BC0084FDFCCF1092F80A0895409103
:10924000D40A262F30E0240F311D21323105DCF401
:109250002091F80A2430C9F4FC0180E090E08617E0
:1092600058F43091D40A2191DC01AC54B54FA30FCE
:10927000B11D2C930196F3CF8091D40A680F6093AF
:10928000D40A80E0089581E0089582E008958FEF88
:109290009FEF08958FEF9FEF08958091B30A90E0BC
:1092A0009195819591090895CF93DF93CB01EA01C0
:1092B000642F0E941F49CE01DF91CF910895CF9373
:1092C000DF931F92CDB7DEB7698361E0CE010196CF
:1092D0000E941F4981E090E00F90DF91CF910895A7
:1092E0000F931F93CF93DF931F92CDB7DEB78C01FF
:1092F000DC01ED91FC910084F185E02D1995892B1D
:1093000051F0BE016F5F7F4FF80184850E94EF45E9
:10931000898190E002C08FEF9FEF0F90DF91CF9196
:109320001F910F910895FC0184850C944046CF93C2
:10933000DF931F92CDB7DEB741E050E0BE016F5F13
:109340007F4FFC0184850E944046181619061CF4C4
:10935000898190E002C08FEF9FEF0F90DF91CF9156
:109360000895FC018485843011F00C94464480E01B
:1093700090E0089544E050E0BC018FE090E00C9450
:10938000863744E050E0BC0185E090E00C948637DD
:1093900044E050E0BC0181E090E00C9486370895F1
:1093A0008CBD9DBD08956F927F928F929F92AF92D8
:1093B000BF92CF92DF92EF92FF921F93CF93DF93F2
:1093C0001F921F92CDB7DEB75C013B016A01FC0121
:1093D0001485143041F481E090E0F5019383828399
:1093E00080E090E05BC07A014130584018F0E12CF9
:1093F00088E0F82ECE0101960E94752A89819A8113
:109400000E94D049812F0E94BF574C0163E070E059
:10941000812F0E94D145873111F08C3121F48E14B7
:109420009F0440F302C0E12CF12CCE0101960E9472
:10943000752A89819A810E94D0499701A30160E031
:1094400070E0812F0E945A5760E270E0812F0E94E5
:10945000652A62E070E0812F0E94D14584FD14C02E
:1094600063E070E0812F0E94D145811104C0812FFB
:109470000E940545B0CFCE0101960E94752A8981D0
:109480009A810E94D049E5CF40E162E070E0812FEF
:109490000E94FB44EF2809F49ECFC6010F900F9065
:1094A000DF91CF911F91FF90EF90DF90CF90BF9011
:1094B000AF909F908F907F906F9008958F929F9222
:1094C000AF92BF92DF92EF92FF920F931F93CF93D1
:1094D000DF931F921F92CDB7DEB7FC0124852430A5
:1094E00009F082C05A018B017C01D12C8D2D0E9484
:1094F0006147811103C0F701D48607C08B7F883193
:10950000D1F3D394F4E0DF12F1CFF70184858430F6
:1095100009F46AC020910302309104022F5F3F4F8B
:1095200011F420E030EC30930402209303024091C8
:1095300003025091040220E061E00E942845F801F6
:1095400082818F3F51F483818F3F99F484818F3FD3
:1095500081F485818F3F69F444C081110AC0F8010C
:109560008381811106C08481811103C08581882394
:10957000C1F1A114B104A9F1F701D484CE0101967F
:109580000E94752A89819A810E94D049B8016E5F34
:109590007F4F8D2D0E940848B5018D2D0E94F74701
:1095A00064E070E08D2D0E94652A0E9424634B01C7
:1095B0005C01F4E98F0EF1E19F1EA11CB11CC701F3
:1095C0000E947A2A873141F161E070E080E090E00A
:1095D0000E94EA620E94D12EC7010E947A2A81115C
:1095E00006C084E0F701848780E090E01DC00E94FF
:1095F000246386169706A806B90608F7F70184853E
:109600000E94054584E0F701848764EA7DE08DEBE4
:1096100097E00E940838E8CF69E97DE08DEB97E09C
:109620000E94083881E090E00F900F90DF91CF9179
:109630001F910F91FF90EF90DF90BF90AF909F90A0
:109640008F90089578941F920F920FB60F92112465
:109650000BB60F92CF92DF92EF92FF920F931F9370
:109660002F933F934F935F936F937F938F939F932A
:10967000AF93BF93CF93DF93EF93FF9380917000ED
:109680008E7F809370000FE310E08BE1E82EF12CC9
:109690009BE2C92ED12CC091210BD091220B209797
:1096A000F9F40332110508F43BC003521109E091AB
:1096B0001F0BF091200B908120911E0B822F809523
:1096C000982390839BE0D7011197F1F79150D9F738
:1096D0008081822B8083C6010197F1F780E00DC065
:1096E0000B301105E8F00B501109E091230BF091BC
:1096F000240BEC0FFD1F319780810E94EC482196CE
:10970000D093220BC093210B809101029091020211
:109710008C179D0708F0BFCF1092220B1092210BDF
:1097200080917000816080937000FF91EF91DF91D4
:10973000CF91BF91AF919F918F917F916F915F91E9
:109740004F913F912F911F910F91FF90EF90DF90DC
:10975000CF900F900BBE0F900FBE0F901F901895DB
:1097600081E08093B20A80910002282F30E0F90155
:10977000ED5BF24FE491F0E0EE0FFF1FED57F34F7A
:10978000459154915093200B40931F0BF901E350E6
:10979000F34FE491E0931E0B61E00E94AE6283E020
:1097A0008093B100E0E7F0E08081816080830895DC
:1097B000CF93DF931816190644F0809170008E7FC6
:1097C000809370001092B20A19C0EC018091230BB3
:1097D0009091240B0E94896DCE01C130D24014F0CB
:1097E00080E092E090930202809301020E94F16C6B
:1097F0009093240B8093230B892B29F4109202025F
:109800001092010208C08091B20A811104C0DF9158
:10981000CF910C94B04BDF91CF910895FF920F93AD
:109820001F93CF93DF938C01F62E8091B20A8111A2
:1098300002C00E94B04BE8012197C11582E0D80711
:1098400098F480910102909102028017910718F418
:10985000C8010E94D84B8091230B9091240B009754
:1098600019F0C80FD91FF882DF91CF911F910F9186
:10987000FF9008951F920F920FB60F9211240BB60E
:109880000F922F933F934F935F936F937F938F9399
:109890009F93AF93BF93EF93FF938091B900887F1D
:1098A000803609F49CC068F5883209F45BC090F4F6
:1098B000803109F454C038F4882309F4F2C08830A8
:1098C00009F44DC0F2C0883109F44CC0803209F46B
:1098D0005DC0EBC0803409F468C048F4803309F4FB
:1098E00055C0883309F0E1C08093F70AD4C08035B1
:1098F00009F44FC0883509F45DC0883409F0D5C03B
:10990000D2C0883909F4C3C0A8F4883709F467C005
:1099100038F4883609F463C0803709F460C0C5C0E4
:10992000883809F4B4C0803909F45FC0803809F080
:10993000BCC05BC0803B09F484C038F4803A09F4B1
:1099400066C0883A09F47DC0B0C0803C09F4A3C069
:10995000883C09F4A0C0883B09F486C0A6C0809169
:109960001D0B10C090911C0B80911B0B981770F56C
:10997000E0911C0B81E08E0F80931C0BF0E0E55012
:10998000F54F80818093BB0085EC82C08093F70AFD
:109990008AC0E0911C0B81E08E0F80931C0B80919C
:1099A000BB00F0E0E550F54F808390911C0B809157
:1099B0001B0B6AC0E0911C0B81E08E0F80931C0B87
:1099C0008091BB00F0E0E550F54F80838091FA0A6A
:1099D000811169C081E08093F90A84EA5DC083E067
:1099E0008093F80A1092F60ACFCF8091F60A80325F
:1099F00008F04DC0E091F60A81E08E0F8093F60AE0
:109A00008091BB00F0E0EA52F54F8083BDCF85EC3A
:109A10008093BC001092F80A8091F60A803230F4EC
:109A2000E091F60AF0E0EA52F54F10826091F60AF2
:109A300070E086ED9AE0E0E0F0E019951092F60A09
:109A400034C084E08093F80A1092D50A1092D40AA8
:109A5000E0E0F0E019958091D40A811105C081E021
:109A60008093D40A1092B40AE091D50A81E08E0F57
:109A70008093D50AF0E0EC54F54F80818093BB00D1
:109A80009091D50A8091D40A981708F47DCF85E883
:109A90008093BC000AC085EC8093BC001092F80A49
:109AA00004C01092F70A0E941549FF91EF91BF91EF
:109AB000AF919F918F917F916F915F914F913F9166
:109AC0002F910F900BBE0F900FBE0F901F90189507
:109AD0008F929F92AF92BF92CF92DF92EF92FF92BE
:109AE0000F931F93CF93DF93CDB7DEB72B970FB6AE
:109AF000F894DEBF0FBECDBF8C01CE0101967C0174
:109B00006C018AE0882E912CA12CB12CC6018E19F3
:109B10009F09411551056105710581F0CB01BA011D
:109B2000A50194010E946E77942F852F605DF60148
:109B300061936F01A901692F782FE8CFFC0131975C
:109B4000EE0DFF1DD8019E012150310940814D933A
:109B50003197E217F307D1F7F801E80FF91F1082E8
:109B60002B960FB6F894DEBF0FBECDBFDF91CF911D
:109B70001F910F91FF90EF90DF90CF90BF90AF902B
:109B80009F908F9008958F929F92AF92BF92CF92A5
:109B9000DF92EF92FF920F931F93CF93DF938C018D
:109BA0004A016901E090B00AF090B10AC62F660F31
:109BB000DD0BE114F10449F1F7018085863029F5C8
:109BC00068EE74E0C7010E9427385C01F2E08F164E
:109BD000910439F083E08816910451F46DEE74E03D
:109BE00002C061EF74E0C7010E9427387C0102C007
:109BF000E12CF12CA114B10451F0F50161857285BD
:109C0000AE01C8010E944C7C08C0E12CF12CAE01D1
:109C100062E97DE0C8010E940F70AE0162EC73E062
:109C2000C8010E942E7CE114F10421F0F701618546
:109C300072850FC0F2E08F169104A1F083E08816C0
:109C4000910461F08A94892899F46091AE0A709128
:109C5000AF0AAE01C8010E942E7C0AC0AE016CE8BA
:109C60007DE003C0AE0169E87DE0C8010E94F16FAC
:109C7000AE0162EC73E0C8010E942E7CC114D104D5
:109C800029F0AE01B601C8010E942E7CC801DF9107
:109C9000CF911F910F91FF90EF90DF90CF90BF90E9
:109CA000AF909F908F900895CF93DF931F921F9254
:109CB000CDB7DEB780914F0B9091500B009711F408
:109CC0008BE59BE0BE016F5F7F4F681B790B072E12
:109CD000000C880B990B0F900F90DF91CF91089596
:109CE000AF92BF92CF92DF92EF92FF920F931F93AA
:109CF000CF93DF93CDB7DEB7AF970FB6F894DEBF43
:109D00000FBECDBF7C015B016A0101E213E01A8343
:109D100009831B821C821D821E82CE0109960E942D
:109D200076441BA70AA71CA61DA61EA61FA68091E7
:109D3000620890916308A0916408B09165088EA3B1
:109D40009FA3A8A7B9A78B839C83AD83BE831886E6
:109D50001F82AE01465D5F4FB501CE0101960E94A4
:109D60002A3F81309105B1F4D701ED91FC91068431
:109D7000F785E02D1DA30CA38CA59DA5AEA5BFA5C1
:109D80008EA39FA3A8A7B9A7A601BE016C5D7F4FB4
:109D9000C7011995AF960FB6F894DEBF0FBECDBFC1
:109DA000DF91CF911F910F91FF90EF90DF90CF90B7
:109DB000BF90AF90089569E57FE08DEB97E00E943A
:109DC0007B5BE0E0F0E01994CF93DF931F92CDB777
:109DD000DEB71982892B21F0FB016281738103C0F8
:109DE000BE016F5F7F4F86E390E00E948C2F64EB93
:109DF00070E18DEB97E00E947B5B0F90DF91CF913C
:109E00000895CF93DF93C0E0D0E060E0CE010E94E0
:109E100050772196C11582E0D807B9F764EA70E15E
:109E20008DEB97E0DF91CF910C947B5B0F931F93A9
:109E3000CF93DF93CDB7DEB72C970FB6F894DEBF84
:109E40000FBECDBF8B0121E233E03A8329831B8211
:109E50001C821D821E8238872F8319861A861B86D4
:109E60001C8683309105B9F144F48130910509F4E1
:109E70005BC0029709F443C064C084309105B9F017
:109E8000059709F05EC0BE01695F7F4FF8018085CC
:109E900091850E94EC3EBE01892B19F0695F7F4FCE
:109EA00002C06F5F7F4F82E190E00E94CD3EBE0115
:109EB000695F7F4FF801868197810E94EC3EBE0169
:109EC000892B19F0695F7F4F02C06F5F7F4F8EE073
:109ED00090E00E94CD3EBE01695F7F4FF801848112
:109EE00095810E94EC3EBE01892B19F0695F7F4F7E
:109EF00002C06F5F7F4F8AE090E00E94CD3EBE01BE
:109F0000695F7F4FF801828193810E94EC3EBE0120
:109F1000892B19F0695F7F4F02C06F5F7F4F86E02A
:109F200090E00E94CD3E0DC0BE016F5F7F4F86E086
:109F300090E00E94CD3E64E970E18DEB97E00E94D5
:109F40007B5B6DE870E18DEB97E00E947B5B2C966C
:109F50000FB6F894DEBF0FBECDBFDF91CF911F913A
:109F60000F910895CF93DF93CDB7DEB72C970FB63F
:109F7000F894DEBF0FBECDBF1C821B821E821D82E5
:109F80008FEF9FEF98878F838CE693E09A83898386
:109F900088E490E09A8789871C861B8663E770E1D6
:109FA0008DEB97E00E947B5B609113067091140625
:109FB000CE0101960E946F346FEFCE0101960E9490
:109FC000523363E670E18DEB97E00E947B5B2C9649
:109FD0000FB6F894DEBF0FBECDBFDF91CF910895CD
:109FE0000F931F93CF93DF93CDB7DEB769970FB66B
:109FF000F894DEBF0FBECDBF8FE290E09A838983D5
:10A00000FE01339687E1DF011D928A95E9F76EE440
:10A0100070E18DEB97E00E947B5B2DE93AE0DE0179
:10A020001196AE01435F5F4F8D01F90161919F0170
:10A03000862F90E074E0959587957A95E1F7895A97
:10A040009C4FFC01808111968C931197E62FEF7045
:10A05000F0E0E95AFC4F808112968C931297129689
:10A06000A417B50711F71E8666EF74E0C8010E94B9
:10A07000087CB8018DEB97E00E94495CC8010E9402
:10A080005F3E1E866EEF74E0C8010E94087CB80136
:10A090008DEB97E00E94495C68E075E0C8010E9482
:10A0A0000E2A69960FB6F894DEBF0FBECDBFDF91C2
:10A0B000CF911F910F910895CF93C1E068EE73E0A7
:10A0C00080E090E00E94EA626C2F8DEB97E00E94A6
:10A0D0004238CF5FC43191F7CF9108950F931F930A
:10A0E000CF93DF93CDB7DEB728970FB6F894DEBFD6
:10A0F0000FBECDBF0E94DF2E62EB7DE08DEB97E0BF
:10A100000E947B5BCE0101960E94A456CE0101966F
:10A110000E944E5601E213E01A8309831B821C82BF
:10A120001D821E82CE0107960E94752A8F81988516
:10A130000E94D04944E050E0BE016D5F7F4F81E056
:10A1400090E00E9456370E94CF49CE0101960E94AE
:10A150004E561A8309831B821C821D821E82CE01E9
:10A1600007960E94752A8F8198850E94D04944E005
:10A1700050E0BE016D5F7F4F85E090E00E94563752
:10A180000E94CF49CE0101960E944E5668ED7DE0B7
:10A190008DEB97E00E947B5B28960FB6F894DEBFAC
:10A1A0000FBECDBFDF91CF911F910F9108957F9288
:10A1B0008F929F92AF92BF92CF92DF92EF92FF92D7
:10A1C0000F931F93CF93DF93CDB7DEB729970FB6C9
:10A1D000F894DEBF0FBECDBF809113069091140698
:10A1E000009709F45FC26AE075E00E9427389093F7
:10A1F0002E0B80932D0B009709F4A5C00E94BC3B49
:10A20000082F10E00115110509F49DC0000F111F62
:10A21000000F111F8091260B9091270B892B09F0BD
:10A2200083C0C8010E94F16C9093270B8093260B8A
:10A2300010923D0B10923C0B1092300B10922F0B92
:10A2400010923B0B10923F0B10923E0B78010130A5
:10A2500082E018071CF0E12C32E0F32EC7010196D2
:10A260000E94F16C9093410B8093400B90933A0BBA
:10A270008093390B8E0D9F1D9093340B8093330B7D
:10A280000E9424636093350B7093360B8093370BD9
:10A290009093380B80E090E0E091400BF091410BFF
:10A2A000E80FF91F10820196E816F906ACF782E074
:10A2B00090E090933D0B80933C0B80E98093C90024
:10A2C0001092C8001092CD0083E08093CC008EE005
:10A2D0008093CA00F0920702E09206022091400BA0
:10A2E0003091410B8091060290910702820F931FDB
:10A2F0009093340B8093330B232B09F41AC162E83B
:10A300007FE08DEB97E00E947B5BB8018DEB97E0DF
:10A310000E9400388DEB97E00E94455C80EA9FE147
:10A320009093320B8093310B65EF7FE08DEB97E0DC
:10A330000E947B5BB8018DEB97E00E9400388DEBAB
:10A3400097E00E94455C60E175E080911306909172
:10A3500014060E9427388C010097A1F00E94BC3B94
:10A360008111EEC00FC069ED7FE08DEB97E00E9498
:10A370007B5BB7018DEB97E00E9400388DEB97E097
:10A380000E94455CE0901306F090140664E175E0CD
:10A39000C7010E94273890932C0B80932B0B6BE105
:10A3A00075E0C7010E9427388C0190930E068093B8
:10A3B0000D0661E275E0C7010E9427389093B10A4B
:10A3C0008093B00A1092AD051092AC0501151105ED
:10A3D00011F1F801E680F78021E7A22E22E0B22EEB
:10A3E00000910D0610910E060115110569F0E1149A
:10A3F000F10451F0F70180858530B1F7C7010E9463
:10A40000BC3B823088F3C8C0F80186819781909365
:10A41000AD058093AC05E0901306F09014066DE056
:10A4200075E0C7010E9427388C019093160680932F
:10A43000150668E275E0C7010E94273890932A0B41
:10A440008093290B01151105A1F0F80106811781F0
:10A450000115110571F0F8018085863031F41A83F9
:10A460000983CE0101960E945122F80102811381D5
:10A47000EFCF64EB7FE08DEB97E00E947B5B6CEAB3
:10A480007FE08DEB97E00E947B5B81E020910D06E1
:10A4900030910E06232B09F480E00E94C12F63EA5D
:10A4A0007FE08DEB97E00E947B5B81E020911506B9
:10A4B00030911606232B09F480E00E94C12F6AE92F
:10A4C0007FE08DEB97E00E947B5B81E020912B0B7E
:10A4D00030912C0B232B09F480E00E94C12F63E9FB
:10A4E0007FE08DEB97E00E947B5B81E02091290B60
:10A4F00030912A0B232B09F480E00E94C12F8DEBB1
:10A5000097E00E94455C0E94544E6B017C016EE80E
:10A510007FE08DEB97E00E947B5B2AE0B701A6010C
:10A520008DEB97E00E94B45B8DEB97E00E94455C59
:10A53000B9C06BE67FE08DEB97E00E940838EECE65
:10A5400061E0C8010E941A38FC01E184F284909114
:10A55000B20A992359F0809170008E7F8093700029
:10A560001092B20A109202021092010283E08093CC
:10A57000000291110E94B04BC7010E94D84B01E02C
:10A5800010E0E016F1060CF4EECE60E0C8010E9487
:10A590000E4C0F5F1F4FF5CFBA82A982FC82EB826F
:10A5A000CE0101960E94FD20CE0101960E942E2030
:10A5B000882309F473C060E070E0CE0101960E9428
:10A5C00097208C0197FF07C01195019511098824E8
:10A5D0008394912C02C0812C912C60E0CE010196D5
:10A5E0000E94EA20C82ED12C8985853019F086304A
:10A5F00021F154C0CD2829F462E0CE0101960E94D9
:10A60000C52061E0802F0E94AE6260E0802F0E9432
:10A61000AA4161ED7FE08DEB97E00E947B5BB80182
:10A620008DEB97E00E9400386CEC7FE08DEB97E0BB
:10A630000E947B5B6AEC7FE02DC0702E61E0802F72
:10A640000E94AE6261E0892821F0CA94CD2829F4E5
:10A6500003C0CA94CD2809F060E0C62ED12C872D06
:10A660000E94AA4165EC7FE08DEB97E00E947B5B46
:10A67000B8018DEB97E00E94003863EC7FE08DEB32
:10A6800097E00E947B5BB6018DEB97E00E9400385B
:10A6900061EC7FE08DEB97E00E947B5BF701E2804D
:10A6A000F3809ECE29960FB6F894DEBF0FBECDBFC5
:10A6B000DF91CF911F910F91FF90EF90DF90CF909E
:10A6C000BF90AF909F908F907F900895CF93DF932E
:10A6D000CDB7DEB72C970FB6F894DEBF0FBECDBF57
:10A6E00063E370E18DEB97E00E947B5B8DEB97E07D
:10A6F0000E94455C88E490E00E9448778B37A1F582
:10A700001C821B821E821D828FEF9FEF98878F8392
:10A710008CE693E09A83898388E490E09A8789871E
:10A720001C861B860E943D60CE0101960E94442A31
:10A730009093140680931306892B19F466E170E157
:10A7400015C06FE070E18DEB97E00E947B5B8DEBB5
:10A7500097E00E94455C0E94D75083E29AE00E94F5
:10A76000824581E090E00CC062E270E18DEB97E001
:10A770000E947B5B8DEB97E00E94455C80E090E05F
:10A780002C960FB6F894DEBF0FBECDBFDF91CF91F0
:10A7900008950C946653CF92DF92EF92FF92CF937D
:10A7A000DF93EC010E9424636B017C0180916C08B3
:10A7B00090916D08DC01ED91FC910084F185E02D14
:10A7C0001995892B79F40E942463DC01CB018C1943
:10A7D0009D09AE09BF0988399A43A105B10530F337
:10A7E00080E00DC080916C0890916D08DC01ED91C6
:10A7F000FC910284F385E02D1995888381E0DF9137
:10A80000CF91FF90EF90DF90CF9008954F925F929D
:10A810006F927F928F929F92AF92BF92CF92DF9270
:10A82000EF92FF920F931F93CF93DF931F921F928C
:10A83000CDB7DEB75C018EE698E00E94CB53811164
:10A840003AC036C08C01CE0101960E94CB538823BA
:10A8500079F1C80101962981F70121937F01422FE7
:10A860004F7750E0449DB001459D700D549D700D93
:10A870001124C60ED71E47E0440C551C661C771CDD
:10A880004A95D1F727FF27C085309105D9F68FEF7C
:10A890009FEF909308098093070980916C0890912D
:10A8A0006D08DC01ED91FC910488F589E02D199586
:10A8B00080E090E08EC090906E0819828FE6E82EBE
:10A8C00088E0F82E01E010E0C12CD12C412C512C55
:10A8D00032014394B8CFF92DF07FFA832FEF280F80
:10A8E000D5012C93F03319F58259974F0E94CB5321
:10A8F0008823F1F2C8018059974F0E94CB538823D7
:10A90000B9F2C8010396D501EC91F0E0E859F74F90
:10A91000E780F12CFE2CEE242085E20EF11C209124
:10A920006E0821FF08C0B2E0EB0EF11C04C020E06D
:10A93000E12CF12C01C022E0422E512CFC01E859FF
:10A94000F74F4F018C01481A590A2EEF622E7724D7
:10A950007A94C801840D951D8C159D0578F5CE015E
:10A9600001960E94CB53882309F4A2CF8091050958
:10A97000909106090097B1F0FA81F03399F4D5016E
:10A980002C91F301E21BF1099F01200F311FE21608
:10A99000F30640F4DC01ED91FC910190F081E02D93
:10A9A000698119950038110518F48981F4018683AD
:10A9B0000F5F1F4FFFEF8F1A9F0ACBCF80910509C2
:10A9C00090910609892B21F40138110508F070CF08
:10A9D000C8010F900F90DF91CF911F910F91FF90C1
:10A9E000EF90DF90CF90BF90AF909F908F907F902F
:10A9F0006F905F904F9008952F923F924F925F9289
:10AA00006F927F928F929F92AF92BF92CF92DF927E
:10AA1000EF92FF920F931F93CF93DF931F92CDB7C7
:10AA2000DEB70E945727382E882309F422C10E94DE
:10AA300024632B013C018091F4089091F508A091CA
:10AA4000F608B091F708A3019201281B390B4A0BB5
:10AA50005B0BDA01C90189399A43A105B105A8F454
:10AA60008091F0089091F108A091F208B091F3085C
:10AA7000A3019201281B390B4A0B5B0BDA01C901B8
:10AA800089399A43A105B105C8F12091F808809150
:10AA90006C0890916D08222371F02CEF3FEF3093FA
:10AAA000080920930709DC01ED91FC910488F589E0
:10AAB000E02D1995DDC020EC20936E0810926F08F0
:10AAC000DC01ED91FC910280F381E02D42E050E049
:10AAD0006EE678E019954092F0085092F108609285
:10AAE000F2087092F3084092F4085092F5086092D0
:10AAF000F6087092F70881E08093F80880916C085E
:10AB000090916D08DC01ED91FC910084F185E02DC0
:10AB10001995892B09F4ADC0CE0101960E94065407
:10AB20005C01892B09F4A0C04092F4085092F5080A
:10AB30006092F6087092F70880916E08807F8033EB
:10AB400009F076C08091F9089091FA08892B09F4F0
:10AB500090C0E980F12CF701E859F74F078110E028
:10AB6000102F00278085080F111D97012059374F9E
:10AB70004901B7016F58774FA801C9010E94E37BD3
:10AB8000B8016E0D7F1DDB01A859B74F18961C92B6
:10AB9000189780916E088670282EE091F908F09140
:10ABA000FA0832E0831337C01996CC901997D12C4C
:10ABB000DC2CCC241A968C91C80ED11C4BEF5FEF85
:10ABC0004E195F09401B510B4A0D5B1D6D58774FA5
:10ABD000C401199580E480936E0820926F08D0928A
:10ABE0007008C092710880916C0890916D08DC012A
:10ABF000ED91FC910280F381E02D44E050E06EE69F
:10AC000078E019954092F0085092F1086092F208AD
:10AC10007092F3082EC04DEF5FEF4E195F09401B95
:10AC2000510B4A0D5B1D6F58774FC401199521C018
:10AC3000803CA9F480ED80936E0810926F0880919B
:10AC40006C0890916D08DC01ED91FC910280F3811C
:10AC5000E02D42E050E06EE678E019950AC0803DB4
:10AC600041F41092F80805C00E945727811101C0D5
:10AC7000312C832D0F90DF91CF911F910F91FF9079
:10AC8000EF90DF90CF90BF90AF909F908F907F908C
:10AC90006F905F904F903F902F900895AF92BF922A
:10ACA000CF92DF92EF92FF921F93CF93DF9300D06A
:10ACB00000D0CDB7DEB76C017C0110E08AE0A82E91
:10ACC000B12C1330A9F0F701828190E0A0E0B0E050
:10ACD00089839A83AB83BC83BE82AD82BE016F5FE2
:10ACE0007F4F8DEB97E00E94572169EC70E114C013
:10ACF000F601858190E0A0E0B0E089839A83AB8380
:10AD0000BC83BE82AD82BE016F5F7F4F8DEB97E04B
:10AD10000E94572166EC70E10E947B5B1F5FFFEF92
:10AD2000EF1AFF0A143069F626960FB6F894DEBFC4
:10AD30000FBECDBFDF91CF911F91FF90EF90DF90BD
:10AD4000CF90BF90AF9008950F931F93CF93DF9351
:10AD50001F921F92CDB7DEB78C0181E293E0F8011C
:10AD6000918380831282138214821582CE01019610
:10AD70000E94752A89819A810E94D049B8016E5F2C
:10AD80007F4F44E050E08FE090E00E9456370E94F1
:10AD9000CF49C8010F900F90DF91CF911F910F9174
:10ADA0000895CF93DF93C8E6D8E080EE8E831F82AC
:10ADB0008C819D81DC01ED91FC910280F381E02D7D
:10ADC00042E050E06EE678E019958FEF9FEF9093A8
:10ADD0000809809307098C819D81DC01ED91FC912C
:10ADE0000680F781E02D19958C819D81DC01ED9124
:10ADF000FC910488F589E02D19950E9424636093E5
:10AE0000F0087093F1088093F2089093F308609330
:10AE1000F4087093F5088093F6089093F708DF9193
:10AE2000CF910895AF92BF92CF92DF92EF92FF92AF
:10AE30000F931F93CF93DF931F921F92CDB7DEB76F
:10AE40007A836983BA01A901E981FA81F770082F31
:10AE500010E0000F111F0D5F194FD8018D919C91CB
:10AE60008E0F9F1F9F01240F351F21303840A0F007
:10AE70007A015B0160E078E06B01CE1ADF0AA6017F
:10AE8000B5010E945637A7014C195D09B5016C0D3B
:10AE90007D1DF801808191810F900F90DF91CF91FE
:10AEA0001F910F91FF90EF90DF90CF90BF90AF90E8
:10AEB0000C9456379F92AF92BF92CF92DF92EF924F
:10AEC000FF920F931F93CF93DF93982E8B015A011C
:10AED000690164E270E00E94D145E82EF12C65E240
:10AEE00070E0892D0E94D145FE2CEE24E82AE8016D
:10AEF000CE0DDF1D9E013770E92CF12CC701880FA4
:10AF0000991FAC0145505A4F7A01FA018081918115
:10AF1000820F931FA9014C0D5D1D4130584090F0E8
:10AF200000E018E0021B130BA801B5010E94863750
:10AF3000A601401B510BB501600F711FF701808105
:10AF4000918102C0A601B5010E948637CC0DDD1D9E
:10AF50004D2F64E270E0892D0E94FB444C2F65E286
:10AF600070E0892DDF91CF911F910F91FF90EF90AD
:10AF7000DF90CF90BF90AF909F900C94FB44FF92D6
:10AF80000F931F93CF93DF93F82E00E010E08F2DE7
:10AF90000E94E837EC01892B21F08F2D0E94E837C1
:10AFA0008C01C017D10799F7CE01DF91CF911F9186
:10AFB0000F91FF90089520E3FC0120833296862FA5
:10AFC00082958F7090E1899F601911246A3014F482
:10AFD000605D01C0695C6293682F8111F0CF0895B4
:10AFE0002F923F924F925F926F927F928F929F9299
:10AFF000AF92BF92CF92DF92EF92FF920F931F9387
:10B00000CF93DF93CDB7DEB7E2970FB6F894DEBFEC
:10B010000FBECDBF7C012A013B0169010E94246360
:10B020004B015C0187010D5B1F4FC8010E94074760
:10B0300018161906A4F00E942463DC01CB018819BC
:10B040009909AA09BB09481659066A067B06D8F071
:10B0500062E370E080E090E00E94EA62E6CF42E2C4
:10B0600050E0BE016F5F7F4FC8010E94BF468981DB
:10B07000823011F080E060C1F801848995898334C1
:10B080009105C1F702C08FEF57C16D817E818F811D
:10B0900098850E94D9774B015C01F601608371832A
:10B0A0008283938346E050E0B701685F7F4FCE0113
:10B0B0004D960E94D67B892BE9F6F701808191811C
:10B0C000A281B38188169906AA06BB0698F28481EC
:10B0D0009581A681B78188159905AA05BB0550F20F
:10B0E00089899A89AB89BC8986879787A08BB18B20
:10B0F0008EECC82ED12CC8010E94DE46F1E0CF1A9A
:10B10000D108C9F7712CC70182969AA789A7F701C0
:10B11000B696FCA7EBA708969EA78DA73C974F0174
:10B12000899698AB8FA73897FAABE9AB1701F6E190
:10B130002F0E311C27018EE1480E511CF801818D24
:10B14000928D181619060CF0F6C0C8010E94DE4652
:10B150008333910509F4C9C0F4F481309105B9F144
:10B160001CF4892B59F3DBC083309105C1F106979C
:10B1700009F0D5C0C8010E94DE466C0144E050E0F1
:10B18000B201C8010E94BF46A12CB12CDD2494E07D
:10B19000C91AD1083FC08A33910509F47AC03CF43A
:10B1A0008533910561F0C69709F43FC0B8C08B3371
:10B1B000910509F484C08F3F910501F2B0C0C80128
:10B1C0000E94DE46C8010E94DE46782EB7CFC80135
:10B1D0000E94DE4644E050E069A97AA93AC0C8015D
:10B1E0000E94DE466C0144E050E0B101C8010E94BB
:10B1F000BF46A12CB12CDD24F4E0CF1AD108AC1449
:10B20000BD040CF09BCFC8010E94DE468FEFA81A48
:10B21000B80AF5CFAC14BD040CF090CFC8010E9461
:10B22000DE46EFEFAE1ABE0AF5CFC8010E94DE4639
:10B23000682EF701828D811110C0838D81110DC0A0
:10B24000848D81110AC0858D811107C044E050E0D2
:10B25000B401C8010E94BF4671CFEFA5F8A9A08034
:10B26000B180C280D380B401CE0183960E944B5C32
:10B270008DA19EA1AFA1B8A5A816B906CA06DB0686
:10B2800029F3662009F45ACFC8010E94DE466A9469
:10B29000F8CFC8010E94DE4644E050E06BA57CA5D3
:10B2A000C8010E94BF46F70166A177A180A591A5BC
:10B2B0000E94D97766A377A380A791A73FCFC80143
:10B2C0000E94DE4644E050E06DA57EA5C8010E94C4
:10B2D000BF46F70162A573A584A595A50E94D977FD
:10B2E00062A773A784A795A729CFC8010E94DE464D
:10B2F00044E050E069A57AA5C8010E94BF46F70165
:10B3000062A173A184A195A10E94D97762A373A3BE
:10B3100084A395A366A777A780AB91AB0FCFC80195
:10B320000E94DE46D82EDD2009F408CFC8010E9415
:10B33000DE46DA94F8CF872DE2960FB6F894DEBF9A
:10B340000FBECDBFDF91CF911F910F91FF90EF9076
:10B35000DF90CF90BF90AF909F908F907F906F9035
:10B360005F904F903F902F900895CF92DF92EF9291
:10B37000FF920F931F93CF93DF936C017A018B01A0
:10B38000C0E0D0E0CE15DF0581F0D8016D918D01D0
:10B39000D601ED91FC910190F081E02DC601199547
:10B3A000892B11F02196EECF7E01C701DF91CF915D
:10B3B0001F910F91FF90EF90DF90CF900895FC01C7
:10B3C000538D448D252F30E0842F90E0821B930B0A
:10B3D000541710F0CF96089501970895FC01918DB0
:10B3E000828D981761F0828DDF01A80FB11D5D96E7
:10B3F0008C91928D9F5F9F73928F90E008958FEF55
:10B400009FEF0895FC01918D828D981731F0828D08
:10B41000E80FF11D858D90E008958FEF9FEF08955F
:10B42000FC01918D228D892F90E0805C9F4F821BC3
:10B4300091098F739927089580E297E00E94105A2E
:10B4400021E0892B09F420E0822F08958DEB97E00D
:10B450000E94105A21E0892B09F420E0822F0895E0
:10B46000FC01848DDF01A80FB11DA35ABF4F2C91A1
:10B47000848D90E001968F739927848FA689B78970
:10B480002C93A089B1898C91837080648C93938D67
:10B49000848D981306C00288F389E02D80818F7D0A
:10B4A00080830895EF92FF920F931F93CF93DF93C2
:10B4B000EC0181E0888F9B8D8C8D981305C0E88905
:10B4C000F989808185FD26C0F62E0B8D10E00F5F77
:10B4D0001F4F0F731127E02E8C8DE8120CC00FB692
:10B4E00007FCFACFE889F989808185FFF5CFCE0185
:10B4F0000E94305AF1CF8B8DFE01E80FF11DE35A07
:10B50000FF4FF0829FB7F8940B8FEA89FB89808107
:10B5100080620AC09FB7F894EE89FF896083E8894A
:10B52000F98980818370806480839FBF81E090E08F
:10B53000DF91CF911F910F91FF90EF900895CF93DE
:10B54000DF93EC01888D8823C9F0EA89FB8980812B
:10B5500085FD05C0A889B9898C9186FD0FC00FB6FD
:10B5600007FCF5CF808185FFF2CFA889B9898C913E
:10B5700085FFEDCFCE010E94305AE7CFDF91CF910A
:10B58000089580E090E0892B21F00E94265A8111D5
:10B5900021C080E090E0892B41F080E090E0892B91
:10B5A00021F00E940000811118C080E090E0892BFA
:10B5B00021F00E941C5A811113C080E090E0892B79
:10B5C000A1F080E090E0892B81F00E9400008111C1
:10B5D0000AC008950E940000DCCF0E940000E5CF61
:10B5E0000E940000EACF0C94000008950E94B77BEF
:10B5F000EF92FF920F931F93CF93DF93EC018B0198
:10B600007A010E942463FE01E857FF4F6083718333
:10B61000828393838C819D81DC01ED91FC9102807A
:10B62000F381E02DA701B801DF91CF911F910F9118
:10B63000FF90EF9019941F93CF93DF93EC01162F97
:10B640000E942463FE01E857FF4F60837183828369
:10B6500093838C819D81DC01ED91FC910190F081BF
:10B66000E02D612FDF91CF911F911994DC01ED91B5
:10B67000FC910190F081E02D19948F929F92AF92EE
:10B68000BF92CF92DF92EF92FF920F931F93CF93CF
:10B69000DF937C018B014C0182E0880E911C5701E5
:10B6A000E5E0AE0EB11CC0E0D0E0F40161914F01C5
:10B6B000C8010E9442386C016EE2C8010E94365BEC
:10B6C0008C0D9D1DC80FD91F8A149B0471F7F701BB
:10B6D0006581C8010E9442388C0F9D1FDF91CF9178
:10B6E0001F910F91FF90EF90DF90CF90BF90AF90A0
:10B6F0009F908F900895EF92FF920F931F93CF9397
:10B70000DF938C017B01C0E0D0E0F701EC0FFD1F5F
:10B710006491662361F0D801ED91FC910190F08174
:10B72000E02DC8011995892B11F02196EECFCE019D
:10B73000DF91CF911F910F91FF90EF9008956115C8
:10B74000710579F0FB0101900020E9F73197AF0115
:10B75000461B570BDC01ED91FC910280F381E02D3B
:10B76000199480E090E008958F929F92AF92BF92DB
:10B77000EF92FF920F931F93CF93DF93CDB7DEB776
:10B78000A1970FB6F894DEBF0FBECDBF7C01FA01C2
:10B79000CB0119A2223008F42AE08E010F5D1F4F61
:10B7A000822E912CA12CB12CBF01A50194010E94E5
:10B7B0006E77F901CA01015011096A3014F4605D15
:10B7C00001C0695CD8016C93232B242B252B61F7D6
:10B7D000B801C7010E949F5BA1960FB6F894DEBF27
:10B7E0000FBECDBFDF91CF911F910F91FF90EF90D2
:10B7F000BF90AF909F908F900895CF92DF92EF927D
:10B80000FF920F931F93CF93DF932115310581F49E
:10B81000DC01ED91FC910190F081E02D642FDF912E
:10B82000CF911F910F91FF90EF90DF90CF901994DF
:10B830002A30310501F577FF1DC06A017B01EC015B
:10B840006DE20E94365B8C0144275527BA014C19E2
:10B850005D096E097F092AE0CE010E94B45B800F6A
:10B86000911FDF91CF911F910F91FF90EF90DF908B
:10B87000CF9008952AE0DF91CF911F910F91FF9013
:10B88000EF90DF90CF900C94B45B6AE074E00C947E
:10B890009F5B0C949F5BDC0181E293E08D939D9311
:10B8A00084E0FB0101900D928A95E1F708951F92C3
:10B8B0000F920FB60F9211240BB60F922F933F9356
:10B8C0004F935F936F937F938F939F93AF93BF93A8
:10B8D000EF93FF9380E297E00E94305AFF91EF913F
:10B8E000BF91AF919F918F917F916F915F914F9198
:10B8F0003F912F910F900BBE0F900FBE0F901F9096
:10B9000018951F920F920FB60F9211240BB60F923B
:10B910002F938F939F93EF93FF93E0913007F091D4
:10B9200031078081E0913607F091370782FD12C020
:10B930009081809139078F5F8F7320913A0782172A
:10B9400051F0E0913907F0E0E05EF84F958F809379
:10B95000390701C08081FF91EF919F918F912F91C5
:10B960000F900BBE0F900FBE0F901F9018951F9257
:10B970000F920FB60F9211240BB60F922F933F9395
:10B980004F935F936F937F938F939F93AF93BF93E7
:10B99000EF93FF938DEB97E00E94305AFF91EF9168
:10B9A000BF91AF919F918F917F916F915F914F91D7
:10B9B0003F912F910F900BBE0F900FBE0F901F90D5
:10B9C00018951F920F920FB60F9211240BB60F927B
:10B9D0002F938F939F93EF93FF93E091CD07F09177
:10B9E000CE078081E091D307F091D40782FD12C089
:10B9F00090818091D6078F5F8F732091D707821730
:10BA000051F0E091D607F0E0E354F84F958F809322
:10BA1000D60701C08081FF91EF919F918F912F9167
:10BA20000F900BBE0F900FBE0F901F9018951F9296
:10BA30000F920FB60F9211240BB60F922F933F93D4
:10BA40004F935F938F939F93EF93FF932091400BBE
:10BA50003091410B80913E0B90913F0BAC014F5FB9
:10BA60005F4F50933F0B40933E0BF901E80FF91FD6
:10BA700080818093CE0080910602909107022091F0
:10BA80003E0B30913F0B8217930748F48FEF9FEFE7
:10BA900090933F0B80933E0B88E48093C900FF9105
:10BAA000EF919F918F915F914F913F912F910F90C7
:10BAB0000BBE0F900FBE0F901F9018951F920F9204
:10BAC0000FB60F9211242F933F938F939F93209142
:10BAD0003C0B30913D0B80913E0B90913F0B213000
:10BAE0003105A9F48F3F2FEF920789F41092C80017
:10BAF0001092CD0089E08093CC0086E28093CA004A
:10BB00001092CE0010923F0B10923E0B17C0892B63
:10BB1000A9F41092C8001092CD0083E08093CC006D
:10BB20008EE08093CA0088E28093C9001092CE0014
:10BB300081E090E090933F0B80933E0B9F918F911B
:10BB40003F912F910F900FBE0F901F9018951F924D
:10BB50000F920FB60F9211240BB60F922F933F93B3
:10BB60004F935F936F937F938F939F93AF93BF9305
:10BB7000EF93FF939091C8008091CE0094FF08C08E
:10BB800081E080933B0B8091400B9091410B57C01B
:10BB900090913B0B913099F481110EC082E080931B
:10BBA0003B0B0E9424636093350B7093360B80939C
:10BBB000370B9093380B3EC010923B0B44C0923031
:10BBC00009F041C0E091390BF0913A0B908189174F
:10BBD00021F091E09093050280832091390B309100
:10BBE0003A0B8091330B9091340B2817390711F5DC
:10BBF00010923B0B809105028823D1F08091310B8C
:10BC00009091320B892BA1F01092C900E091310B79
:10BC1000F091320B199580E98093C9001092C80009
:10BC20001092CD0083E08093CC008EE08093CA0018
:10BC3000109205028091390B90913A0B01969093E6
:10BC40003A0B8093390BFF91EF91BF91AF919F9188
:10BC50008F917F916F915F914F913F912F910F90B5
:10BC60000BBE0F900FBE0F901F901895CF92DF92D2
:10BC7000EF92FF920F931F93CF93DF936C018B0191
:10BC800086E090E00E94F16CEC019093430B80936E
:10BC9000420BF60101900020E9F7CF018C199D09B4
:10BCA0000E94F16C7C01B6010E94277CF601019094
:10BCB0000020E9F73197EC19FD09EE0DFF1D108208
:10BCC000F982E8821B830A838091A9059091AA05D5
:10BCD0009D838C83D093AA05C093A905DF91CF9152
:10BCE0001F910F91FF90EF90DF90CF900895CF922A
:10BCF000DF92EF92FF920F931F93CF93DF93CDB715
:10BD0000DEB7EC970FB6F894DEBF0FBECDBFDC01F7
:10BD10002C91222309F451C063E474E00E941E7048
:10BD20009A8389837E01B3E0EB0EF11C01E010E001
:10BD3000D02EC12E63E474E080E090E00E941E707B
:10BD4000F701819391937F010E31110539F4009130
:10BD5000420B1091430BE980FA8008C00F5F1F4F20
:10BD6000892B31F7F4CFF8010481158101151105F4
:10BD7000A1F0D8016D917C91C7010E941E7C892B96
:10BD800091F7D8011296ED91FC911397BE016F5F68
:10BD90007F4F8D2D9C2D199506C06FEC70E18DEBBA
:10BDA00097E00E9408388DEB97E00E94455C6BECB1
:10BDB00070E18DEB97E00E947B5BEC960FB6F894F8
:10BDC000DEBF0FBECDBFDF91CF911F910F91FF90CE
:10BDD000EF90DF90CF900895FB012481358142815F
:10BDE00053812417350758F440815181DA01A20F9D
:10BDF000B31F8C938481958101969583848380E021
:10BE00000895FC01848195810895089580E090E073
:10BE10000895AF92BF92CF92DF92EF92FF920F936D
:10BE20001F93CF93DF93CDB7DEB7C154D1090FB6BF
:10BE3000F894DEBF0FBECDBF5C016B018A016BE4DD
:10BE400071E18DEB97E00E947B5BB5018DEB97E094
:10BE50000E94495C68E471E18DEB97E00E947B5B96
:10BE6000C114D10409F4A4C00C0D1D1DF8011082E9
:10BE70000E94544E6A3F71051CF463E471E14DC0A9
:10BE80007601E016F10641F0F70161917F018DEB3B
:10BE900097E00E94365BF5CF8DEB97E00E94455C02
:10BEA0008091AE059091AF059E012F5F3F4F7901C4
:10BEB00020E030E0049719F443E050E019C042E07C
:10BEC00050E061E4C7010E94C34DF70101900020DA
:10BED000E9F731978F010E191F09A801B701C501B4
:10BEE0000E943E7C0097A9F020E030E041E050E065
:10BEF00061E4C7010E94C34DF70101900020E9F7FA
:10BF000031978F010E191F09A801B701C5010E94C1
:10BF10003E7C892B39F068E371E18DEB97E00E945C
:10BF20007B5B46C00A0D1B1D6DE275E0C8010E94D7
:10BF30001E7C892B69F4F60101900020E9F7319706
:10BF4000EC19FD09329720F0C6010E94775E30C0DF
:10BF50006FE270E0C8010E94137C5C01009741F021
:10BF6000FC0110828181843219F1FFEFAF1ABF0A00
:10BF7000F80180818432E1F0B801C7010E945626A1
:10BF8000C7010E942E20882399F029858091AE0553
:10BF90009091AF05273019F48430910549F041E0C4
:10BFA000049709F440E09501B601C7010E94D11B36
:10BFB000CF5BDF4F0FB6F894DEBF0FBECDBFDF9172
:10BFC000CF911F910F91FF90EF90DF90CF90BF9096
:10BFD000AF900895DF92EF92FF920F931F93CF934C
:10BFE000DF9300D000D0CDB7DEB760E571E18DEB17
:10BFF00097E00E947B5B0DE91AE0D12C80E1E82EEE
:10C00000F12CF8018081803130F466E375E08DEB2E
:10C0100097E00E94495CF8018081F5E090E0A0E0A3
:10C02000B0E089839A83AB83BC83FE82ED82BE013C
:10C030006F5F7F4F8DEB97E0DF1639F00E9457213D
:10C040006EE471E10E947B5B04C00E9457210E9454
:10C05000455CD3940F5F1F4F86E0D812D2CF26964F
:10C060000FB6F894DEBF0FBECDBFDF91CF911F9109
:10C070000F91FF90EF90DF900895CF92DF92EF92B3
:10C08000FF928091130690911406892B09F44CC0FD
:10C090000E94544E6B017C0160E271E18DEB97E0F0
:10C0A0000E947B5B2AE0B701A6018DEB97E00E941E
:10C0B000B45B80911306909114060E94192A109285
:10C0C000140610921306109216061092150610927E
:10C0D0000E0610920D061092B10A1092B00A10923C
:10C0E0002A0B1092290B10922E0B10922D0B1092EE
:10C0F0002C0B10922B0B0E94544E6B017C016BE1B8
:10C1000071E18DEB97E00E947B5B2AE0B701A6010D
:10C110008DEB97E00E94B45B8DEB97E0FF90EF9082
:10C12000DF90CF900C94455CFF90EF90DF90CF9024
:10C1300008955F926F927F928F929F92AF92BF927B
:10C14000CF92DF92EF92FF920F931F93CF93DF93E3
:10C15000CDB7DEB7E4970FB6F894DEBF0FBECDBF04
:10C160006C017B013A01590161E00E94EA20002341
:10C1700061F0682F6062C6010E94C5206AE071E12B
:10C180008DEB97E00E947B5BC0C01AA219A2FE0152
:10C19000B3968EE0DF011D928A95E9F720E030E04A
:10C1A00043E050E060E2CE0101960E94C34DD6010B
:10C1B0001296ED91FC9113976081718140E250E0FD
:10C1C000CE0101960E942E7CB2E0EB16F104C9F07C
:10C1D0003CF4E114F104E1F0EA94EF2879F05FC057
:10C1E00086E0E816F10451F09EE0E916F10481F0D2
:10C1F000A5E0EA16F10409F052C003C064E674E059
:10C2000002C067E674E0CE0181960E94277C50C090
:10C21000A114B10409F44CC08501C12CD12C88E3D0
:10C22000A82E85E0B82E94E0592E7E01B1E3EB0EE6
:10C23000F11C4301E1E08E1A9108C614D704C4F53D
:10C24000D8018C9111969C910E5F1F4F9F938F93F5
:10C25000BF92AF921F925F92FF92EF920E945B7C1F
:10C2600040E150E0B701CE0181960E942E7C0FB6CE
:10C27000F894DEBF0FBECDBFC814D90461F06BE3E4
:10C2800075E0C7010E94277C40E150E0B701CE0174
:10C2900081960E942E7CFFEFCF1ADF0ACECF6CEF83
:10C2A00070E18DEB97E00E947B5B8FEF9FEF2FC0DB
:10C2B00066EF70E18DEB97E00E947B5BBE016F5FE4
:10C2C0007F4F8DEB97E00E94495C63EF70E18DEB4F
:10C2D00097E00E947B5BBE016F5D7F4F8DEB97E027
:10C2E0000E94495C8DEB97E00E94455C0E945727B5
:10C2F000882359F08091AB05811107C0BE016F5DA5
:10C300007F4FCE0101960E94692880E090E0E4967C
:10C310000FB6F894DEBF0FBECDBFDF91CF911F9156
:10C320000F91FF90EF90DF90CF90BF90AF909F90D4
:10C330008F907F906F905F900895FF920F931F935F
:10C34000CF93DF93CDB7DEB729970FB6F894DEBF52
:10C350000FBECDBF8C010E942E20882309F46BC034
:10C3600060E0C8010E94EA20D8011896FC90B7E06E
:10C37000FB1671F0823009F45CC020F4813009F4BE
:10C380005DC006C0853009F454C0863009F456C03B
:10C39000C8010E947320362F272F4F2D50E04A30BE
:10C3A000510508F046C0FA018827EE51FF4F8F4F24
:10C3B0000C94D177D8011496ED91FC911597808556
:10C3C0008530B9F567EE70E18DEB97E00E947B5BFD
:10C3D000D8011496ED91FC911597068117810115EE
:10C3E000110539F1F80161857285CE0101960E942F
:10C3F0005626CE0101960E942E20882311F1CE01EF
:10C4000001960E949D61892BE1F06FED70E18DEB4B
:10C4100097E00E947B5B12C0292F990F330B03C05A
:10C42000832F922F9C0181E090E0232B81F480E008
:10C430000EC080E004C08FEF9FEF09C081E090E064
:10C4400006C0D80112960D911C911397C8CF29965A
:10C450000FB6F894DEBF0FBECDBFDF91CF911F9115
:10C460000F91FF9008953FB7F8948091490B9091F8
:10C470004A0BA0914B0BB0914C0B26B5A89B05C065
:10C480002F3F19F00196A11DB11D3FBFBA2FA92F53
:10C49000982F8827820F911DA11DB11DBC01CD01D0
:10C4A00042E0660F771F881F991F4A95D1F70895BC
:10C4B00090E0FC013197E231F10508F04EC0882789
:10C4C000E451FF4F8F4F0C94D177809180008F778C
:10C4D00003C0809180008F7D8093800008958091BB
:10C4E0008000877FF9CF84B58F7702C084B58F7DB8
:10C4F00084BD08958091B0008F7703C08091B00013
:10C500008F7D8093B0000895809190008F7707C051
:10C51000809190008F7D03C080919000877F8093F1
:10C52000900008958091A0008F7707C08091A000AF
:10C530008F7D03C08091A000877F8093A000089525
:10C54000809120018F7707C0809120018F7D03C0EB
:10C5500080912001877F809320010895CF93DF93FE
:10C5600090E0FC01E350F34F2491FC01ED5BF24FAE
:10C570008491882361F190E0880F991FFC01ED51AF
:10C58000F34FC591D491FC01ED57F34FA591B491B0
:10C59000611109C09FB7F894888120958223888310
:10C5A000EC912E230BC0623061F49FB7F894888120
:10C5B000322F309583238883EC912E2B2C939FBFB1
:10C5C00006C08FB7F894E8812E2B28838FBFDF91A8
:10C5D000CF9108958F929F92AF92BF92CF92DF92A8
:10C5E000EF92FF926B017C010E9433624B015C0170
:10C5F000C114D104E104F104F1F00E943362DC01C2
:10C60000CB0188199909AA09BB09883E9340A10565
:10C61000B10570F321E0C21AD108E108F10888EEF3
:10C62000880E83E0981EA11CB11CC114D104E10442
:10C63000F10419F7DDCFFF90EF90DF90CF90BF901E
:10C64000AF909F908F9008952FB7F8946091450B0D
:10C650007091460B8091470B9091480B2FBF089526
:10C660001F920F920FB60F9211242F933F938F9327
:10C670009F93AF93BF938091450B9091460BA091F0
:10C68000470BB091480B3091440B23E0230F2D371B
:10C6900020F40196A11DB11D05C026E8230F0296C6
:10C6A000A11DB11D2093440B8093450B9093460B25
:10C6B000A093470BB093480B8091490B90914A0B84
:10C6C000A0914B0BB0914C0B0196A11DB11D809315
:10C6D000490B90934A0BA0934B0BB0934C0BBF911B
:10C6E000AF919F918F913F912F910F900FBE0F901F
:10C6F0001F901895CF93DF93CDB7DEB7C656D109FB
:10C700000FB6F894DEBF0FBECDBF789484B58260BB
:10C7100084BD84B5816084BD85B5826085BD85B5E5
:10C72000816085BD80916E00816080936E00109263
:10C7300081008091810082608093810080918100DE
:10C74000816080938100809180008160809380006F
:10C750008091B10084608093B1008091B0008160CD
:10C760008093B000809191008260809391008091CD
:10C77000910081608093910080919000816080930E
:10C7800090008091A10082608093A1008091A1001F
:10C7900081608093A1008091A00081608093A000BF
:10C7A000809121018260809321018091210181602B
:10C7B00080932101809120018160809320018091EC
:10C7C0007A00846080937A0080917A0082608093FE
:10C7D0007A0080917A00816080937A0080917A005B
:10C7E000806880937A001092C1001092EC0510923C
:10C7F000AA051092A90526E040E052EC61E070E045
:10C800008DEB97E00E94A0386BE578E08DEB97E028
:10C810000E947B5B6EE670E586ED93E00E94365EDB
:10C8200062EB7FE48BED93E00E94365E69EC73E58A
:10C8300080EE93E00E94365E62E072E385EE93E064
:10C840000E94365E64E67BE289EE93E00E94365EEB
:10C850006CE570E58DEE93E00E94365E60EF7FE45C
:10C8600082EF93E00E94365E66E17FE486EF93E01C
:10C870000E94365E64EE7EE489EF93E00E94365EAD
:10C8800061E07FE48DEF93E00E94365E6BED7EE425
:10C8900083E094E00E94365E0E94DF2E5DE9C52EA3
:10C8A0005AE0D52E5601F12C00E010E0C8010E949C
:10C8B0004877F50181935F0181508E3F10F4FF248A
:10C8C000F3940F5F1F4F0630110581F7FF20B1F180
:10C8D0000E94EA5F0E94665361E08DE00E94AE62B2
:10C8E00026E040E855E260E070E080E297E00E94D8
:10C8F000A03886EC9EE290931E0A80931D0A80E683
:10C900009BE29093200A80931F0A8CE59BE2909310
:10C91000220A8093210A64E170E080E090E00E94A6
:10C92000EA6289E09FE59093FA088093F90864EF42
:10C9300071E080E090E00E94EA625BC06FE578E021
:10C940008DEB97E00E947B5B43EAA42E4AE0B42E75
:10C9500004EC13E040E150E060E070E0C8010E94A8
:10C96000B46EF60161936F016AE370E0C8010E9442
:10C97000137C009709F4ACCFFC012081222309F439
:10C98000A7CF8C010F5F1F4FAC14BD0419F7A0CFC8
:10C990008DEB97E00E94EE59182F8A3061F5E091F7
:10C9A000EC05F0E0E055FA4F10826AE074E08DEBA0
:10C9B00097E00E94495C80EB95E00E94775E1092C0
:10C9C000EC058DEB97E00E94105A892B09F70E9425
:10C9D0006411029714F00E94FC540E94B9228091C5
:10C9E0000D0690910E06892B49F50E94C22B0E94DC
:10C9F000C15AA895E6CF8D3091F2883069F468E08D
:10CA00008DEB97E00E94365B8091EC058823C9F29C
:10CA100081508093EC05D5CF682F8DEB97E00E9475
:10CA2000365BE091EC05EB3360F681E08E0F80938E
:10CA3000EC05F0E0E055FA4F1083C3CF8091AE05CE
:10CA40009091AF05049709F4CAC30E942463009132
:10CA5000ED051091EE052091EF053091F0050617D8
:10CA600017072807390708F0BAC320E022242394C7
:10CA7000312CE091AC05F091AD05309709F4AFC3CE
:10CA80002111ADC38085853009F092C321E732E0E2
:10CA900063963FAF2EAF63976596FFAFEEAF659796
:10CAA000CE018F5A9F4F0E94FD200E9424632B01CC
:10CAB0003C016A968FAD6A97843061F008F460C3D8
:10CAC000883009F45DC3893009F4D8C0853009F095
:10CAD0005CC356C380910B0690910C06892B09F01C
:10CAE000C5C0CE018F5A9F4F0E9474288111BEC0CD
:10CAF0006796AEACBFAC6797F5018085853009F0CD
:10CB000064C4C5010E94BC3BC82ED12CF2E0CF16F4
:10CB1000D1040CF45AC430920C0620920B0660E04B
:10CB200070E0CE018F5A9F4F0E9497204C0161E028
:10CB300070E0CE018F5A9F4F0E9497208C01F5E044
:10CB4000CF16D1040CF4B2C464E0C5010E941A38B7
:10CB5000FC01C184D28426E240E855E260E070E046
:10CB600080E297E00E94A03880920B0980E297E073
:10CB700090930A09809309091092160A1092180AD4
:10CB80001092170AF1E0CF16D10409F43FC40CF457
:10CB900023C432E0C316D10409F02AC410930D094E
:10CBA00000930C0930920F0920920E0983E00E9435
:10CBB00005396F968FAF6F976F965FAD6F97511175
:10CBC00036C48091100990911109A1969FAF8EAF44
:10CBD000A197092E000CAA0BBB0B89839A83AB8308
:10CBE000BC83E0E1F0E0FE83ED836596EEADFFAD42
:10CBF0006597C080D18067EE78E08DEB97E00E946A
:10CC00007B5BB6018DEB97E00E94495C60EE78E0BB
:10CC10008DEB97E00E947B5BBE016F5F7F4F8DEBDA
:10CC200097E00E9457210E94455CA1966EAD7FADB2
:10CC3000A197CE018F5A9F4F0E94AE2810920C06EA
:10CC400010920B06C090AC05D090AD05F601828124
:10CC5000938121E732E03A8329839C838B83CE0141
:10CC600001960E94FD20CD2809F000C4CE018F5A04
:10CC70009F4F0E94722980ED97E089C280910B0638
:10CC800090910C06892B91F7CE018F5A9F4F0E94ED
:10CC900074288111EBCF30920C0620920B060E9473
:10CCA00066366C01892B19F086E0F601808720E05A
:10CCB00030E043E050E060E2CE0101960E94C34DB7
:10CCC0006596EEADFFAD6597608171814FE150E0F3
:10CCD000CE0101960E942E7C6DE074E0CE0101969B
:10CCE0000E94087C26E040E855E260E070E080E2C7
:10CCF00097E00E94A03860E070E0CE018F5A9F4F0D
:10CD00000E94972080930B0980E297E090930A0994
:10CD1000809309091092160A1092180A1092170AA5
:10CD200024E338E030930D0920930C094AE050E0E9
:10CD300050930F0940930E0983E00E940539811139
:10CD4000C1C060EC78E08DEB97E00E947B5B00E176
:10CD500019E024E2A22E29E0B22EF80181919191EE
:10CD60008F01092E000CAA0BBB0B25968CAF9DAF33
:10CD7000AEAFBFAF259720E130E027963FAF2EAF93
:10CD80002797BE016F5B7F4F8DEB97E00E94572185
:10CD90006EEB78E00E947B5BA016B106F1F68DEB9E
:10CDA00097E00E94455C6091140970911509072E67
:10CDB000000C880B990B0E940B7920E030E048ECC6
:10CDC00052E40E9461789B01AC0163E174E0C6010A
:10CDD0000E94D1290091180910911909A80165E153
:10CDE00074E0C6010E94663860911A0970911B09AF
:10CDF000072E000C880B990B0E940B7920E030E085
:10CE000048EC52E40E9461789B01AC0169E174E056
:10CE1000C6010E94D12960911C0970911D09072E3D
:10CE2000000C880B990B0E940B7920E030E040E267
:10CE300051E40E9461789B01AC0167E174E0C60196
:10CE40000E94D12940911009509111096BE174E0C1
:10CE5000C6010E946638012B09F452C067968EAD58
:10CE60009FAD6797FC012085253009F049C061E03E
:10CE70000E941A38009709F443C024E630E06C960B
:10CE80003FAF2EAF6C97FC0161857285CE018F5B41
:10CE90009F4F0E945626CE018F5B9F4F0E942E20EF
:10CEA000882371F1E12CF12C01E09E01265A3F4FBD
:10CEB00041E050E060E070E0CE018F5B9F4F0E9448
:10CEC000DF081EC090E0A0E0B0E025968CAF9DAFDB
:10CED000AEAFBFAF259720E130E027963FAF2EAF32
:10CEE000279768EA78E08DEB97E00E947B5BBE01B4
:10CEF0006F5B7F4F8DEB97E00E9457210E94455C4E
:10CF00008091100983FF14C08EE398E090930D097F
:10CF100080930C0930920F0920920E0983E00E9441
:10CF2000053981110CC0409110095091110902C0BE
:10CF300040E050E06EE174E0C6010E94663862E3B2
:10CF400070E080E090E00E94EA6243E150E050939C
:10CF50000D0940930C0984E090E090930F098093B1
:10CF60000E0983E00E9405398111A7C06EE978E0BF
:10CF70008DEB97E00E947B5B00E119E098E1A92E20
:10CF800099E0B92EF801619171918F018DEB97E0D5
:10CF90000E9400386CE978E08DEB97E00E947B5BA3
:10CFA000A016B10679F78DEB97E00E94455C0091E1
:10CFB00010091091110901151105D1F0B801012EC8
:10CFC000000C880B990B0E940B792DEE3EE94CE387
:10CFD0005EE30E94C07922E538EB42E152E40E9410
:10CFE000EF779B01AC0162E274E0C6010E94D12997
:10CFF0006091120970911309072E000C880B990B90
:10D000000E940B792DEE3EE94CE35EE30E94C0796D
:10D0100022E538EB42E152E40E94EF774B015C01DC
:10D020009B01AC0161E174E0C6010E94D1296091CD
:10D0300016097091170916161706A4F4072E000C8E
:10D04000880B990B0E940B7920E030E040E251E41C
:10D050000E9461789B01AC0166E274E0C6010E9407
:10D06000D12907C040E050E066E274E0C6010E94AA
:10D07000663820E030E040E252E4C501B4010E948D
:10D08000BB791816B4F5012BA1F10E94572788230C
:10D0900029F08091AB05882309F42CC2E12CF12CF6
:10D0A00001E020E030E040E050E062E070E0CE01DE
:10D0B0008F5A9F4F0E94DF081CC090E0A0E0B0E0B4
:10D0C00025968CAF9DAFAEAFBFAF259720E130E086
:10D0D00027963FAF2EAF279766E878E08DEB97E075
:10D0E0000E947B5BBE016F5B7F4F8DEB97E00E94E0
:10D0F000572180E091E00E94F16C8C01892B61F155
:10D1000025961FAE1EAE259727961FAE1EAE2797FB
:10D110008FEF9FEF29969FAF8EAF29978DE392E017
:10D1200023969FAF8EAF23972B961FAE1EAE2B97E5
:10D130002D961FAF0EAF2D9780E091E061969FAFC7
:10D140008EAF61972F961FAE1EAE2F97B601CE0100
:10D150008F5B9F4F0E946F340E945727882329F0CE
:10D160008091AB05882309F4D0C1C8010E94896D64
:10D17000C6010E94192A10920C0610920B0676CD59
:10D18000CE018F5A9F4F0E94722984E690E0092EAB
:10D19000000CAA0BBB0B480E591E6A1E7B1E409248
:10D1A000ED055092EE056092EF057092F00521E0DA
:10D1B000E091AC05F091AD05828193819093AD052E
:10D1C0008093AC05892B09F054CCE0910D06F091C9
:10D1D0000E06868197819093AD058093AC050E94E1
:10D1E00024630091F1051091F2052091F30530912F
:10D1F000F405601771078207930708F4F6CBE091F6
:10D200000D06F0910E06309709F4EFCB06811781D9
:10D21000F12C0115110541F1F8018085853001F5EA
:10D2200060E0C8010E941A38FC0181859285A385BF
:10D23000B4850597A105B10599F4C8010E94BC3BCE
:10D2400090E005976CF064E0C8010E941A381C0158
:10D25000892B31F0C1010E94BC3B823008F05BC1D8
:10D26000F80102811381D5CF0E942463DC01CB0138
:10D27000805D9A48AF4FBF4F8093F1059093F205C0
:10D28000A093F305B093F4050E94544E2B013C018A
:10D290000E9424634B015C010E945727882309F4F4
:10D2A00062C020E030E041E050E060E4CE01019651
:10D2B0000E94C34D40E450E067E279E0CE01019660
:10D2C0000E94F16F62EC73E0CE0101960E94087C2F
:10D2D00040E450E06EE179E0CE0101960E94F16FEA
:10D2E000B301A201CE018F5B9F4F0E94684DBE012A
:10D2F0006F5B7F4FCE0101960E94692820E030E0ED
:10D3000041E050E060E4CE0101960E94C34D40E44C
:10D3100050E067E279E0CE0101960E94F16F62EC85
:10D3200073E0CE0101960E94087C40E450E067E182
:10D3300079E0CE0101960E94F16FC501B40128EE9B
:10D3400033E040E050E00E946E77BA01A901CE01BF
:10D350008F5B9F4F0E94684DBE016F5B7F4FCE0178
:10D3600001960E946928FF20C1F00E94544E4B0193
:10D370005C0162E379E08DEB97E00E947B5B2AE041
:10D38000B501A4018DEB97E00E94B45B63E474E007
:10D390008DEB97E00E94495C28CB0E94544E4B01D4
:10D3A0005C0160E379E08DEB97E00E947B5B2AE013
:10D3B000B501A4018DEB97E00E94B45B6EE279E0C9
:10D3C0008DEB97E00E947B5B10CB64E079E08DEB06
:10D3D00097E00E947B5B4ACCCD2811F510930D0994
:10D3E00000930C0930920F0920920E0981E0DFCBE7
:10D3F00043E0C416D104A1F410930D0900930C0965
:10D4000030920F0920920E0984E0D1CB10930D09C0
:10D4100000930C09D0920F09C0920E0982E0C7CB8D
:10D420006CEE78E08DEB97E00E947B5BC5CB6F964E
:10D43000FFAD6F978F2F90E0A0E0B0E089839A83D3
:10D44000AB83BC8320E130E03E832D836AEC78E03F
:10D450008DEB97E00E947B5BBE016F5F7F4F8DEB92
:10D4600097E00E9457210E94455CE8CBCE010196CF
:10D470000E942E20882309F4F9CB8985843009F095
:10D48000F5CB60E070E0CE0101960E9497208816EF
:10D49000990609F0EBCB61E070E0CE0101960E94A5
:10D4A00097200817190709F0E1CB04C082E0C82EC5
:10D4B000D12C51CBA1966EAD7FADA197CE01019637
:10D4C0000E94AE28E091AC05F091AD058281938178
:10D4D0009093AD058093AC05892B09F0C7CBE09103
:10D4E0000D06F0910E06868197819093AD0580938D
:10D4F000AC05BCCB6596EEADFFAD659760817181E3
:10D5000086E394E00E940E2AC9CDB801CE010196AF
:10D510000E940E2A2ACE61E0C8010E941A38FC013E
:10D52000F184D28462E0C8010E941A38FC0181842F
:10D530009284A384B48463E0C8010E941A38FC0179
:10D540002185328543855485A5962CAF3DAF4EAFDE
:10D550005FAFA59760E0C1010E941A38FC014184C9
:10D5600052846384748461E0C1010E941A38FC0112
:10D5700041855285638574854115510561057105A5
:10D5800071F4F801608171818DEB97E00E94495C34
:10D5900067E679E08DEB97E00E947B5B14C0415019
:10D5A000510961097109FC014187528763877487BA
:10D5B000452B462B472B39F4F801608171818AE2B3
:10D5C00094E00E940E2A20E030E048E152E4C301DA
:10D5D000B2010E94BB7918163CF4F8016081718198
:10D5E00086E394E00E940E2A6D96FFAE6D976E96CC
:10D5F000DFAE6E97C501B4010E940B794B015C014F
:10D60000A396CEACDFACA397F8010190F081E02D9A
:10D61000A796FFAFEEAFA7978DEB97E00E94455C12
:10D62000A7966EAD7FADA7978DEB97E00E94495C02
:10D6300061E679E08DEB97E00E947B5B42E0C501FB
:10D64000B4010E94822A6BE579E08DEB97E00E949D
:10D650007B5B42E0C301B2010E94822A65E579E06A
:10D660008DEB97E00E947B5BA3966EAD7FADA39799
:10D670008DEB97E00E9400386E962EAD3FAD6E9711
:10D6800061E08F2D37FF08C081950E94AE6232E0C5
:10D69000C316D10449F41FC00E94AE6242E0C41612
:10D6A000D10409F069C01CC035E0C316D10499F05B
:10D6B00061E0C1010E941A38FC0181859285A38531
:10D6C000B485892B8A2B8B2B91F46E962EAD3FADB2
:10D6D0006E9737FF05C060E08F2D81950E94AA41AB
:10D6E00060E08F2D0E94AA4160E579E021C020E032
:10D6F00030E040E85FE3C501B4010E94EF779B0191
:10D70000AC01C301B2010E945C7887FF18C06E961D
:10D710002EAD3FAD6E9737FF05C060E08F2D819530
:10D720000E94AA4161E08F2D0E94AA416CE479E039
:10D730008DEB97E00E947B5BFF24F39491CDA301D6
:10D740009201C501B4010E945C78181694F06E969F
:10D750004EAD5FAD6E9757FF05C061E08F2D81958F
:10D760000E94AA4160E08F2D0E94AA4167E479E0FF
:10D77000DFCF68E379E0DCCF45E0C416D10409F4DB
:10D78000AFCF96CFE0E2F7E01382128248EE53E08B
:10D7900060E070E044835583668377838FE892E08E
:10D7A0009183808325ED30E03587248724ED30E0B8
:10D7B0003787268720ED30E0318B208B21ED30E05C
:10D7C000338B228B22ED30E0358B248B26ED30E03D
:10D7D000378B268B118E128E138E148EEDEBF7E0A5
:10D7E0001382128244835583668377839183808377
:10D7F00085EC90E09587848784EC90E09787868716
:10D8000080EC90E0918B808B81EC90E0938B828B0D
:10D8100082EC90E0958B848B86EC90E0978B868BE6
:10D82000118E128E138E148EE0E3FAE081E293E003
:10D83000918380831282138214821582E6E3FAE0D8
:10D84000918380831282138214821582ECE3FAE0C2
:10D85000918380831282138214821582EAE5F8E0B4
:10D86000918380831282138214821582E2E4FAE0AB
:10D87000918380831282138214821582E8E4FAE095
:10D88000918380831282138214821582EEE4FAE07F
:10D89000918380831282138214821582E4E5FAE078
:10D8A000918380831282138214821582E0E6F8E06D
:10D8B000918380831282138214821582EAE5FAE052
:10D8C00013821282448355836683778321EA32E090
:10D8D00031832083E6E6FAE091838083128213820B
:10D8E00014821582ECE6FAE091838083128213821F
:10D8F00014821582E3E2FAE0138212824483558394
:10D90000668377832BEF32E03183208324E0248702
:10D9100010921E0A10921D0A1092200A10921F0ADD
:10D920001092220A1092210AA8E6B8E013961C92DF
:10D930001E92129723EB32E011963C932E93909314
:10D94000FC088093FB081092FD081092FE081092CC
:10D95000FF08109200092FEF3FEF30930809209342
:10D9600007091596FC93EE931497109206091092EE
:10D970000509E2E7FAE09183808312821382148220
:10D980001582E8E7FAE09183808312821382148281
:10D990001582EEE7FAE0918380831282138214826B
:10D9A0001582E4E8FAE09183808312821382148264
:10D9B0001582EAE8FAE0918380831282138214824E
:10D9C0001582E0E9FAE08FEF8083128211821486DB
:10D9D00013868FEF9FEFDC0187839087A187B28743
:10D9E00008950F931F93CF93DF938230910510F426
:10D9F00082E090E0E091510BF091520B20E030E09A
:10DA0000A0E0B0E0309719F140815181028113818B
:10DA100048175907C8F08417950769F4109731F033
:10DA200012960C93129713961C9327C00093510BD8
:10DA30001093520B22C02115310519F042175307DC
:10DA400018F49A01BD01EF01DF01F801DBCF2115C8
:10DA50003105F9F0281B390B2430310580F48A8117
:10DA60009B816115710521F0FB019383828304C0C2
:10DA70009093520B8093510BFE01329644C0FE01ED
:10DA8000E20FF31F81939193225031093983288348
:10DA90003AC020914F0B3091500B232B41F4209131
:10DAA0000A0230910B023093500B20934F0B2091C0
:10DAB0000802309109022115310541F42DB73EB716
:10DAC00040910C0250910D02241B350BE0914F0B3D
:10DAD000F091500BE217F307A0F42E1B3F0B281711
:10DAE000390778F0AC014E5F5F4F2417350748F0D7
:10DAF0004E0F5F1F5093500B40934F0B81939193A8
:10DB000002C0E0E0F0E0CF01DF91CF911F910F91D3
:10DB10000895CF93DF93009709F481C0FC013297F9
:10DB200013821282A091510BB091520B109781F485
:10DB300020813181820F931F20914F0B3091500B28
:10DB40002817390751F5F093500BE0934F0B67C03E
:10DB5000ED0120E030E0CE17DF0740F44A815B8121
:10DB60009E0141155105F1F0EA01F5CFD383C2833F
:10DB700040815181840F951FC817D90759F48881B6
:10DB80009981840F951F0296918380838A819B815E
:10DB9000938382832115310529F4F093520BE0938E
:10DBA000510B3DC0E901FB83EA8349915991C40FB0
:10DBB000D51FEC17FD0761F480819181840F951FBB
:10DBC0000296E90199838883828193819B838A836A
:10DBD000E0E0F0E012968D919C911397009719F078
:10DBE000FD01DC01F7CF8D919C9111979D012E5F76
:10DBF0003F4F820F931F20914F0B3091500B2817EE
:10DC0000390769F4309729F41092520B1092510B96
:10DC100002C013821282B093500BA0934F0BDF917E
:10DC2000CF9108958F929F92AF92BF92CF92DF9241
:10DC3000EF92FF92CF93DF93EC01688179818A8123
:10DC40009B81611571058105910521F464E279EDEF
:10DC50008BE597E02DE133EF41E050E00E949077B3
:10DC600049015A019B01AC01A7EAB1E40E94AF77D8
:10DC70006B017C01ACEEB4EFA50194010E94BD776D
:10DC8000DC01CB018C0D9D1DAE1DBF1DB7FF03C078
:10DC90000197A109B04888839983AA83BB83BC01FB
:10DCA000CD019F77DF91CF91FF90EF90DF90CF90E4
:10DCB000BF90AF909F908F9008958F929F92AF9258
:10DCC000BF92CF92DF92EF92FF9260910E0270911D
:10DCD0000F0280911002909111026115710581056A
:10DCE000910521F464E279ED8BE597E02DE133EFC6
:10DCF00041E050E00E94907749015A019B01AC013C
:10DD0000A7EAB1E40E94AF776B017C01ACEEB4EFFF
:10DD1000A50194010E94BD77DC01CB018C0D9D1DF6
:10DD2000AE1DBF1DB7FF03C00197A109B048809386
:10DD30000E0290930F02A0931002B0931102BC0147
:10DD4000CD019F77FF90EF90DF90CF90BF90AF9085
:10DD50009F908F90089560930E0270930F028093AE
:10DD600010029093110208953F924F925F926F922A
:10DD70007F928F929F92AF92BF92CF92DF92EF925B
:10DD8000FF920F931F93CF93DF935C016B017A0196
:10DD90006115710519F0FB0191838083E114F10491
:10DDA00029F0C7010297839708F0C9C0E5012196C1
:10DDB000F5011081812F90E00E94DF6F892B11F017
:10DDC0005E01F4CF1D3229F42196F501118101E0A5
:10DDD00007C01B3221F4E5012296F501118100E014
:10DDE000E114F104B1F0F0E1EF16F10429F4B0C050
:10DDF00010E3E114F10401F12AE0E216F104B1F1BB
:10DE000080E1E816F10471F0E8E0EE16F104F1F4B7
:10DE100013C0103341F588818F7D883549F719810A
:10DE200022960260F0E1EF2EF12C88248A94982C3F
:10DE3000A82CAFE0BA2E20C078E0E72EF12C882481
:10DE40008A94982CA82CEFE1BE2E16C06FEF7FEFBE
:10DE5000CB0197010F2C000C440B550B0E946E77E1
:10DE600049015A0109C08AE0E82EF12C69E9862EA1
:10DE7000982CA82C69E1B62E40E060E070E0CB0160
:10DE800027010F2C000C66087708FE0150ED352E97
:10DE9000310E29E0231570F42FEB210F2A3118F4ED
:10DEA00039EC332E06C02FE9210F2A3130F529EA4B
:10DEB000322E310E232D30E02E153F05F4F44F3F66
:10DEC000C9F086169706A806B90688F0A301920144
:10DED0000E945E77232D30E040E050E0620F731F18
:10DEE000841F951F621773078407950710F44FEF7F
:10DEF00001C041E021961081C8CFC114D10451F076
:10DF0000442311F0219703C001FF04C02297F601BA
:10DF1000D183C08300FF07C090958095709561956F
:10DF20007F4F8F4F9F4F4F3F79F482E290E0909365
:10DF30005A0B8093590B3FEF2FEF9FEF0DC040E03E
:10DF400030E020E090E008C0462F372F282F04C093
:10DF5000103309F067CF5FCF642F732F822FDF91CB
:10DF6000CF911F910F91FF90EF90DF90CF90BF90D6
:10DF7000AF909F908F907F906F905F904F903F9069
:10DF80000895FC0188279927E89421912032E9F32C
:10DF9000293010F02E30C8F32B3241F02D3239F4F5
:10DFA000689404C00E945470820F911D21912053E7
:10DFB0002A30C0F31EF4909581959F4F08959111DA
:10DFC0000C945A76803219F089508550C8F708951C
:10DFD000FB01DC018D91059080190110D9F3990B9B
:10DFE0000895FB01DC010D900020E9F711974150E5
:10DFF000504028F0059000200D92C9F708951C921A
:10E000000895FB01DC014150504030F08D910590A6
:10E01000801919F40020B9F7881B990B0895FB01AA
:10E02000DC014150504048F005900D920020C9F7A6
:10E0300001C01D9241505040E0F708954DE45BE06F
:10E040000C942270FA01A191B081009719F41097F5
:10E05000E1F0CD01DC01CD010D90002011F4C001F3
:10E0600013C0FB012191222319F02015D9F7F3CF1A
:10E07000FB012191201519F41E92119606C022234E
:10E08000C1F70D900020A1F7D001FA01A193B08350
:10E090000895BB274A3031F4992322F4BDE29095CC
:10E0A00081959F4F0C945D707AE0979F902D879F8C
:10E0B000802D910D11240895BB27FB015527AA2718
:10E0C000880F991FAA1FA41710F0A41B8395505105
:10E0D000B9F7A05DAA3308F0A95DA193009779F77D
:10E0E000B111B1931192CB010C948576FC0123817F
:10E0F00027FF10C0E3E5FBE0208131818217930701
:10E1000011F41182108232962BE0E935F207A1F763
:10E110000E94896D80E090E008950F931F93CF9344
:10E12000DF93009731F46115710519F480E090E0F8
:10E130003AC08B01EC016EE070E081E090E00E945B
:10E140003E76FC01892B91F380E88383011511054C
:10E1500071F01387028781E883838091530B90913C
:10E16000540B892B21F4F093540BE093530B20971D
:10E17000C9F0D187C0878381826083838091550BEA
:10E180009091560B892B71F4F093560BE093550B3D
:10E190008091570B9091580B892B21F4F093580BD9
:10E1A000E093570BCF01DF91CF911F910F9108950D
:10E1B000CF93DF93EC012B8120FF33C026FF0AC0F1
:10E1C0002F7B2B838E819F8101969F838E838A81F3
:10E1D00090E029C022FF0FC0E881F9818081082EDC
:10E1E000000C990B009719F420622B831AC031960A
:10E1F000F983E8830EC0EA85FB85199597FF09C06E
:10E200002B81019611F080E201C080E1822B8B838B
:10E2100008C02E813F812F5F3F4F3F832E83992778
:10E2200002C08FEF9FEFDF91CF9108950F931F935F
:10E23000CF93DF93CDB7DEB708851985F8018381C9
:10E2400088608383AE01445F5F4F6A857B85C80128
:10E250000E945071F8012381277F2383DF91CF91A2
:10E260001F910F9108950F931F93CF93DF93CDB715
:10E27000DEB708851985F801838188608383AE0144
:10E28000445F5F4F6A857B85C8010E941975F8015C
:10E290002381277F2383DF91CF911F910F910895D1
:10E2A0002F923F924F925F926F927F928F929F92A6
:10E2B000AF92BF92CF92DF92EF92FF920F931F9394
:10E2C000CF93DF93CDB7DEB72B970FB6F894DEBFB1
:10E2D0000FBECDBF6C017B018A01FC011782168243
:10E2E000838181FFCCC1CE0101963C01F60193816F
:10E2F000F70193FD859193FF81917F01882309F4B4
:10E30000BAC1853239F493FD859193FF81917F01E4
:10E31000853229F4B60190E00E949576E7CF912CE2
:10E32000212C312CFFE1F315D8F08B3279F038F441
:10E33000803279F08332A1F4232D20611DC08D320B
:10E3400061F0803369F4232D216016C0832D826033
:10E35000382EE32DE4603E2E2AC0F32DF8601DC058
:10E3600037FC2DC020ED280F2A3040F08E32B9F452
:10E3700036FC81C1232D2064322E19C036FE06C022
:10E380008AE0989E200D1124922E11C0EAE02E9E64
:10E39000200D1124222EF32DF0623F2E08C08C3662
:10E3A00021F4832D8068382E02C0883641F4F701AD
:10E3B00093FD859193FF81917F018111B3CF982FB8
:10E3C0009F7D9554933028F40C5F1F4F9FE39983F2
:10E3D0000DC0833631F0833771F0833509F059C0B1
:10E3E00021C0F801808189830E5F1F4F88248394A8
:10E3F000912C530113C02801F2E04F0E511CF8017B
:10E40000A080B18036FE03C0692D70E002C06FEFBE
:10E410007FEFC5010E947A764C018201F32DFF77D0
:10E420003F2E16C0280122E0420E511CF801A080A8
:10E43000B18036FE03C0692D70E002C06FEF7FEF40
:10E44000C5010E9468764C01F32DF0683F2E8201D1
:10E4500033FC1BC0822D90E088169906B0F4B601FB
:10E4600080E290E00E9495762A94F4CFF50137FC83
:10E47000859137FE81915F01B60190E00E9495760B
:10E4800021102A9421E0821A91088114910471F7D5
:10E49000E8C0843611F0893641F5F80137FE07C02F
:10E4A00060817181828193810C5F1F4F08C0608100
:10E4B0007181072E000C880B990B0E5F1F4FF32DF7
:10E4C000FF763F2E97FF09C09095809570956195D6
:10E4D0007F4F8F4F9F4FF0683F2E2AE030E0A3011F
:10E4E0000E94EA76882E861845C0853731F4232DA0
:10E4F0002F7EB22E2AE030E025C0932D997FB92ED1
:10E500008F36C1F018F4883579F0B5C0803719F02E
:10E51000883721F0B0C0E92FE061BE2EB4FE0DC0F7
:10E52000FB2DF460BF2E09C034FE0AC0292F2660DF
:10E53000B22E06C028E030E005C020E130E002C085
:10E5400020E132E0F801B7FE07C06081718182816D
:10E5500093810C5F1F4F06C06081718180E090E065
:10E560000E5F1F4FA3010E94EA76882E8618FB2DAE
:10E57000FF773F2E36FE0DC0232D2E7FA22E89144D
:10E5800058F434FE0BC032FC09C0832D8E7EA82EB9
:10E5900005C0B82CA32C03C0B82C01C0B92CA4FE14
:10E5A0000FC0FE01E80DF11D8081803321F49A2D0A
:10E5B000997EA92E09C0A2FE06C0B394B39404C0EC
:10E5C0008A2D867809F0B394A3FC11C0A0FE06C082
:10E5D000B21488F4280C922C9B180EC0B21460F46C
:10E5E000B60180E290E00E949576B394F7CFB21422
:10E5F00018F42B1802C0982C212CA4FE10C0B601D0
:10E6000080E390E00E949576A2FE17C0A1FC03C0B3
:10E6100088E790E002C088E590E0B6010CC08A2D42
:10E62000867859F0A1FE02C08BE201C080E2A7FC0F
:10E630008DE2B60190E00E949576891438F4B60117
:10E6400080E390E00E9495769A94F7CF8A94F30144
:10E65000E80DF11D8081B60190E00E949576811051
:10E66000F5CF222009F442CEB60180E290E00E946C
:10E6700095762A94F6CFF6018681978102C08FEFB6
:10E680009FEF2B960FB6F894DEBF0FBECDBFDF9184
:10E69000CF911F910F91FF90EF90DF90CF90BF909F
:10E6A000AF909F908F907F906F905F904F903F9032
:10E6B0002F90089520FD09C0FC0123FD05C022FF15
:10E6C00002C07383628351834083089544FD17C061
:10E6D00046FD17C0AB01BC01DA01FB01AA0FBB1F4D
:10E6E000EE1FFF1F1094D1F74A0F5B1F6E1F7F1F95
:10E6F000CB01BA01660F771F881F991F09C033E04D
:10E7000001C034E0660F771F881F991F3150D1F781
:10E71000620F711D811D911D08950F931F93CF935B
:10E72000DF938C01C8010E94D870EC0197FD08C0EE
:10E730000E94DF6F892BB1F7B801CE010E94D1761C
:10E74000CE01DF91CF911F910F9108958F929F92EB
:10E75000AF92BF92EF92FF920F931F93CF93DF93ED
:10E760008C01D62F7A01B22E0E94D8709C013327DB
:10E770002B32310531F02D32310561F48B2D80685B
:10E78000B82ED15011F480E068C0C8010E94D87042
:10E7900097FDF9CFCB2DCD7F2B2D207309F580333D
:10E7A000F9F4AA24AA94AD0E09F443C0C8010E944A
:10E7B000D87097FD3EC09C012F7D33272835310549
:10E7C00049F4C264D250A9F1C8010E94D87097FFE1
:10E7D00007C02FC0B6FE02C0C26001C0C261DA2D00
:10E7E000812C912C540120ED280F283080F0C4FF9B
:10E7F00004C0B8010E94D17619C02A3040F0C6FF8B
:10E80000F8CF2F7D3FEE320F363098F727504C2F40
:10E81000C501B4010E9466734B015C01C260D15016
:10E8200059F0C8010E94D87097FFDDCFC1FD04C028
:10E83000AACF812C912C5401C7FF08C0B094A0949A
:10E8400090948094811C911CA11CB11C2C2FB501AB
:10E85000A401C7010E945A7381E0DF91CF911F91FB
:10E860000F91FF90EF90BF90AF909F908F90089581
:10E870005F926F927F928F929F92AF92BF92CF9250
:10E88000DF92EF92FF920F931F93CF93DF93CDB759
:10E89000DEB7A0970FB6F894DEBF0FBECDBF5C0108
:10E8A000962E7A01F9018E010F5F1F4F680180E2F9
:10E8B000D8011D928A95E9F7D50113968C9080E0D6
:10E8C00090E0612C712C30E061E070E083FC2591D8
:10E8D00083FE21918F01522E211103C080E090E030
:10E8E00092C02E3511F4009751F1432F50E0481794
:10E8F00059073CF42D3559F12D3219F4772009F1DF
:10E9000003C0772009F46AC0452D46954695469583
:10E91000D601A40FB11D452D47708B0102C0000F19
:10E92000111F4A95E2F7A8015C91452B4C936514A1
:10E9300059F0561410F45394E7CF5A94E5CF31E0D0
:10E9400004C07724739401C0712C0196BFCF772047
:10E9500019F08E8180628E83311103C088248394E4
:10E9600017C0F6019E012F5D3F4F808180958193F6
:10E970002E173F07D1F7F2CFE114F10429F0D701A8
:10E980008C93F70131967F019A94812C9920F9F0AC
:10E99000C5010E94D87097FD18C0FC01FF2723E035
:10E9A000F595E7952A95E1F7EC0DFD1D208130E006
:10E9B000AC014770552702C0359527954A95E2F777
:10E9C00020FDDACFB5010E94D176811087CFE11406
:10E9D000F10411F0D7011C92C80115C0422F4695D1
:10E9E00046954695D601A40FB11D422F47708B0165
:10E9F00002C0000F111F4A95E2F7A8015C91452B58
:10EA00004C93622EA2CFA0960FB6F894DEBF0FBE35
:10EA1000CDBFDF91CF911F910F91FF90EF90DF90CD
:10EA2000CF90BF90AF909F908F907F906F905F90AE
:10EA300008955F926F927F928F929F92AF92BF9252
:10EA4000CF92DF92EF92FF920F931F93CF93DF93BA
:10EA50006C01EB015A01FC0117821682512CF60160
:10EA6000E380FE01E3FC8591E3FE8191182FEF0125
:10EA7000882309F4EEC090E00E94DF6F892B21F01B
:10EA8000C6010E948D73EBCF153241F4FE01E3FC09
:10EA90001591E3FE1191EF01153281F4C6010E9438
:10EAA000D87097FDD4C0412F50E09C013327241724
:10EAB0003507A9F2B6010E94D176CBC01A3239F4DB
:10EAC000E3FC1591E3FE1191EF0101E001C000E0CC
:10EAD000F12C20ED210F2A3080F402606F2D70E0C0
:10EAE00080E090E040E20E946673F62EFE01E3FCB7
:10EAF0001591E3FE1191EF01ECCF01FF03C0F1107E
:10EB000003C0A7C0FF24FA94183619F01C3651F040
:10EB100010C0FE01E3FC1591E3FE1191EF011836E0
:10EB200041F408600460FE01E3FC1591E3FE1191DD
:10EB3000EF01112309F48DC0612F70E082E095E0B0
:10EB40000E945D76892B09F484C000FD07C0F501A1
:10EB500080809180C50102965C0102C0812C912CBD
:10EB60001E3651F4F6014681578160E070E0202F97
:10EB7000C4010E945A7373CF1336A9F401FD02C079
:10EB8000FF24F394C6010E94D87097FD60C08114E1
:10EB9000910429F0F4018083C40101964C01FA9498
:10EBA000F110F0CF50C01B3559F49E01A4016F2D18
:10EBB000C6010E943874EC01892B09F044C03EC0A4
:10EBC000C6010E948D7397FD42C01F3661F128F483
:10EBD000143639F1193651F128C0133771F0153751
:10EBE00001F123C08114910429F0F4016082C40171
:10EBF00001964C01FA94FF2071F0C6010E94D87072
:10EC00003C0197FD08C00E94DF6F892B59F3B601C4
:10EC1000C3010E94D17681149104A9F0F4011082FD
:10EC200012C0006203C0006101C00064202FA40173
:10EC30006F2DC6010E94A673811105C0F601838164
:10EC4000807329F406C000FD0ACF539408CF5520E5
:10EC500019F0852D90E002C08FEF9FEFDF91CF91EB
:10EC60001F910F91FF90EF90DF90CF90BF90AF90EA
:10EC70009F908F907F906F905F9008950F931F9358
:10EC8000CF93DF93869F8001879F100D969F100D75
:10EC90001124C8010E94F16CEC01009729F0A80131
:10ECA00060E070E00E947376CE01DF91CF911F91FA
:10ECB0000F910895992788270895FC01059006165D
:10ECC00021F00020D9F7C00108953197CF010895B0
:10ECD000FC010590615070400110D8F78095909527
:10ECE0008E0F9F1F0895DC0101C06D93415050406D
:10ECF000E0F70895FC016150704001900110D8F7D1
:10ED0000809590958E0F9F1F0895DC01FC01672F61
:10ED100071917723E1F7329704C07C916D937083F2
:10ED20006291AE17BF07C8F308950F931F93CF9357
:10ED3000DF93FB01238121FD03C08FEF9FEF2CC0E8
:10ED400022FF16C04681578124813581421753071F
:10ED500044F4A081B1819D012F5F3F4F3183208317
:10ED60008C93268137812F5F3F4F3783268314C0D2
:10ED70008B01EC01FB010084F185E02D1995892BB5
:10ED8000E1F6D80116968D919C91179701961796EA
:10ED90009C938E931697CE01DF91CF911F910F9187
:10EDA0000895FB01238120FF12C026FD10C08F3F74
:10EDB0003FEF930761F082832F7D206423832681B8
:10EDC00037812150310937832683992708958FEFA2
:10EDD0009FEF0895FA01AA27283051F1203181F1DF
:10EDE000E8946F936E7F6E5F7F4F8F4F9F4FAF4F53
:10EDF000B1E03ED0B4E03CD0670F781F891F9A1F66
:10EE0000A11D680F791F8A1F911DA11D6A0F711D19
:10EE1000811D911DA11D20D009F468943F912AE025
:10EE2000269F11243019305D3193DEF6CF0108950D
:10EE3000462F4770405D4193B3E00FD0C9F7F6CF3E
:10EE4000462F4F70405D4A3318F0495D31FD405206
:10EE5000419302D0A9F7EACFB4E0A695979587959C
:10EE600077956795BA95C9F700976105710508957B
:10EE70009B01AC010A2E0694579547953795279527
:10EE8000BA95C9F7620F731F841F951FA01D0895BF
:10EE9000F999FECF92BD81BDF89A992780B5089562
:10EEA000262FF999FECF1FBA92BD81BD20BD0FB6A6
:10EEB000F894FA9AF99A0FBE01960895DB018F93A0
:10EEC0009F930E94AF77BF91AF91A29F800D911D3C
:10EED000A39F900DB29F900D11240895A1E21A2EC8
:10EEE000AA1BBB1BFD010DC0AA1FBB1FEE1FFF1FEE
:10EEF000A217B307E407F50720F0A21BB30BE40B3E
:10EF0000F50B661F771F881F991F1A9469F7609584
:10EF10007095809590959B01AC01BD01CF0108953E
:10EF2000052E97FB1EF400940E94A77757FD07D08B
:10EF30000E946E7707FC03D04EF40C94A77750958F
:10EF40004095309521953F4F4F4F5F4F08959095D5
:10EF50008095709561957F4F8F4F9F4F08950E94C8
:10EF6000C277A59F900DB49F900DA49F800D911D19
:10EF700011240895B7FF0C94AF770E94AF77821BDE
:10EF8000930B0895A29FB001B39FC001A39F700D82
:10EF9000811D1124911DB29F700D811D1124911DA1
:10EFA0000895EE0FFF1F881F8BBF0790F691E02D8D
:10EFB000199469279627692778278727782708953E
:10EFC0000E94C277332312F48A1B9B0B0C94EA77BE
:10EFD0000E94C277B7FF0895821B930B0895505883
:10EFE000BB27AA270E9407780C9481790E94737925
:10EFF00038F00E947A7920F039F49F3F19F426F412
:10F000000C9470790EF4E095E7FB0C946A79E92F83
:10F010000E94927958F3BA1762077307840795071D
:10F0200020F079F4A6F50C94B4790EF4E0950B2E4B
:10F03000BA2FA02D0B01B90190010C01CA01A0014A
:10F040001124FF27591B99F0593F50F4503E68F1A5
:10F050001A16F040A22F232F342F4427585FF3CFE6
:10F06000469537952795A795F0405395C9F77EF4B7
:10F070001F16BA0B620B730B840BBAF09150A1F000
:10F08000FF0FBB1F661F771F881FC2F70EC0BA0F86
:10F09000621F731F841F48F4879577956795B7950E
:10F0A000F7959E3F08F0B0CF9395880F08F0992709
:10F0B000EE0F9795879508950E94467908F481E0B0
:10F0C00008950E9475780C9481790E947A7958F09D
:10F0D0000E94737940F029F45F3F29F00C946A791B
:10F0E00051110C94B5790C9470790E94927968F35F
:10F0F0009923B1F3552391F3951B550BBB27AA27F1
:10F1000062177307840738F09F5F5F4F220F331F2A
:10F11000441FAA1FA9F335D00E2E3AF0E0E832D0F2
:10F1200091505040E695001CCAF72BD0FE2F29D0F5
:10F13000660F771F881FBB1F261737074807AB07C7
:10F14000B0E809F0BB0B802DBF01FF2793585F4F3C
:10F150003AF09E3F510578F00C946A790C94B57999
:10F160005F3FE4F3983ED4F3869577956795B7951E
:10F17000F7959F5FC9F7880F911D9695879597F929
:10F180000895E1E0660F771F881FBB1F62177307A2
:10F190008407BA0720F0621B730B840BBA0BEE1FB7
:10F1A00088F7E09508950E94DA786894B1110C947C
:10F1B000B57908950E949A7988F09F5798F0B92FF1
:10F1C0009927B751B0F0E1F0660F771F881F991F9C
:10F1D0001AF0BA95C9F714C0B13091F00E94B47911
:10F1E000B1E008950C94B479672F782F8827B85F21
:10F1F00039F0B93FCCF3869577956795B395D9F7F4
:10F200003EF490958095709561957F4F8F4F9F4FFD
:10F210000895E89409C097FB3EF490958095709509
:10F2200061957F4F8F4F9F4F9923A9F0F92F96E952
:10F23000BB279395F695879577956795B795F111C7
:10F24000F8CFFAF4BB0F11F460FF1BC06F5F7F4F64
:10F250008F4F9F4F16C0882311F096E911C0772376
:10F2600021F09EE8872F762F05C0662371F096E87F
:10F27000862F70E060E02AF09A95660F771F881F4E
:10F28000DAF7880F9695879597F90895990F0008F2
:10F29000550FAA0BE0E8FEEF16161706E807F90768
:10F2A000C0F012161306E407F50798F0621B730B03
:10F2B000840B950B39F40A2661F0232B242B252B84
:10F2C00021F408950A2609F4A140A6958FEF811D27
:10F2D000811D089597F99F6780E870E060E00895C8
:10F2E0009FEF80EC089500240A941616170618065E
:10F2F0000906089500240A9412161306140605063A
:10F300000895092E0394000C11F4882352F0BB0FCA
:10F3100040F4BF2B11F460FF04C06F5F7F4F8F4F2D
:10F320009F4F089557FD9058440F551F59F05F3F68
:10F3300071F04795880F97FB991F61F09F3F79F017
:10F3400087950895121613061406551FF2CF469599
:10F35000F1DF08C0161617061806991FF1CF86951B
:10F360007105610508940895E894BB2766277727FF
:10F37000CB0197F908950E94467908F48FEF08951C
:10F380000E94D3790C9481790E94737938F00E949D
:10F390007A7920F0952311F00C946A790C947079A5
:10F3A00011240C94B5790E94927970F3959FC1F362
:10F3B000950F50E0551F629FF001729FBB27F00D23
:10F3C000B11D639FAA27F00DB11DAA1F649F662778
:10F3D000B00DA11D661F829F2227B00DA11D621FC7
:10F3E000739FB00DA11D621F839FA00D611D221F81
:10F3F000749F3327A00D611D231F849F600D211D65
:10F40000822F762F6A2F11249F5750409AF0F1F0E7
:10F4100088234AF0EE0FFF1FBB1F661F771F881F50
:10F4200091505040A9F79E3F510580F00C946A79A5
:10F430000C94B5795F3FE4F3983ED4F386957795C5
:10F440006795B795F795E7959F5FC1F7FE2B880FF6
:10F45000911D9695879597F90895FA01EE0FFF1F74
:10F46000309621053105A1F16115710561F48038EF
:10F47000BFE39B0749F168949038810561F08038BB
:10F48000BFEF9B0741F099234AF5FF3FE1053105A6
:10F49000210519F1E8940894E795D901AA2329F4E4
:10F4A000AB2FBE2FF85FD0F310C0FF5F70F4A695AE
:10F4B000E0F7F73950F019F0FF3A38F49F779F934F
:10F4C0000DD00F9007FC9058089546F00C94707979
:10F4D00060E070E080E89FE308954FE79F775F93D7
:10F4E0004F933F932F930E942D7B2F913F914F91EC
:10F4F0005F910E94C0790C948A7A0E944679880BA9
:10F50000990B089529F416F00C946A790C94B47947
:10F510000C9470790E949A79A8F39638A0F707F8AE
:10F520000F92E8942BE33AEA48EB5FE70E94D67922
:10F530000F920F920F924DB75EB70F920E94757B9C
:10F54000ECEFF1E00E94BC7A4F915F91EF91FF9157
:10F55000E595EE1FFF1F49F0FE57E0684427EE0FC8
:10F56000441FFA95E1F74195550B0E94EF7A0F90F1
:10F5700007FE0C94E37A0895DF93CF931F930F93C4
:10F58000FF92EF92DF927B018C01689406C0DA2E25
:10F59000EF010E94D379FE01E894A5912591359160
:10F5A00045915591A6F3EF010E940778FE0197015E
:10F5B000A801DA9469F7DF90EF90FF900F911F9107
:10F5C000CF91DF9108959B01AC0160E070E080E88D
:10F5D0009FE30C9461780C946A790C94A97B0E9447
:10F5E0009A79D8F39923C9F3940F511DA3F391503D
:10F5F000504094F059F0882332F0660F771F881F2F
:10F6000091505040C1F79E3F51052CF7880F911D36
:10F610009695879597F908955F3FACF0983E9CF0DA
:10F62000BB27869577956795B79508F4B160939554
:10F63000C1F7BB0F58F711F460FFE8CF6F5F7F4F42
:10F640008F4F9F4FE3CF0C94B57916F00C94A97BA4
:10F650000C94707968940C946A790E949A79A8F352
:10F660009923C1F3AEF3DF93CF931F930F93FF92D0
:10F67000C92FDD2788232AF02197660F771F881F5F
:10F68000DAF720E030E040E85FEB9FE3883920F0D4
:10F69000803E38F021968F770E94F077E4E2F2E026
:10F6A00004C00E94F077E1E5F2E00E94BC7A8B0191
:10F6B000BE01EC01FB2E6F5771097595771F880B02
:10F6C000990B0E940B7928E132E741E35FE30E9446
:10F6D000D379AF2D9801AE01FF900F911F91CF917B
:10F6E000DF910E9407780C948179FA01DC01AA0F5E
:10F6F000BB1F9B01AC01BF5728F4222733274427A7
:10F70000507820C0B75190F4AB2F00244695379520
:10F710002795011CA395D2F3002071F0220F331F0F
:10F72000441FB395DAF30ED00C94EF776130710576
:10F73000A0E88A07B94630F49B01AC016627772719
:10F7400088279078309621F0208331834283538339
:10F7500008959F3F31F0915020F4879577956795F4
:10F76000B795880F911D9695879597F9089581E033
:10F7700090E0F8940C94F27C0F931F93CF93DF9357
:10F780008C01FC0101900020E9F7CF01801B910B57
:10F790000E94F16CEC01009719F0B8010E94277CDF
:10F7A000CE01DF91CF911F910F910895FB01DC01F4
:10F7B00004C08D910190801921F441505040C8F748
:10F7C000881B990B08956817790768F4FB01DC0121
:10F7D000E40FF51FA40FB51F02C002900E92415016
:10F7E0005040D8F708950C94E97CFB01DC018D9121
:10F7F00081341CF08B350CF4805E619161341CF017
:10F800006B350CF4605E861B611189F3990B0895CA
:10F81000FB01DC010D900020E9F7119701900D929A
:10F820000020E1F70895FC018191861721F08823DB
:10F83000D9F7992708953197CF010895FB01DC018D
:10F840008D91019080190110D9F3990B0895FB0156
:10F85000DC0101900D920020E1F70895FB01DC012D
:10F860000D900020E9F711974150504028F0019089
:10F8700000200D92C9F708951C920895FB01DC0148
:10F880004150504030F08D910190801919F40020C2
:10F89000B9F7881B990B0895FB01DC0141505040DA
:10F8A00048F001900D920020C9F701C01D9241500F
:10F8B0005040E0F708950F931F93CF93DF93CDB798
:10F8C000DEB72E970FB6F894DEBF0FBECDBF0E8900
:10F8D0001F89888D998D26E02C831A83098397FFD1
:10F8E00002C080E090E801979E838D83AE01445E64
:10F8F0005F4F6A8D7B8DCE0101960E9450714D81C4
:10F900005E8157FD0AC02F813885421753070CF4DA
:10F910009A01F801E20FF31F10822E960FB6F894A9
:10F92000DEBF0FBECDBFDF91CF911F910F91089524
:10F930000F931F93CF93DF93CDB7DEB72E970FB6FC
:10F94000F894DEBF0FBECDBF0E891F8986E08C8381
:10F950001A8309838FEF9FE79E838D83AE01465EF6
:10F960005F4F688D798DCE0101960E945071EF81B5
:10F97000F885E00FF11F10822E960FB6F894DEBFC7
:10F980000FBECDBFDF91CF911F910F910895CF93FF
:10F99000DF93CDB7DEB72E970FB6F894DEBF0FBE5C
:10F9A000CDBF85E08C838C899D899A838983AE0144
:10F9B000485E5F4F6E897F89CE0101960E9419755E
:10F9C0002E960FB6F894DEBF0FBECDBFDF91CF915C
:10F9D0000895FB01DC0102C001900D92415050409E
:08F9E000D8F70895F894FFCF59
:10F9E80003100000C001200000005B0B8000010034
:10F9F800000000044D5154540400000000000000B1
:10FA080000000000000000000000000000000000EE
:10FA1800000000000000000000000000001B32B5DC
:10FA280059065F0C325A3238326832CD32015F00E3
:10FA38000000009332B559065F0C32D43290336817
:10FA480032CD32015F00000000000000000000001D
:10FA580000DF08D11B000000009332B559065F0C87
:10FA680032D43280336832CD32015F000000005258
:10FA78005AB559DF599F5A105AEE59025A000000D8
:10FA8800005F495449065F89434D494A494749003F
:10FA98000000001B5BF85A065F055F00000000F6D7
:10FAA8005AB559065F055FF65AF65AF65A0000002D
:10FAB80000F65AB559065F055F00000000F65AF6D1
:10FAC8005A065FF65AF65AF65AF65AF65AF65AF699
:10FAD8005AF65AF65AF65A00000000C748D34906A3
:10FAE8005FD443B149974970495E4A704E93498241
:10FAF800451B44CC43E948E748C143DD48000000C2
:10FB0800003D5B00000000F65A01005E00000000A6
:10FB18000000008A43D543065F8943A043DE462799
:10FB28004680471148744580489044AD470747BF11
:10FB380046B843A843A443303132333435363738D6
:10FB48003941424344454600000000005233B5594C
:10FB5800065F0C32A53263336832CD32015F4C6FD9
:10FB6800616465642066726F6D20666C61736820DD
:10FB780049503A0020444E533A002047573A002053
:10FB88004D41534B3A000A4E6F204950206461742E
:10FB98006120666F756E6420696E20666C6173689B
:10FBA8000A002F0064653A61643A62653A65663A0C
:10FBB80066653A65640068656C7000736176650017
:10FBC8006C6F616400676574006D6163006B696CDC
:10FBD8006C007265710069700070776400636C6511
:10FBE8006172007265626F6F74000D0A005F737452
:10FBF800617400560052504D004900737700666CDE
:10FC0800740073657400707772002F616C61726D97
:10FC18002F736E7372002F616C61726D2F6F767225
:10FC280068740020002325325825325825325800A0
:10FC38006974656D0073636D640072636D6400655B
:10FC48006D6974004F4E004F464600540053003B08
:10FC5800006E756C6C0066616C7365007472756516
:10FC6800006E616E00696E66006F76660025783AF0
:10FC780025783A25783A25783A25783A257825D18D
:10FC880081006D6170002F636E662F253032782DEC
:10FC9800253032782D253032782D253032782D25B3
:10FCA8003032782D253032782E636F6E6669672E74
:10FCB8006A736F6E0022002D002E002525253278EC
:10FCC8000057495A6E657400726F6F74006F7574CF
:10FCD8000062637374002F726573702F23002F7294
:10FCE80065712F636F6E66003100646D78696E0010
:10FCF800646D78006D6F64627573006974656D7307
:10FD080000746F70696373006D7174740024636F9D
:0EFD18006D6D616E640030002564002C0000EB
:00000001FF
